:10000000206000108D0500009705000021C102004E
:100010009B0500009D0500009F050000C4C2FCEF89
:10002000000000000000000000000000A10500002A
:10003000A305000000000000A5050000A7050000C2
:10004000A9050000AB050000AD050000AF050000EC
:10005000B1050000B3050000B5050000B7050000BC
:10006000B9050000BB050000BD050000BF0500008C
:10007000C105000000000000C3050000C505000028
:10008000C7050000C9050000CB050000CD05000034
:10009000CF050000D1050000D3050000698C0200E7
:1000A000D7050000D9050000DB050000DD050000D4
:1000B000DF050000E1050000E3050000E5050000A4
:1000C000E7050000E9050000EB050000ED05000074
:1000D000EF050000F1050000F3050000F505000044
:0400E000F705000020
:10010000DECEA5ED02003078343038380000000033
:10011000000000000000484D49373030000000006A
:1001200000000000000053696D706C65484D490087
:1001300000000000000000000000000000000000BF
:100140000000000000000507FE00DAF7DECEA5ED96
:100150000200307834303838000000000000000021
:10016000000053504C6174436F6E74726F6C6C6519
:1001700072004170706C69636174696F6E00000099
:10018000000000000000000000000000000000006F
:0801900000000000FE00DAF798
:0402FC0000000000FE
:10030000310002000F000000C100020018000000D0
:10031000C10202000D000000E90302000D00000010
:10032000110502000D0000002D060200140000005F
:10033000152B020014000000D54302001400000039
:100340002D46020013000000FD67020013000000AC
:10035000D56D020013000000A97402001700000010
:10036000AD790200FA000000C97C02000A0000001A
:100370009D8C020001000000918F02000C00000023
:100380000D930200000000006198020009000000C7
:10039000AD98020005000000319A02000400000040
:1003A000199D0200040000004DA50200020000009B
:1003B00005A702001E00000045B00200100000006A
:1003C000A5BB02000E00000081BF02000300000078
:1003D000ADC502000600000065C90200140000005F
:1003E00011E5030012000000FDF003000A00000008
:1003F00059F403000A00000065FC0300140000002B
:100400002502040008000000C90C040017000000C9
:1004100085460400070000002D4D04001000000078
:1004200019520400130000001964040013000000B6
:100430008995040016000000F5ED04001700000087
:10044000F5290500160000001D2B0500170000000F
:10045000A13C050015000000B13D0500170000009B
:100460002F49072291438D462E492F480A1A06D05C
:100470000722914381F30988022282F314882B48D2
:100480002B492C4A00F039F82B482C492C4A00F013
:1004900034F82C482C492D4A00F02FF82C482D49CF
:1004A0002D4A00F02AF82D482D492E4A00F025F853
:1004B0002D482E492E4A00F020F82E482E490022C1
:1004C00000F026F82D482E49091A082903DB0022DE
:1004D0000260043001601F481F49884205D002684D
:1004E000043003B4904703BCF7E700208646EC468F
:1004F00000200021234A9047FEE7884207D0521A85
:1005000005D0037801300B700131013AF9D1704701
:10051000884202D002700130FAE770471A487047EB
:1005200020600010207000102060001078F9060094
:10053000E80000100C0200100000020000000200A1
:10054000841E060078F90600E8000010E80000109C
:100550000006000000060000000600000006000083
:100560000006000000060000D41F0600D41F06008D
:1005700078F906000C020010CC5B0010185C00102B
:10058000205C0010119F0200FFFFFFFF1A481B496B
:100590000160FFF765BFFEE7FEE7FEE7FEE7FEE767
:1005A000FEE7FEE7FEE7FEE7FEE7FEE7FEE7FEE723
:1005B000FEE7FEE7FEE7FEE7FEE7FEE7FEE7FEE713
:1005C000FEE7FEE7FEE7FEE7FEE7FEE7FEE7FEE703
:1005D000FEE7FEE7FEE7FEE7FEE7FEE7FEE7FEE7F3
:1005E000FEE7FEE7FEE7FEE7FEE7FEE7FEE7FEE7E3
:1005F000FEE7FEE7FEE7FEE708ED00E00000000092
:020000021000EC
:1000000000000000000000000000000000000000F0
:1000100000000000000000000000000000000000E0
:100020000000000000000000000000000000224F5F
:10003000F40321B90000008320B78300EC0F018690
:1000400000004A8601004A6800202906AA005729B4
:100050000755005780006BF4030480000000F6028F
:10006000FC0016F602FD0026800072F4030437003F
:100070000000F4300980215CF610FB0D01530227CB
:1000800046463030303030300309F610FB0D015356
:10009000022733333030303030300309F610FB1490
:1000A0000166464F4E546B50726F704E6F726D54B6
:1000B00065787403F610FB16016527464645304502
:1000C0003045300227464636303630363003F6109B
:1000D000FB120163307078023070780231023130E7
:1000E00030250203F610FB0301520309F00500005E
:1000F0000AF101008200FCF00000000AF10A000091
:10010000F00100000A094A05F636FB86FF016AF68F
:100110003BFB03F62482016A9EF639FB8702016AE3
:10012000F63BFB03F62482016A9EF639FB87020147
:100130006AF63BFB06F62482016AF639FB87020168
:100140006AF10500F63BFB06F62482016AF639FBEC
:10015000F10504980000000087020169F63BFB08E6
:10016000F62482016AF639FB02094A04094A05F6B7
:1001700036FB86FF0183F63CFB0186000184018685
:100180000101A309F639FB87020183F63CFBF6392E
:10019000FB87020183F63BFBFFF639FB87050183F2
:1001A000800074F639FB87050183F610FB040153C8
:1001B0000203F00000000A80007509F10704F10550
:1001C000088301CDF1080892F10804910993F10523
:1001D000009A990000007EF61F01E19800000000DF
:1001E00009F10600AA01EC998000007E90F5170045
:1001F000F5180009F10704979A8301CDABF10604C5
:100200009A92F1080409F10507F305F10500F313CB
:10021000F10204F30CF10205F302F10206F1060704
:1002200009F10507F10106F301F10600F304F101FC
:1002300004F312F10105F30BF106070992F105042D
:10024000980000007F979183025A92F108049083EE
:10025000027609830261F1060009830261F1080058
:1002600009B000F10200B001F10201B002F1020296
:10027000B003F1020309F10500800282F10700805A
:100280000282F10100B100F10101B101F10102B1FD
:1002900002F10103B10309F10500F30000F30A00C4
:1002A00000F31104F31700BBF30701F31900F30681
:1002B000F1080092F3210090BDBE02AE09F10510D5
:1002C000AB986100008A8301CD9EF1020C99610018
:1002D000008A92F1081091F10510AB98700000842B
:1002E0008301CD9EF1020D997000008492F10810F7
:1002F000919EF1020E09AA01BA990000008EF61C27
:1003000001BA990000808F979109F30002F311045C
:10031000F30A0000F30497F31A00F3000009F30056
:1003200002F31104F30A0000F304F31900F30000D0
:1003300009F30002F31101F30A0000F304F31800BB
:10034000F3000009F30002F31101F30A0000F304C3
:10035000F31700F3000009F30003F31104F30A009C
:1003600000F30497F31A00F3000009F30003F311FC
:1003700004F30A0000F304F31900F3000009F3008A
:1003800003F31101F30A0000F304F31800F3000073
:1003900009F30003F31101F30A0000F304F317005B
:1003A000F3000009F10500F00300000D09F0000062
:1003B000000D09F00500000DF1010009F007000033
:1003C0000DF106009900000000F61F01BA98000028
:1003D000007E09F10500F00300000B09F0000000A9
:1003E0000B09F00700000BF106009900000000F671
:1003F0001F01BA980000007E099624F610FB020146
:1004000064F609FB0402F610FB0702023002300218
:100410000309F00001000C09F00700000CF10600D0
:100420000999A3D70A7890F10500F00300000CF0B9
:100430000000000C09F430F610FB1501666D7972AE
:1004400069616470726F72656736302E666F6E0315
:10045000F610FB080146632D31023003F610FB1B3A
:1004600001405C43484D493730305C6E53504C611D
:100470007420436F6E74726F6C7303F40280047B9C
:10048000832046F610FB1801405C43484D49373045
:100490003020466163746F7279205465737403F67B
:1004A00010FB0D01650227464630303030303003F6
:1004B000F00600C085F10101F10100F610FB0D010D
:1004C000405C6E4669726D776172653AEF4435EF54
:1004D0004535F60AFBF610FB012EEF4436EF4536A4
:1004E00001F60AFBF610FB0103EF4535F40EF406A6
:1004F000F40260032004FEF4070000C804F0832027
:1005000046F610FB1001405C43546F7563687363DB
:100510007265656E03F610FB0D01650227464630D5
:100520003030303030038320B7F10A0001F0010091
:10053000000AF610FB3C01405C6E546F7563682046
:1005400074686520746F75636873637265656E2E79
:100550002020446F65732069745C6E7265717569E3
:10056000726520726563616C6962726174696E673D
:100570003F03F610FB2B0150310234023002332EC0
:100580003802392E3802526563616C02020202029F
:1005900002022746463130313031300202020E026B
:1005A00003F610FB0701463130023003F610FB2240
:1005B00001404F72206A756D7020737472616967B3
:1005C000687420746F2074686520525443206361FE
:1005D0006C03F610FB2C0150023132023002332E34
:1005E0003802392E3802446F20525443020202026C
:1005F0000202022746463130313031300202020F0A
:100600000203F4026002200626600420062660032E
:10061000200626800602F610FB0401530203F000B8
:1006200000000A8004FEF10A0000F00100000A60E8
:10063000022006166004201C24832046F610FB14BA
:1006400001405C433356332063616C6962726174AC
:10065000696F6E03F610FB0D0165022746463030C8
:1006600030303030038303E2F610FB1401405C6E3F
:100670004578697374696E672043616C203D20037F
:10068000F610FB1101666E6F726D616C626F6C64C7
:100690002E666F6E03F62DF610FB020140EF443517
:1006A000EF45358106AEF609FB05038006B7F61067
:1006B000FB05556E63616CF610FB0103EF45358257
:1006C00006C7980000007E9624F610FB11016673A1
:1006D000797364656661756C742E666F6E03F610CF
:1006E000FB0E01405C6E4E65772043616C203D033C
:1006F000F610FB2A01500233023002332E38023941
:100700002E380255700272323002020202020227B3
:100710004646313031303130020202100203F61009
:10072000FB2C01500237023002332E3802392E38AA
:1007300002446F776E027232300202020202022716
:100740004646313031303130020202110203F610D8
:10075000FB2B0150023302313002372E3802313187
:100760002E38025361766502020202020202274617
:10077000463030464630300202021202038307C878
:10078000F40260032007E2800780F610FB11016687
:100790006E6F726D616C626F6C642E666F6E03F6C5
:1007A00010FB0701463202313003F610FB02014014
:1007B000EF96379424F609FB0503F610FB0103EFCF
:1007C0009437099903126F7594249096248303D368
:1007D00080078A9983126F758007C88303DC6803DA
:1007E0002009832046F610FB1401405C4331365645
:1007F0002063616C6962726174696F6E03F610FB4D
:100800000D01650227464630303030303003830317
:10081000BC9624F610FB1401405C6E457869737435
:10082000696E672043616C203D2003F610FB1101C7
:10083000666E6F726D616C626F6C642E666F6E03B4
:10084000F610FB020140F609FB0503F610FB01035D
:10085000F610FB11016673797364656661756C74DB
:100860002E666F6E03F610FB0E01405C6E4E6577D0
:100870002043616C203D03F610FB2A015002330235
:100880003002332E3802392E38025570027232305F
:100890000202020202022746463130313031300274
:1008A0000202130203F610FB2C0150023702300241
:1008B000332E3802392E3802446F776E027232308E
:1008C0000202020202022746463130313031300244
:1008D0000202140203F610FB2B01500233023130E6
:1008E00002372E380231312E38025361766502020A
:1008F00002020202022746463030464630300202EB
:1009000002150203F610FB0701463132023003F6EE
:1009100010FB520140546869732077696C6C206148
:100920006C736F2061646A7573742074686520311C
:10093000302E3456207261696C2E5C6E5C6E416C98
:10094000736F20636F6E6669726D207468652066D0
:1009500069786564202D3756207261696C2069734F
:10096000206F6B2E038303A4F40260032009CA8066
:100970000968F610FB1101666E6F726D616C626F33
:100980006C642E666F6E03F610FB0701463202316F
:100990003003F610FB020140EF96379424F609FB72
:1009A0000503F610FB0103EF9437099983126F7565
:1009B00094249096248303A48009729903126F757E
:1009C0008009B08303AD68032009832046F610FB3D
:1009D0001C01405C4356636F6D2028332E38562926
:1009E0002063616C6962726174696F6E03F610FB5B
:1009F0000D01650227464630303030303003832108
:100A0000A09624F610FB1401405C6E45786973745F
:100A1000696E672043616C203D2003F610FB1101D5
:100A2000666E6F726D616C626F6C642E666F6E03C2
:100A3000F610FB020140F609FB0503F610FB01036B
:100A4000F610FB11016673797364656661756C74E9
:100A50002E666F6E03F610FB0E01405C6E4E6577DE
:100A60002043616C203D03F610FB2A015002330243
:100A70003002332E3802392E38025570027232306D
:100A80000202020202022746463130313031300282
:100A90000202160203F610FB2C015002370230024C
:100AA000332E3802392E3802446F776E027232309C
:100AB0000202020202022746463130313031300252
:100AC0000202170203F610FB2B01500233023130F1
:100AD00002372E380231312E380253617665020218
:100AE00002020202022746463030464630300202F9
:100AF00002180203832188F4026003200B59800A44
:100B0000F7F610FB1101666E6F726D616C626F6CAF
:100B1000642E666F6E03F610FB0701463202313019
:100B200003F610FB020140EF96379424F609FB050B
:100B300003F610FB0103EF9437099903126F7594C4
:100B400024909624832188800B019983126F7580ED
:100B50000B3F83219168032009832046F610FB2375
:100B6000016330250230250233332E332502323023
:100B70002502030165022746463038303030300305
:100B8000015203F610FB1A01630232302502020201
:100B900003016502274646313030303030030152C0
:100BA00003F610FB1A01630234302502020203012E
:100BB000650227464632303030303003015203F6AA
:100BC00010FB1A016302363025020202030165029E
:100BD00027464634303030303003015203F610FBE4
:100BE0001A0163023830250202020301650227461A
:100BF0004638303030303003015203F610FB240108
:100C00006333332E3325023025020231362E363738
:100C10002502030165022746463030303430300368
:100C2000015203F610FB1D01630231362E363725C3
:100C30000202020301650227464630303038303068
:100C400003015203F610FB1D01630233332E3334CC
:100C5000250202020301650227464630303130305A
:100C60003003015203F610FB1A01630235302502EE
:100C7000020203016502274646303032303030032D
:100C8000015203F610FB1D01630236362E3638255D
:100C9000020202030165022746463030343030300C
:100CA00003015203F610FB1D01630238332E333566
:100CB00025020202030165022746463030383030F3
:100CC0003003015203F610FB21016336362E362520
:100CD0000230250202323025020301650227464612
:100CE00030303030303803015203F610FB1A016304
:100CF00002323025020202030165022746463030E7
:100D00003030313003015203F610FB1A0163023414
:100D1000302502020203016502274646303030309A
:100D2000323003015203F610FB1A016302363025FC
:100D3000020202030165022746463030303034306B
:100D400003015203F610FB1A016302383025020238
:100D50000203016502274646303030303830030147
:100D60005203F610FB0E01633002300231023130C3
:100D700030250203F610FB0D016502274646303090
:100D80003030433003F610FB03015203F610FB032F
:100D9000016303F610FB0F01405C434C43442052B7
:100DA000474235363503F610FB140150300202027B
:100DB0000202020202020202020202020203F40220
:100DC0006103200DBE832046F610FB1A01405C43F0
:100DD0004C434420436F6C6F7572202620436F6E26
:100DE000747261737403F610FB0D016502274646A9
:100DF00030303030303003F610FB130163352502FC
:100E00003025023430250231322E35250203F6100A
:100E1000FB0D01650227464630303030303003F696
:100E200010FB03015203F610FB1601633525023156
:100E3000322E3525023430250231322E352502037B
:100E4000F610FB0D01650227464632343234323447
:100E500003F610FB03015203F610FB140163352562
:100E600002323525023430250231322E3525020377
:100E7000F610FB0D01650227464634383438343805
:100E800003F610FB03015203F610FB160163352530
:100E90000233372E3525023430250231322E3525E6
:100EA0000203F610FB0D0165022746463643364322
:100EB000364303F610FB03015203F610FB140163E3
:100EC000352502353025023430250231322E3525C4
:100ED0000203F610FB0D0165022746463930393012
:100EE000393003F610FB03015203F610FB160163C1
:100EF00035250236322E3525023430250231322E88
:100F000035250203F610FB0D0165022746464234E3
:100F10004234423403F610FB03015203F610FB1473
:100F20000163352502373525023430250231322E52
:100F300035250203F610FB0D0165022746464439AC
:100F40004439443903F610FB03015203F610FB1633
:100F5000016335250238372E35250234302502311C
:100F6000322E35250203F610FB0D01650227464699
:100F700046464646464603F610FB03015203F6106A
:100F8000FB1401633435250230250234302502314B
:100F9000322E35250203F610FB0D01650227464669
:100FA00046464646464603F610FB03015203F6103A
:100FB000FB1701633435250231322E3525023430DA
:100FC000250231322E35250203F610FB0D01650294
:100FD00027464643303030303003F610FB030152D1
:100FE00003F610FB15016334352502323525023432
:100FF00030250231322E35250203F610FB0D016536
:101000000227464643304330303003F610FB0301DD
:101010005203F610FB1701633435250233372E35A2
:1010200025023430250231322E35250203F610FB1D
:101030000D01650227464630304330303003F6104C
:10104000FB03015203F610FB15016334352502350D
:101050003025023430250231322E35250203F610B8
:10106000FB0D01650227464630304330433003F61E
:1010700010FB03015203F610FB1701633435250200
:1010800036322E3525023430250231322E352502F6
:1010900003F610FB0D016502274646303030304321
:1010A0003003F610FB03015203F610FB1501633405
:1010B000352502373525023430250231322E3525CB
:1010C0000203F610FB0D016502274646433030301F
:1010D000433003F610FB03015203F610FB170163C4
:1010E0003435250238372E35250234302502313289
:1010F0002E35250203F610FB0D016502274646300A
:10110000303030303003F610FB03015203F402613B
:101110000320110D832046F610FB200150300230D1
:101120000230023130302502313030250202683180
:101130000202020202020202020203F610FB0D0189
:10114000650227464646464646464603F610FB03DA
:10115000015203F4026103201153832046F610FB71
:10116000200150300230023002313030250231305F
:101170003025020268310202020202020202020269
:1011800003F610FB0D016502274646464630303017
:101190003003F610FB03015203F40261032011999E
:1011A000832046F610FB200150300230023002311D
:1011B000303025023130302502026831020202024D
:1011C00002020202020203F610FB0D01650227462D
:1011D0004630304646303003F610FB03015203F42C
:1011E0000261032011DF832046F610FB20015030FE
:1011F0000230023002313030250231303025020217
:1012000068310202020202020202020203F610FB2D
:101210000D01650227464630303030433003F6106A
:10122000FB03015203F4026103201225832046F6DA
:1012300010FB1001405C434469676974616C20498C
:101240002F4F03F610FB0D01650227464630303064
:1012500030303003F610FB18015030020202020257
:101260000268316431020202020202020202020337
:10127000F610FB0E016331023002330231303025AB
:101280000203F610FB03015203F610FB0301630394
:10129000F610FB050146310203F610FB1C01405419
:1012A000657374696E672C20706C65617365207757
:1012B0006169742E2E2E5C6E03B900B7001E00000B
:1012C00014B2008212ECBAF610FB060140426974B7
:1012D00020EF4435EF4535F60AFBF610FB08206693
:1012E00061696C656403EF453580133D4F00500024
:1012F000548113B3F610FB1D0140556E657870657F
:10130000637465642061637469766520696E7075C5
:10131000743A5C6E03F610FB0701404F503D250305
:101320004F004A08832118F610FB0801402049505D
:101330003D250350004A0883211880133DF610FB19
:1013400018015030020202020202683064300202C8
:10135000020202020202020203F610FB2B015031CC
:101360000234023002332E3802392E3802526574AC
:1013700072790202020202020227464631303130FF
:1013800031300202020E0203F40260032013CC612A
:1013900002201388690220F610FB15015031020269
:1013A00002023002020202020202020202020203EE
:1013B000801254B800BCBA870812BBF610FB0D01AE
:1013C00040492F4F20616C6C206F6B034A004AFF2D
:1013D00051001E000064832046F610FB0B01405CA8
:1013E0004342656570657203F610FB0D01650227C7
:1013F000464630303030303003F610FB2801405C78
:101400006E5072657373204E65787420696620741F
:101410006865206265657065722069732062656524
:1014200070696E67035808F40261032014274308AB
:10143000832046F610FB1A01405C434261636B6CEB
:10144000696768742063616C6962726174696F6E48
:1014500003F610FB0D016502274646303030303070
:1014600030038304189624F610FB1401405C6E458B
:1014700078697374696E672043616C203D2003F6C0
:1014800010FB1101666E6F726D616C626F6C642E81
:10149000666F6E03AA14AAF610FB020140F609FB60
:1014A0000402F610FB01038014B5F610FB0701409F
:1014B0004E6F6E6503830412980000007F8303F96A
:1014C000F610FB11016673797364656661756C745F
:1014D0002E666F6E03F610FB0E01405C6E4E657754
:1014E0002043616C203D03F610FB300150023302B3
:1014F0003002332E3802392E38024272696768741E
:10150000657202723230020202020202274646313E
:101510003031303130020202190203F610FB2E0185
:10152000500237023002332E3802392E3802446915
:101530006D6D6572027232300202020202022746AB
:10154000463130313031300202021A0203F610FB0C
:101550002B0150023302313002372E380231312E46
:1015600038025361766502020202020202274646F1
:101570003030464630300202021B0203831589F4E4
:101580000260032015FE80157FF610FB1101666EC8
:101590006F726D616C626F6C642E666F6E03F61015
:1015A000FB0701463202313003F610FB020140EF27
:1015B00096379424F609FB0402F610FB0103EF941E
:1015C000370994249923D70A7890990000007FF670
:1015D0001D15D8980000007F8303F9801589942495
:1015E00099A3D70A78909900000000F61F15D898A3
:1015F000000000008015D88304216803200983209F
:10160000B7832046F610FB0F01405C43416E616CCE
:101610006F677565205403F610FB0D0165022746C0
:101620004630303030303003983851EC7BAF00F624
:1016300010FB0C01654855456B477265790203F64E
:1016400010FB7201405C6E506C6561736520696EC1
:10165000736572742054206C696E6B7320616E64C4
:101660005C6E696E7374616C6C207468652074655F
:10167000737420706C75672E5C6E28416E4F7574A4
:1016800020746F20416E496E3120616E642076694E
:10169000612034375220746F20416E496E302E29FC
:1016A0005C6E4E657874207768656E207265616443
:1016B000792E2E2E03F40C03206903208318DFF605
:1016C00010FB0A0140302E3330325C6E03F610FB03
:1016D000080140302E323937038F34001E00000AD3
:1016E0006003201717F610FB0A0163370231370237
:1016F000020203B900981AFBA07D831945B901982D
:1017000018129D7D831945F610FB030163032934EC
:101710000316DC1E000064832046F610FB0F014018
:101720005C43416E616C6F677565204903F610FB81
:101730000D01650227464630303030303003984581
:1017400069757CAF00F610FB0C01654855456B4789
:101750007265790203F610FB3D01405C6E506C65CA
:10176000617365206D6F7665206C696E6B73207494
:101770006F20746865204920706F736974696F6E9B
:101780002E5C6E4E657874207768656E2072656198
:1017900064792E2E2E03F40C03206903208318DFB6
:1017A000F610FB0A0140302E3231395C6E03F61020
:1017B000FB080140302E323831038F34001E000008
:1017C0000A60032017F8F610FB0A0163370231376D
:1017D00002020203B90098600D1B7C831945B90110
:1017E000980FDF3B7D831945F610FB030163032946
:1017F000340317BD1E000064832046F610FB0F0162
:10180000405C43416E616C6F677565205603F6104E
:10181000FB0D0165022746463030303030300398EA
:101820000000007EAF00F610FB0C01654855456BCB
:10183000477265790203F610FB3D01405C6E506C07
:1018400065617365206D6F7665206C696E6B7320C2
:10185000746F20746865205620706F736974696FA7
:101860006E2E5C6E4E657874207768656E207265AA
:101870006164792E2E2E03F40C0320690320831853
:10188000DFF610FB080140302E355C6E03F610FBCE
:10189000060140302E35038F34001E00000A60031D
:1018A0002018D5F610FB0A01633702313702020215
:1018B00003B900980000007E831945B90198000023
:1018C000007E831945F610FB0301630329340318D6
:1018D0009A1E0000649800000000AF0080197EF698
:1018E00010FB06014636023003F610FB1D014020B6
:1018F0002020202020204578706563743A20202025
:10190000536565696E673A5C6E03F610FB0B014028
:10191000416E496E303A5C6E03F610FB090140419E
:101920006E496E313A03F610FB0D016527464646B7
:1019300046464646460203F610FB09016337023766
:101940000202020309EE60003401BA9923D70A7833
:101950008320CF01EE66003482196EF610FB02017F
:1019600040F609FB0503F610FB035C6E0309F61055
:10197000FB0B01405061737365645C6E0309832047
:1019800046F610FB0F01405C4354544C20536572E3
:1019900069616C03F610FB0D016502274646303085
:1019A0003030303003F610FB3B01405C6E436F6E0D
:1019B0006E656374206120274E554C4C204D4F447A
:1019C000454D27206361626C655C6E626574776566
:1019D000656E2074686520322054544C20706F72FC
:1019E00074732E03F610FB1D01405C6E434F4D30A7
:1019F000202D3E20434F4D313A2054657374696E5B
:101A0000672E2E2E03F4026003201AC44AFFF63715
:101A1000FDF610FC07313233342E350D1E00000563
:101A20004A0DF636FD86FF1A05F63BFDFF991A5062
:101A30000089F625811A05F610FB060146023134AD
:101A400003F610FB0D01405061737320202020200D
:101A50002003F610FB1D01405C6E434F4D31202DDD
:101A60003E20434F4D303A2054657374696E672EA3
:101A70002E2E03F4026003201AC44AFFF637FCF648
:101A800010FD073637382E32350D1E0000054A0D81
:101A9000F636FC86FF1A73F63BFCFF992990008806
:101AA000F625811A73F610FB06014602313403F65F
:101AB00010FB0D0140506173732020202020200373
:101AC0001E000064832046F610FB1401405C435462
:101AD000544C20587769726520262034383503F637
:101AE00010FB0D01650227464630303030303003A0
:101AF000F610FB4401405C6E436F6E6E65637420AC
:101B00006120484D49343330207769746820746807
:101B1000652058776972652F343835207465737481
:101B2000206170702E5C6E5877697265203D5C6E26
:101B30005253343835203D03F5320010F602FE00D2
:101B400036690520690620980000000096304AFF9B
:101B5000F637FE9816B43893962CF53900600520B8
:101B60001BCEF610FB06014633023803985781C09E
:101B700093F610FE0120F608FE0907F610FE010D8F
:101B800099A000008292ABF4061E0000014A0DF6F7
:101B900036FE87FF1BA0F40700000A1B89801BB2DA
:101BA000F63BFEFF4A0DF636FE0CF637FEF62582B2
:101BB0001BC0F610FB0701404661696C03801BCE19
:101BC000F610FB070140506173730368052060063F
:101BD000201C08F610FB06014632023803942C99AB
:101BE000A0000082929530F625821BFAF610FB07C2
:101BF00001404661696C03801C08F610FB07014038
:101C000050617373036806206003201C1E67052063
:101C100067062004821C1E1E000005801B5DF53631
:101C20001E000032832046F610FB1401405C435234
:101C300054432043616C6962726174696F6E03F68C
:101C400010FB0D016502274646303030303030033E
:101C5000832176F610FB1101667379736465666102
:101C6000756C742E666F6E03F610FB1901405C6E86
:101C70004578697374696E672063616C2076616C66
:101C80007565203D20F609FB0700F610FB0103F601
:101C900010FB0E0163320230023202313030250275
:101CA00003F610FB03015203F610FB250140506CB4
:101CB0006561736520636F6E6E656374207468651B
:101CC00020475053206F7363696C6C61746F722E80
:101CD00003F610FB03016303F40283216D821D04EC
:101CE0006003201F86801CD8F610FB1801503002BC
:101CF000020202020268316431020202020202029E
:101D000002020203F610FB0E0163320230023202BD
:101D1000313030250203F610FB03015203F610FBAD
:101D200019014057616974696E6720666F7220738C
:101D3000746162696C6974792E03F610FB030163A8
:101D4000031E000032F610FB06014632023003F497
:101D500006F40283216D811C24F4070000C81D5184
:101D6000F610FB18015030020202020202683164D0
:101D7000310202020202020202020203F610FB0E0C
:101D80000163320230023202313030250203F61094
:101D9000FB03015203F610FB200140506572666F91
:101DA000726D696E67205254432063616C69627280
:101DB0006174696F6E2E2E2E03F610FB0301630310
:101DC00083215EF4028321640186011DC3F610FBAA
:101DD0000E0163320230023502313030250203F643
:101DE00010FB03015203F610FB03016303F610FB23
:101DF000050146320203081E011DC31E331E771E55
:101E0000B783217FF610FB1E014043616C6962724B
:101E10006174696F6E206F6B215C72475053206351
:101E200079636C65733DF609FB0800F610FB01034E
:101E3000801EEF83217FF610FB1801404E6F204774
:101E400050532031304D487A2C20636F756E746585
:101E50006420F609FB0800F610FB195C72507265ED
:101E6000737320627574746F6E20746F2072657462
:101E700072792E03801F07F610FB39014046616915
:101E80006C656420746F2077726974652063616C7F
:101E900020746F20454550524F4D2E5C7250726534
:101EA000737320627574746F6E20746F2072657422
:101EB00072792E03801F0783217FF610FB240140D7
:101EC00043616E27742063616C20616E79206265C6
:101ED000747465722E5C72475053206379636C652D
:101EE000733DF609FB0800F610FB0103801EEF832B
:101EF0002176F610FB0701402043616C3DF609FB9B
:101F00000800F610FB0103690320690220F610FBAC
:101F100018015030020202020202683064300202EC
:101F2000020202020202020203F610FB2B015031F0
:101F30000234023002332E3802392E3802526574D0
:101F40007279020202020202022746463130313023
:101F500031300202020E0203F4026003201F866188
:101F600002201F07F610FB15015031020202023059
:101F70000202020202020202020202020383216D35
:101F8000811C8F801D60832046F610FB1501405C8C
:101F90004354657374696E6720436F6D706C65742C
:101FA0006503F610FB0D01650227464630303030E0
:101FB000303003F610FB4601405C6E45697468657D
:101FC00072202752657465737427206F7220274E24
:101FD00065787427207361766520726573756C74FB
:101FE0005C6E616E6420746F20737461727420740F
:101FF00068652064656D6F206170702E03F610FBBC
:102000002C0150310233023002332E3802392E387F
:1020100002526574657374020202020202022746CC
:10202000463130313031300202020E0203F40260D8
:1020300002200480610320202D8F06AA8F07550EF1
:10204000FFF402802041690320690220690420F620
:1020500010FB0401530203F610FB2A015030022D3D
:1020600033022D31300233023130024E6578740272
:10207000020202020202274646313031303130027C
:1020800002021C0203F610FB0E0163300230023123
:1020900002313030250203F610FB0D0165022746A0
:1020A0004630303030433003F610FB03015203F664
:1020B00010FB0301630309F610FB130164302E3893
:1020C00002302E320231323002333002310309F154
:1020D0000500F107044A0099000000001E000002FC
:1020E000EEAE0090AB0C018A0A20DC982000008242
:1020F00093F105088320FBF1060809F10800919A85
:10210000F108044AFFF61D01BA4A000968032009D4
:10211000680220096804200903F1020ABB4A01BDD4
:10212000BF21275780211FF1020BF402F1010AF1B0
:10213000010B5206064A0152F610FB020140EF4421
:1021400035EF4535F60AFBF610FB0103EF4535F197
:10215000010B5601F1020B8780212A090109F000C9
:1021600000200009F005002000F1010009F0050140
:102170002000F1010009F007002000F1060009F03D
:1021800007012000F1060009F10500F00300000E30
:1021900009F00000000E09F00500000EF101000931
:1021A000F00700000EF106009900000000F61F0184
:1021B000BA980000007E09F616F4024A04F6138667
:1021C000FF21B9F30000F3030076F62F010821B7D1
:1021D00021F021F621FC22022208220E2214221ACA
:1021E00022202226222C22322238223E2244224A37
:1021F00083016D8021B98321108021B9832114804E
:1022000021B98307C38021B98307D38021B983070C
:10221000DB8021B98309AB8021B98309BB8021B957
:102220008309C38021B9830B3A8021B9830B4A808B
:1022300021B9830B528021B98315C28021B983153E
:10224000DE8021B98315F78021B983210C8021B963
:10225000000000000000007E0000007F8000007F82
:10226000F030042C04FF03FF0007FFFFFFFFFF0017
:102270006400FFFFFFFF03FF0007FFFFFFFFFF00FA
:102280006400FFFFFFFF03FF0007FFFFFFFFFF00EA
:102290006400FFFFFFFF0604000E04000F0400109F
:1022A00004001104001204001304001404001504B7
:1022B000001604001704001804001904001A040092
:1022C0001B04001C040000460049004C004F005253
:1022D00000550058005B005E006100640067006A02
:1022E000006D00700073FFFFFFFFFFFFFFFFFFFFA8
:1022F000FFFFFFFFFFFFFFFFFFFFFFFFFFFFFFFFEE
:10230000FFFFFFFFFFFFFFFFFFFFFFFFFFFFFFFFDD
:10231000FFFFFFFFFFFFFFFFFFFFFFFFFFFFFFFFCD
:10232000FFFFFFFFFFFFFFFFFFFFFFFFFFFFFFFFBD
:020000022000DC
:1000000051B148F21801C2F209014FF480130B609C
:100010004FF480020A60704748F21C03C2F20903E1
:100020004FF480121A604FF480001860704700BFD0
:10003000F0B583B04FF01C0001A94FF0040209F0A5
:1000400033FD4FF08503C8F26813019A9A4234D009
:1000500040F20000CAF2000040F20001CAF20011B2
:1000600007F02EF8D0B94FF008054FF001074AF21B
:100070002014C0F207044FF00006284639463A46DD
:1000800028F07CFB204626F04BFC284631463246C1
:1000900028F074FB204626F043FCEEE74FF0850184
:1000A000C8F2681102A840F8041D4FF004014FF097
:1000B0001C0209F087FD0BF09BFE03B0F0BD00BFF2
:1000C00010B54FF0000108464FF00002134604F04F
:1000D00047F94CF2503026F023FC48F29804C2F263
:1000E00009044FF4003323604CF2503026F018FC22
:1000F0004FF4802020604FF07E5049F69A11C3F6ED
:1001000099614FF078024FF4167304F029F940F228
:100110000003C5F2000340F20C20C1F200001946B2
:1001200040F20002C5F28002D21A4FF46063C0F2BE
:10013000277300F047FE4FF0010001F0F7F943F29A
:100140006460C0F2060001F0C3FA4FF005004FF002
:10015000000140F2ED12C0F202020AF019FF4FF066
:10016000030040F20101C0F2020140F2DD12C0F2D0
:1001700002020AF00DFF47F2A820C0F2060025F0A7
:10018000E7FA4FF060004FF0010109F0B7FD4FF0C2
:1001900003004FF001010A464FF012030AF098F9EC
:1001A00040F23420C1F2000040F20001CAF28001A6
:1001B0004FF480324FF0020331F0E0FD40F24C206A
:1001C000C1F2000044F24401C4F202014FF01402F3
:1001D0004FF0030331F0D2FD10BD00BF08B519B9CF
:1001E0004FF0050033F026FD08BD00BF08B501291A
:1001F00003D14FF0030033F01DFD08BD002817DDCB
:1002000040F23021C1F200010A6883184EF2E80082
:10021000CAF2980040F20001CAF20011091A8B429A
:1002200012D8801840F23022C1F2000213607047E9
:1002300000280CDA40F23023C1F200031A6880185B
:1002400018604FF0000070474FF0FF3070474EF2DB
:10025000E800CAF29800704708B50BF0D5FD08BD5C
:100260004FF03800704700BF41B940F27023C1F22F
:100270000003186810604FF0000070474FF0140042
:10028000704700BF40F27023C1F2000318686FEAA4
:100290000000704708B54FF00100187051B940F2E6
:1002A0007023C1F200031A60114608F0D1FE4FF02E
:1002B000000008BD4FF000021A704FF0140008BD96
:1002C00010B540F27024C1F200044FF04000214606
:1002D0004FF0080209F0E8FBFFF7D4FF63688342A0
:1002E00005D14FF00100216808F0B2FE0EE04FF09A
:1002F00001004FF07C5108F0ABFE40F27020C1F2DB
:1003000000004FF00002CBF6807202604FF00B004D
:1003100047F2C421C0F2060140F26422C1F2000299
:1003200028F070F810BD00BF08B54FF0010313703E
:1003300081B9FFF7A7FF40F27021C1F200014860C8
:1003400008464FF008014FF0400209F03BFC4FF027
:10035000000008BD4FF0000010704FF0140008BD01
:1003600041B940F28423C1F20003186810604FF0D5
:10037000000070474FF01400704700BF40F2842324
:10038000C1F2000318686FEA0000704738B51446E0
:1003900071B940F28423C1F200035D68FFF7EEFFFC
:1003A000854214BF0020012020704FF0000038BDAE
:1003B0004FF0140038BD00BF08B54FF001001870B1
:1003C00061B940F28423C1F200031A604FF00300C8
:1003D000114608F03DFE4FF0000008BD4FF000024E
:1003E0001A704FF0140008BD10B540F28424C1F219
:1003F00000044FF0280021464FF0080209F054FB9A
:10040000FFF7BCFF6368834205D14FF0030021680A
:1004100008F01EFE0EE04FF003004FF07C5108F094
:1004200017FE40F28420C1F200004FF00002CBF62C
:10043000807202604FF00D0047F2F821C0F2060111
:1004400040F27822C1F2000227F0DCFF10BD00BFAD
:1004500008B54FF00103137081B9FFF78FFF40F229
:100460008421C1F20001486008464FF008014FF0B6
:10047000280209F0A7FB4FF0000008BD4FF0000074
:1004800010704FF0140008BD41B940F29823C1F23A
:100490000003186810604FF0000070474FF0140020
:1004A000704700BF40F29823C1F2000318686FEA5A
:1004B0000000704738B5144671B940F29823C1F274
:1004C00000035D68FFF7EEFF854214BF00200120A6
:1004D00020704FF0000038BD4FF0140038BD00BF51
:1004E00008B54FF00100187061B940F29823C1F2CD
:1004F00000031A604FF00400114608F0A9FD4FF008
:10050000000008BD4FF000021A704FF0140008BD43
:1005100010B540F29824C1F200044FF020002146AB
:100520004FF0080209F0C0FAFFF7BCFF636883428E
:1005300005D14FF00400216808F08AFD0EE04FF06D
:1005400004004FF07C5108F083FD40F29820C1F286
:1005500000004FF00002CBF6807202604FF00E00F8
:1005600047F22C31C0F2060140F28C22C1F20002A7
:1005700027F048FF10BD00BF08B54FF0010313700E
:1005800081B9FFF78FFF40F29821C1F20001486066
:1005900008464FF008014FF0200209F013FB4FF01E
:1005A000000008BD4FF0000010704FF0140008BDAF
:1005B00010B5144661B94FF07E5040F2AC23C1F241
:1005C0000003196834F08AF920604FF0000010BD74
:1005D0004FF0140010BD00BF40F2AC23C1F2000385
:1005E00018686FEA0000704708B54FF001001870F6
:1005F000A9B94FF07E50114634F070F9034640F22D
:10060000AC21C1F2000108604FF002004FF0000180
:100610004FF07E5203F0BCFE4FF0000008BD4FF0DB
:1006200000021A704FF0140008BD00BF10B540F270
:10063000AC24C1F200044FF0300021464FF0080214
:1006400009F032FAFFF7C8FF6368834209D14FF01F
:1006500002004FF000014FF07E52236803F098FE35
:100660000FE04FF07E534FF002004FF000011A46AA
:1006700003F08EFE40F2AC20C1F200004FF0804249
:1006800002604FF00C0047F26031C0F2060140F208
:10069000A022C1F2000227F0B5FE10BD08B54FF050
:1006A0000103137011B101291DD110E0FFF794FF70
:1006B00040F2AC22C1F20002506010464FF0080137
:1006C0004FF0300209F07EFA4FF0000008BD4FF005
:1006D0007E534FF002004FF000011A4603F058FE1F
:1006E0004FF0000008BD4FF0000111704FF01400F2
:1006F00008BD00BF6FF00200704700BF4FF001005F
:10070000704700BF4FF00100704700BF4FF001007D
:10071000704700BFC3688B4206D800691A1891421F
:100720008CBF0020012070474FF00000704700BFD1
:1007300048F20C02C4F20802136813F0100FFBD148
:1007400048F20C01C4F208010A6812F0040F0CD040
:1007500048F20801C4F2080148F20C02C4F208028F
:100760000B68136813F0040FFAD148F20C01C4F2BD
:1007700008010A6812F0020FFBD048F20803C4F225
:100780000803186048F20C00C4F20800016811F078
:10079000040FFBD048F20802C4F208021368D8B272
:1007A000704700BF82B048F20C02C4F2080213681E
:1007B00013F0100FFBD100BF00BF48F25800C2F287
:1007C00009004FF4000101604FF014020192019BF7
:1007D0003BB100BF019800F1FF310191019A002A5D
:1007E000F7D102B0704700BF2DE9F04182B0154645
:1007F0001C46C368C91A019148F25C00C2F20900A4
:100800004FF40002026048F20C01C4F208010B68C8
:1008100013F0020FFBD048F20800C4F208004FF0BA
:100820000B0202609DF8061048F20C00C4F20800AA
:10083000036813F0020FFBD048F20802C4F208026A
:1008400011609DF8051048F20C00C4F2080003681E
:1008500013F0020FFBD048F20802C4F20802116044
:100860009DF8041048F20C00C4F20800036813F06D
:10087000020FFBD048F20802C4F2080211604FF0E8
:100880000000FFF755FF75B34FF0000747F2D4366D
:10089000C0F2060605F1FF3808F001083846FFF7F8
:1008A00047FF80EA1461C8B256F8203083EA042476
:1008B000013D1ED117E03846FFF73AFF80EA146386
:1008C000DAB256F8221081EA042405F1FF353846E1
:1008D000FFF72EFF80EA1460C3B256F8232082EAA5
:1008E0000424013DE7D1FFF75DFF204602B0BDE8DB
:1008F000F081B8F1000FDED03846FFF719FF80EA2B
:100900001462D1B256F8210080EA0424013DD2D10C
:10091000E9E700BF2DE9F04F85B00E461C46C368DD
:10092000D21A039248F25C00C2F209004FF40001AF
:10093000016048F20C05C4F208052F6817F0020F99
:10094000FBD048F20803C4F208034FF00B021A6010
:100950009DF80E0048F20C01C4F208010D6815F074
:10096000020FFBD048F20807C4F2080738609DF870
:100970000D0048F20C02C4F20802136813F0020FD3
:10098000FBD048F20801C4F2080108609DF80C7021
:1009900048F20C05C4F20805286810F0020FFBD0DD
:1009A00048F20805C4F208052F604FF00000FFF779
:1009B000BFFE47F2A032C0F20602116848F22403DB
:1009C000C4F20803196047F2D037C0F2060738684E
:1009D00040F28C12C2F20802106040F26011C2F2C2
:1009E00008010D6040F28013C2F2080347F2A437F9
:1009F000C0F206071F6040F28410C2F208000560D2
:100A000047F2F075C0F20605D5F800B047F298320B
:100A1000C0F206021168019147F2D473C0F20603D6
:100A2000186840F6FF7940F6F87840F2641CC2F28C
:100A3000080C40F26C1EC2F2080E40F28C17C2F293
:100A4000080740F27012C2F2080240F29015AA465E
:100A5000C2F2080A4C4594BF21464146CCF80060DA
:100A60004FEA01534FEA1353DEF8005063F30B05CE
:100A7000CEF800503D6863F30B053D60C2F800B04E
:100A8000019BCAF80030641A761811680842FCD13C
:100A9000002CDFD14FF0000048F22402C4F208021B
:100AA000106040F27013C2F20803186040F2901117
:100AB000C2F208010860FFF775FE4FF0010005B0B3
:100AC000BDE8F08F08B548F25C03C2F209034FF4A9
:100AD00000021A6048F20C00C4F20800016811F02C
:100AE000020FFBD048F20803C4F208034FF00602DD
:100AF0001A60FFF757FE08BD10B548F25C03C2F25A
:100B000009034FF400021A6048F20C00C4F2080016
:100B1000016811F0020FFBD048F20804C4F2080487
:100B20004FF0050323601C462046FFF701FE10F03E
:100B3000010F02D023F01AFEF6E7FFF733FE10BDD7
:100B4000F0B583B004461E46089DC068884231D384
:100B500002F1FF33CB1898422CD8276907F1FF37F1
:100B6000C019814226D8834224D3FFF7ABFF48F255
:100B70005C01C2F209014FF400020A6048F20C0065
:100B8000C4F20800036813F0020FFBD048F208011A
:100B9000C4F208014FF060020A60FFF703FEFFF79E
:100BA000ABFF0EB1E068306075B123692B604FF088
:100BB00001000BE000960195204640F6D133C0F2CB
:100BC000020333F08FFA01E04FF0010003B0F0BDF3
:100BD00010B582B04B68C268981A01908968B1F567
:100BE000004F0BD0B1F5803F05D0B1F5805F51D1FA
:100BF0004FF0200404E04FF0D80401E04FF052041D
:100C0000FFF760FF48F25C03C2F209034FF40002F1
:100C10001A6048F20C00C4F20800016811F0020FDB
:100C2000FBD048F20803C4F208031C609DF80600DC
:100C300048F20C02C4F20802116811F0020FFBD056
:100C400048F20803C4F2080318609DF8050048F252
:100C50000C02C4F20802116811F0020FFBD048F236
:100C60000803C4F2080318609DF8040048F20C025F
:100C7000C4F20802116811F0020FFBD048F2080319
:100C8000C4F208031860FFF78DFDFFF735FF4FF042
:100C9000010001E06FF0080002B010BD2DE9F04F37
:100CA00083B015461F461378FF2B1AD1002F73D03F
:100CB00007F1FF3404F001044FF0010312F8016F53
:100CC000FF2E6ED00FE003F10104234612F8016FEE
:100CD000FF2E08D104F1010312F8014FFF2C6DD053
:100CE00001E04FF00003BB4256D0C068091A0191E1
:100CF000CBB2C3F5807B002F4ED048F25C0AC2F223
:100D0000090A4FF4000948F20C04C4F2080448F23E
:100D10000806C4F208064FF00208FFF7D3FECAF82F
:100D20000090226812F0020FFBD0C6F800809DF8F8
:100D30000600216811F0020FFBD030609DF80520FD
:100D4000236813F0020FFBD032609DF80400216885
:100D500011F0020FFBD03060BB4534BF5A463A4613
:100D6000BF1A4AB1A81815F8013B216811F0020F0B
:100D7000FBD033608542F6D1FFF714FDFFF7BCFED0
:100D80004FF000028DF80420019800F58073019364
:100D90004FF4807B002FC0D14FF0010003B0BDE8BD
:100DA000F08FBB42F8D0002C8DD003F1010312F874
:100DB000014FFF2C97D1BB4285D1EDE7BB4282D1D9
:100DC000EAE700BFF0B585B007460E4615464CF27F
:100DD000C402C4F20F02116841F00050106047F2E3
:100DE000A834C0F20604206840F23001C2F20801C3
:100DF00008604CF2C414C4F20F0420686FF3820040
:100E0000206021686FF3C30121604FF0000140F2C0
:100E10006814C2F20804216040F28810C2F208008F
:100E2000016047F2F474C0F20604246840F26C10CA
:100E3000C2F208000460146844F40010106048F224
:100E40001002C4F208024FF00204146047F2AC3002
:100E5000C0F2060002684CF25814C4F20204226088
:100E60004CF26810C4F2020002604CF26C14C4F23E
:100E70000204226047F2B032C0F2060210684CF25F
:100E80005C14C4F2020420604FF4000048F25802DF
:100E9000C2F20902106048F24002C2F2090214686C
:100EA0000443146048F20402C4F20802146861F3B7
:100EB0004104146047F2CC31C0F206010C6848F2DC
:100EC0000001C4F208010C604FEA132345F2C74445
:100ED000C0F21E14A4FB03E34FEA932404F1FF3392
:100EE000DCB20B6864F30F230B6047F29431C0F25D
:100EF00006010C681460136843F00201116048F2A7
:100F00005C02C2F20902106048F20C00C4F2080050
:100F1000046814F0020FFBD048F20803C4F208037F
:100F20004FF09F0119604FF00000FFF701FC4FF0F8
:100F30000000FFF7FDFB4FF00000FFF7F9FBFFF7A4
:100F400031FC48F25C00C2F209004FF4000202607A
:100F500048F20C04C4F20804236813F0020FFBD01B
:100F600048F20801C4F208014FF050000860FFF792
:100F700019FC48F25C04C2F209044FF4000222603A
:100F800048F20C01C4F208010B6813F0020FFBD009
:100F900048F20800C4F208004FF00104046047F270
:100FA0009C32C0F20602117848F20C04C4F2080424
:100FB000236813F0020FFBD048F20800C4F20800C7
:100FC0000160FFF7EFFB4FF00002009247F2B431EF
:100FD000C0F20601019147F2F873C0F206030293D2
:100FE000384631462A4647F2D873C0F2060332F03B
:100FF000E9FF4FF0010005B0F0BD00BF0B4629B17D
:1010000040F2C421C1F200010968196058B140F2F0
:10101000C423C1F20003196840F2B823C1F20003EF
:101020001B68C91A01602AB140F2BC20C1F200005D
:1010300003681360704700BF40F20003CAF2000368
:101040001868B0F1FF3F04D040F20000CAF200007F
:1010500070474FF00000704790B1026802F1030240
:10106000801820F0030140F20003CAF28003994285
:1010700009D24A68B2F1333F0CBF084600207047DE
:101080004FF0000070474FF00000704738B14268E1
:10109000B2F1333F08D1037B4FF0000008E04FF07E
:1010A00002004FF0000303E04FF002004FF0000396
:1010B00001B10B70704700BF18B10068A0F1380093
:1010C00070474FF00000704710B100F110007047FA
:1010D0004FF00000704700BF08B1806870474FF0C4
:1010E0000000704710B100F1380070474FF0000069
:1010F000704700BF024668B31F4B204999422CD26B
:1011000040F20000CAF200004368B3F1333F27D138
:1011100040F20001CAF200018868904226D040F2F5
:101120000000CAF2000040F20001CAF2800102E0B1
:10113000836893421ED0036803F10303C01820F0B4
:10114000030088420FD24368B3F1333FF0D04FF031
:10115000000070474FF0000070474FF000007047EC
:101160004FF0000070474FF00000704740F2000061
:10117000CAF20000704700BF000080A0000000A07D
:101180002DE9F8438046284B284A9A423CD24FF03A
:10119000000540F20004CAF200044FF6FF7640F268
:1011A0000007CAF280076068B0F1FF3F04D12068F1
:1011B000B0F1FF3F34D129E0E189202930D8B0F1E6
:1011C000333F2DD1636B6FEA03022068904227D131
:1011D0002046FFF787FF81462046FFF76DFF024656
:1011E0003046494625F0B4FB218E814218D1A368D0
:1011F0009D4238BF1D46226802F10302A41824F064
:101200000304BC42CFD301E04FF00005B8F1000F5A
:1012100004D0C8F800504FF0000401E04FF0000483
:101220002046BDE8F88300BF000080A0000000A0B9
:1012300010B540F2C023C1F200031C682CB1204657
:101240001DF00EFA2469002CF9D110BD38B5044602
:10125000154600682018821840F20003CAF2800385
:101260009A4208D22A463DF001FE21684D192560B8
:101270004FF0010038BD4FF0000038BD70B5064694
:10128000294B2A4898421CD240F20004CAF20004BA
:101290006368B3F1333F19D140F20004CAF200048D
:1012A00040F20005CAF28005206800F1030024180E
:1012B00024F00304AC420DD26368B3F1333FF3D0A2
:1012C00008E040F20004CAF2000403E040F2000427
:1012D000CAF20004611840F20000CAF280008142A4
:1012E0001ED24FF07735656040F2B421C1F20001A3
:1012F0000B6803F101030B60A360A28104F11005E8
:10130000284631464FF020023BF08CFD28463DF048
:10131000ABFE00F10100E0814FF03802226001E0F5
:101320004FF00004204670BD000080A0000000A027
:10133000F0B583B0044600286CD04368B3F1FF3F9A
:101340006BD0808910F0010F6AD1216801F103058B
:101350002A1922F0030540F20006CAF28006B542BF
:1013600015D26B68B3F1333F13D12E4640F2000023
:10137000CAF28000326802F10302B31823F00306B8
:10138000864207D27268B2F1333FF3D002E02E46B4
:1013900000E02E4606F1380640F20000CAF2800056
:1013A000864240D240F2BC27C1F200073B6803F1FD
:1013B000FF323A6040F2B820C1F200000768791AA3
:1013C0000160771B204629464FEA970208F08CFA05
:1013D0002D1BE0194FF0FF314FEA95020AF076FD20
:1013E000FFF726FF40F20005CAF20005631B40F23A
:1013F0000007C5F20007D819311B01AA6B4632F06D
:1014000053FE0198C21B5119009A32F015FE4FF09D
:1014100000000AE04FF0020007E04FF0020004E095
:101420004FF0030001E04FF0010003B0F0BD00BF3A
:1014300070B504464368B3F1773F46D10068382859
:1014400003D12046FFF774FF70BD4FF03331616068
:10145000C0F1000505F0030520184FF0FF012A46F2
:101460003DF038FD2046FFF73DFE06462046FFF7DB
:1014700023FE02464FF6FF70314625F069FA2086BA
:1014800022686FEA0203636340F20000CAF20000C0
:10149000211A40F20003C5F20003C8182146AA1819
:1014A00032F0CAFD40F2BC20C1F20000026802F135
:1014B0000102026040F2B823C1F2000318682168FB
:1014C000421855191D60FFF7B3FE70BD70B5054693
:1014D000144B154A9A4221D240F20000CAF2000091
:1014E0004168B1F1333F19D140F20004CAF200045F
:1014F00040F20006CAF2800604F1100029463BF0D3
:1015000017FA68B1236803F10303E41824F0030415
:10151000B44203D26268B2F1333FEDD04FF0000421
:10152000204670BD000080A0000000A02DE9F84F0B
:1015300058B940F2B420C1F20000FFF721FED0F10B
:10154000010038BF0020BDE8F88F4FF0030640F2DD
:101550000008CAF2000840F2000BC5F2000B40F28E
:10156000000ACAF2800AC8EB0A0A40F2B429C1F2A2
:1015700000094FF47A7540465946524632F076FDDE
:101580004846FFF7FDFD074660B14FF0FA042846D4
:1015900025F0C6F904F1FF34284625F0C1F9013CD5
:1015A000F5D168E040F20000C5F2000040F2000111
:1015B000C5F280010A1A40F2C423C1F200031A6086
:1015C0004FF0000040F2B821C1F20001086040F283
:1015D000BC22C1F2000210602F4B304898423ED22C
:1015E00040F20001CAF200014A68B2F1333F36D13D
:1015F0004FF000014FF0010040F20003CAF2000377
:1016000040F20005CAF2800500E020461A68C2F1E7
:10161000000404F00304A418091902F103029B1842
:1016200023F00303AB420AD340F2B822C1F2000216
:10163000116040F2BC21C1F2000108600FE000F12E
:1016400001045A68B2F1333FDFD040F2B823C1F24F
:101650000003196040F2BC21C1F20001086040F2B1
:10166000E800C1F2000005F047F8D7F1010038BFEB
:101670000020BDE8F88F013E7FF47DAF40F200020C
:10168000CAF28002D31B38464FF0FF314FEA930273
:101690000AF01CFC86E700BF000080A0000000A04C
:1016A00040F2C023C1F200031A680261186070475B
:1016B00010B503460068824234BF14460446021B3C
:1016C0000846991822463DF0D1FB204610BD00BFC8
:1016D00010B5044647F65800C0F20600FFF7F6FEC4
:1016E000FFF700FD034608B92CB1234640F2C8229B
:1016F000C1F20002136047F66800C0F20600FFF76F
:10170000E5FEFFF7EFFC40F2CC21C1F200010860DA
:10171000C0B940F2C820C1F20000036840F2CC22F8
:10172000C1F2000213606BB947F67801C0F20601FE
:1017300040F2C820C1F20000016040F2CC23C1F2A7
:101740000003196010BD00BF28B940F2CC21C1F2DE
:1017500000010868FFE7008A704700BF28B940F21F
:10176000CC21C1F200010868FFE7B0F90C00704716
:1017700028B940F2CC21C1F200010868FFE7B0F9B6
:101780000E00704728B940F2CC21C1F20001086870
:10179000FFE74089704700BF28B940F2CC22C1F270
:1017A00000021068FFE7438A8B4206D900EB8102F2
:1017B0005369C31801D0984205D142F20B029142FD
:1017C0000DD0416943185A88D988188801FA82F3E4
:1017D0008342C4BF01F1FF30801882B201E04FF0B4
:1017E000000210B2704700BF28B940F2CC22C1F20B
:1017F00000021068FFE7438A8B4206D900EB8102A2
:101800005369C31801D0984205D142F20B029142AC
:1018100003D041694318188870474FF000007047A3
:1018200028B940F2CC21C1F200010868FFE7006846
:10183000704700BF28B940F2CC21C1F2000108680E
:10184000FFE78088704700BF28B940F2CC21C1F281
:1018500000010868FFE7C088704700BF2DE9F04F1E
:1018600089B0BDF8484028B940F2CC26C1F2000644
:101870003068FFE70693468AA64207D900EB840545
:101880006D694519029501D0A84207D142F20B05B6
:10189000AC4200F0C4804469041902940298B0F983
:1018A00002A08A44B0F90410551A0298C28802EBCB
:1018B0000A0601894A19019200F11000009005936F
:1018C000C3F3C400C3F38521C3F3C4439DF81C20B4
:1018D00060F304028DF81C20BDF81C0061F34A106F
:1018E000ADF81C004FEA102163F3C7018DF81D10FD
:1018F0009DF81B80B8F1FF0F04D0019B9D42C0F200
:10190000818089E001998D422EDB85E05446CAEB47
:1019100008076FEA0A0C0CEB060E0EF0010B50469E
:101920002946079A17F80A3001F0ACFD04F10104CA
:10193000A64279DC11E020462946079A3B5D01F07A
:10194000A1FD04F1010420462946079A3B5D01F000
:1019500099FD04F10104A642EDDCC84405F101053E
:101960000198A84204DC57E0CAEB0609DDF80080C4
:10197000B245CBDBF2E75446009FCAEB07076FEA9C
:101980000A0B0BEB060000F0010B17F80A1008FB1E
:1019900001F389FB0312D31850462946079AC3F373
:1019A000C71301F06FFD04F10104A6424BDC1FE0F8
:1019B000385D08FB00F189FB0102531820462946D7
:1019C000079AC3F3C71301F05DFD04F10104385D0C
:1019D00008FB00F389FB0312D31820462946079A17
:1019E000C3F3C71301F04EFD04F10104A642DFDC8E
:1019F000009903980A18009205F10105019BAB427A
:101A000007DC09E048F28109C8F28009CAEB060246
:101A10000392B245AFDBEFE7029D288801E04FF06B
:101A2000000009B0BDE8F08FBBF1000F83D0204665
:101A30002946079A3B5D01F025FD04F10104A64209
:101A40003FF779AF89E7BBF1000FB1D0385D08FBF4
:101A500000F189FB0102531820462946079AC3F377
:101A6000C71301F00FFD04F10104A642A0DCBFE79B
:101A700070B582B0054664460A2804D1DCF814200B
:101A80000D2A06D11DE00D280CD1DCF814100A290E
:101A900017D02369E360A068FFF7C2FE61680818E9
:101AA00060600EE0DCF80800DCF80C10DCF80420C4
:101AB000DCF80030AEB20096FFF7D0FEE3681818ED
:101AC000E06065614FF0000002B070BDF0B591B00C
:101AD00016AD55F8046B08900A91079210AF47F8BD
:101AE000283D0CAC47F64803C0F206030FCB84E850
:101AF0000F00A76041F67120C0F20200E0602046AE
:101B000010A908F01DFA0A9909914FF000020B92F2
:101B1000059503926FF00043029344F0010404948E
:101B200001A831462A463DF0D7FA11B0F0BD00BFFA
:101B3000F0B4DCF8083093422DD9DCF8000000F155
:101B40001800DCF80C3003EB430402FB040213B36F
:101B50004FF000034C784FEA94048E784FEAD60693
:101B6000CD7811F8040B04F007074FEAD00040EAE3
:101B700047101070507820F0070040EAD40066F358
:101B8000C7005070957003F1010302F10302DCF805
:101B90000C009842DED8F0BC704700BF70B4DCF88F
:101BA0000830934225D9DCF8000000F11800DCF879
:101BB0000C304FEA430402FB0402D3B14FF00003A0
:101BC0004D784FEA95058C784FEAD40411F8036BF1
:101BD0004FEAD606108866F3040065F34A1064F3F2
:101BE000CF2022F8020B03F10103DCF80C0098422D
:101BF000E6D870BC704700BF704700BF704700BF99
:101C000010B56446DCF8080020B10DF05FFE4FF01F
:101C10000003A36010BD00BF10B56446DCF80000EF
:101C200020B10DF053FE4FF00003236010BD00BF44
:101C300070B56446DCF8080090B1DCF80430DCF8DC
:101C400000603568D618AE422CBFC3EB05051546BB
:101C5000C0182A463DF00AF961684D19656070BDEB
:101C6000DCF80450AD18CCF8045070BD2DE9F043F9
:101C700083B005460E4664460EF054FFE0602846E9
:101C800031460EF059FFA060284631460EF068FF3D
:101C9000207403280DD0062802D0022854D10BE06E
:101CA00004F1440848F0010848F265594FF0030771
:101CB0000AE0284610F0F4F904F1340040F001087D
:101CC00040F265594FF00207E368B3F5487F84BFDF
:101CD0004FF44873E360A168B1F5F07F84BF4FF41F
:101CE000F071A160A068E26802FB00F007FB00F75A
:101CF000636813B107F11801196007F118000CF0BF
:101D0000EBF9206000B3E368A16840F61F5262F36C
:101D10001F4202602068C0F8049022689360236824
:101D2000D96021680F6120684FF000024261009283
:101D300028461146434610F0A1F8284610F0A2F9B3
:101D40002846314610F0C8F803B0BDE8F08300BF64
:101D50002DE9F04F8DB005460E4691461F469DF881
:101D6000644000690B90002D00F0088340F61F537B
:101D7000C0F61F532A689A4240F000831799002941
:101D800040F3FC82189B002B40F3F882AB68B3420F
:101D900040F3F482002E06DA8A19179200F1EE82DF
:101DA000BF1B4FF00006D5F80CA0CA4540F3E682F1
:101DB000B9F1000F0FDADDF8608018EB0908CDF8F3
:101DC000608000F1DB82DDF858C0C9EB0C09CDF86A
:101DD00058904FF00009B7F5487F80F2CF82002F6E
:101DE00007DA1799CA19179200F1C882F61B4FF04B
:101DF000000740F22841C1F2000109688F4207DA6A
:101E00007A1A179FBF18179700F1B882B61A0F46B3
:101E1000DDF85C80B84440F22841C1F200018A68D4
:101E200008F1FF3C944507DDC8F1010152181799EC
:101E30008A18179200F1A282169AB2F5F07F80F20A
:101E40009D82002A09DA18998918189100F1968262
:101E5000C2EB09094FF00002169240F22841C1F28C
:101E600000014968DDF8588088450ADAC1EB080CA2
:101E7000189A12EB0C02189200F18082CCEB09093F
:101E800016911699DDF86080884440F22842C1F22C
:101E90000002D16808F1FF3C8C4507DDC8F1010262
:101EA0008918189A5118189100F168829E4280F2A0
:101EB0006582D14580F262829B1BC7F548729A42C7
:101EC000B8BF134617998B42B8BF19460091C9EBAA
:101ED0000A02DDF85880C8F5F0739342A8BF134694
:101EE00018998B42B8BF194601916A692AB905F160
:101EF00018014FF0000003900CE00CF0EDF8039097
:101F0000002800F03B820BA905F118026B6917F05D
:101F1000CFF803996B6840F26552934240F0C68057
:101F2000AB68B3F5487F14D1EA68B2F5F07F10D101
:101F30000098B0F5487F0CD1019AB2F5F07F08D136
:101F4000B94800684FF46E42C0F2020207F0CCFCC0
:101F50000FE20098C0EB030AC0F5487B03FB09665B
:101F600001EB46064FF44873169903FB0177AE4A1E
:101F7000106800EB4707FA2C53D946EA070414F01F
:101F8000030F09D04FEA4A0A4FEA4B09009D4FEA76
:101F9000450CA846019D2EE0009A12F0010FF1D1E8
:101FA0004FF0020392FBF3F4DDF804800BE03846B7
:101FB0003146224607F098FCAA6806EB420607F570
:101FC000C86708F1FF38B8F1000FF0D1D1E101F195
:101FD00002044988104620F8021B04F102016488BB
:101FE000548000F10202023BF1D16744664456443A
:101FF0004F4405F1FF35002D00F0BB81009B002B05
:10200000F5D0A6F10202434608F1FF3101F00104C8
:10201000314652883A8007F10202013B40F0B1811B
:10202000E3E7042C40F2A5814FEA4A0A4FEA4B0B42
:10203000009D33E02A463B8803F01F0003F4FC6C4C
:1020400003F47841338803F01F09C0EB090804FB4F
:1020500008F9C9F3042803F4FC69CCEB090909FB6E
:1020600004F94FEA292909F4FC6903F478435B1A5F
:1020700003FB04F34FEA232303F47843CC444044A6
:102080004CEA0000591840EA01033B80013AD2D1E2
:1020900056445F44019800F1FF310191019B002BF0
:1020A00000F0678100990029C4D1F1E748F265503A
:1020B000834240F0BB80AB68009D581BC5F5487259
:1020C00003FB09634FF0030606FB03114FF4487549
:1020D000DDF8588005FB0877534B1D6805EB470377
:1020E0000293019D002D00F0448106FB00F0069054
:1020F0004FEA42070897009806FB00F00590009A07
:1021000002F1FF3506FB05F39F1904974FEA4500DE
:1021100000F10200099048F28105C8F280050A46E4
:1021200065E03146FFE7877804FB07F785FB078604
:10213000F7194FEAE717FEB2042E33D9FA2E02D967
:1021400006880E802EE00E8806F01F0806F4FC6953
:1021500006F4784C0688FFB206F01F0BC8EB0B0A9A
:1021600007FB0AFBCBF3042A06F4FC6BC9EB0B0B51
:102170000BFB07FB4FEA2B2B0BF4FC6B06F47846AA
:10218000CCEB060606FB07F74FEA272707F478474C
:102190000BEB0906D04446EA080607EB0C0946EAB1
:1021A00009070F8000F1030001F10201867804FBAA
:1021B00006F685FB0697BE194FEAE617FEB2042E17
:1021C00040F2AD8178E1DDF810C06244029B0999CC
:1021D00058180290069FD219029BDDF8208003EB6D
:1021E000080702970199481E019000F0C2800099EB
:1021F0000029EFD0DDF8148002EB080302991046A5
:102200009E1AA6F1030606F001070797967804FBCD
:1022100006F685FB0697BE194FEAE616F7B2042FBD
:1022200040F2EF80B9E000BF1804001048F68804BF
:10223000A34240F09E80AD68009BE81AC3F5487247
:1022400005FB096401EB840B4FF44871169D01FBFB
:102250000577D04B1C6804EB4701019B002B00F075
:1022600088804FEA800704974FEA42050595009859
:102270004FEA80020292009C4FEA440306930D4607
:1022800066E013F8010C042847D9FA2816D953F848
:10229000040C0A90C0F38524C0F3C44604F0070779
:1022A000C0F3C40040EA47101070507820F00700D7
:1022B00040EAD40466F3C70454702EE0168806F092
:1022C0001F0706F4FC6C06F4784653F8044CC4F37C
:1022D000C409C7EB090800FB08F9C9F304284FEA51
:1022E000541909F4FC69CCEB090900FB09F94FEA20
:1022F000192909F4FC694FEA142404F47844A41B56
:1023000000FB04F04FEA102404F4784409EB0C00BD
:1023100047443843A6193043108002F1020201F10C
:10232000FF3003F1040313F8011C042940F2F38188
:10233000A9E1DDF80880C344DDF818904D44DDF8CC
:1023400010C0E344059BED18019A501E019010D077
:10235000009F002FF3D00BF104033946284607F104
:10236000FF3909F0010C13F8012C042A40F22A81EC
:10237000DDE0039C14B120460DF0A8FA0DB0BDE8D5
:10238000F08F002C3FF423AE31F8024F7C8002F135
:102390000202013B7FF41BAE27E6FA2F2FD8B1F8DB
:1023A00000B00BF01F080BF4FC690BF4784C178895
:1023B000F6B207F01F0AC8EB0A0B06FB0BFACAF3CA
:1023C000042A07F4FC6BC9EB0B0B0BFB06FB4FEA73
:1023D0002B2B0BF4FC6B07F47847CCEB070707FBC0
:1023E00006F64FEA262606F47847D944D04449EA4F
:1023F000080907EB0C0649EA06070F8001E016887A
:102400000E8000F1030001F1020698423FF4DBAEBA
:10241000079F002F3FF485AE877804FB07F785FB05
:10242000078C67444FEAE7175FFA87F8B8F1040FA3
:1024300038D9B8F1FA0F33D8B6F800B00BF01F094D
:102440000BF4FC6A0BF47848B0F800C0FFB20CF053
:102450001F0BC9EB0B0B07FB0BFBCBF3042BCDF8CE
:102460001CB00CF4FC6BCAEB0B0B0BFB07FB4FEA2D
:102470002B2B0BF4FC6B0CF4784CC8EB0C0C0CFB0A
:1024800007F74FEA272707F47847DA44DDF81CC03E
:10249000E1444AEA090A47444AEA07074F8001E053
:1024A00007884F8000F1030006F10206984218BF2A
:1024B00031467FF438AE86E6FA2E2ED80E8806F026
:1024C0001F0806F4FC6906F4784A0688FFB206F095
:1024D0001F0BC8EB0B0C07FB0CFBCBF3042C06F417
:1024E000FC6BC9EB0B0B0BFB07FB4FEA2B2B0BF425
:1024F000FC6B06F47846CAEB060606FB07F74FEAC4
:10250000272707F478470BEB0906E04446EA08065C
:10251000BA4446EA0A060E8001E006880E8000F101
:10252000030001F1020198427FF4FDAD4BE6FA2A67
:1025300032D82E8806F01F0706F4FC6806F47846A9
:1025400053F8044CC4F3C40AC7EB0A0902FB09FAA6
:10255000CAF304294FEA541A0AF4FC6AC8EB0A0ABF
:1025600002FB0AFA4FEA1A2A0AF4FC6A4FEA142418
:1025700004F47844A41B02FB04F24FEA122404F48E
:102580007842D04409EB070448EA04049219144342
:102590002C8017E01804001053F8042C0A92C2F3A0
:1025A0008524C2F3C44604F00707C2F3C40242EA1A
:1025B00047122A706A7822F0070242EAD40466F3CE
:1025C000C7046C7000F1020203F1040301393FF407
:1025D000B0AEBCF1000F3FF454AE1E4613F8014CF0
:1025E000042C48D9FA2C30D8178807F01F0C07F4B0
:1025F000FC6807F4784753F8046CC6F3C409CCEBC5
:10260000090A04FB0AF9C9F304294FEA561A0AF425
:10261000FC6AC8EB0A0A04FB0AFA4FEA1A2A0AF40F
:10262000FC6A4FEA162606F47846F61B04FB06F40D
:102630004FEA142606F47844D04409EB0C0648EA25
:102640000606E4193443448015E053F8044C0A9418
:10265000C4F38526C4F3C44706F0070CC4F3C404CE
:1026600044EA4C148470507820F0070444EAD60001
:1026700067F3C700507002F1020203F1040301394D
:102680007FF4FFAD55E6FA292FD8168806F01F070C
:1026900006F4FC6C06F4784653F8044CC4F3C40802
:1026A000C7EB080901FB09F8C8F304284FEA5419DD
:1026B00009F4FC69CCEB090901FB09F94FEA192976
:1026C00009F4FC694FEA142404F47844A41B01FBC8
:1026D00004F14FEA112404F4784409EB0C01474457
:1026E0003943A6193143118015E053F8041C0A91AF
:1026F000C1F38524C1F3C44604F00707C1F3C40144
:1027000041EA47111170517821F0070141EAD404E0
:1027100066F3C704547002F1020203F10403411E80
:102720007FF4AFAD05E600BF2DE9F0419CB002900B
:10273000039108920DF11C080CAE47F67014C0F21C
:10274000060494E80F0086E80F00C6F8088041F6FA
:102750006D43C0F20203F36010AD3046294607F026
:10276000EFFB18AF94E80F0087E80F00C7F8088068
:1027700041F63130C0F20200F86038461CA907F07B
:10278000DFFB14AE94E80F0086E80F00C6F808805F
:1027900041F69D31C0F20201F1603046394607F042
:1027A000CFFB94E80F0085E80F00C5F8088041F6DC
:1027B0001942C0F20202EA602846314607F0C0FB27
:1027C0004FF0000107910691059147F68010C0F285
:1027D000060045F0010241F6F933C0F202030FF0A2
:1027E00065FB069028B30DF0AFFE059008B3069880
:1027F0004EF65961C0F205014FF02C020EF036F989
:102800003CF0DAFBA8B94FF0000300930698194694
:102810000CAA42F001020FF031FB06984FF00401C0
:102820000A460FF0E9FB06980599029A039B0FF000
:1028300007FB06A805A94FF000020FF05FFB079801
:102840001CB0BDE8F08100BF2DE9F041ADF51B6D76
:102850000DF51B6747F82C0D0DF5196647F6701539
:10286000C0F2060595E80F0086E80F00B76041F654
:102870003143C0F20203F3600DF51A64304621467D
:1028800007F05EFB95E80F0084E80F00A76041F6B3
:102890000140C0F20200E06020460DF51B6107F028
:1028A0004FFB4FF00001CDF88019CDF87C19CDF821
:1028B0008819CDF88C19DDF88429106830B10BF037
:1028C0000BFCCDF88C09002800F0CC8047F6801076
:1028D000C0F206004FF000010DF51A6343F001024B
:1028E00041F6FD33C0F2020312F070F9CDF8800911
:1028F000002800F0A7800DF027FECDF87C09002805
:1029000000F0A080DDF880094EF65961C0F20501A3
:102910004FF02C020EF0AAF83CF04EFB002840F0DD
:102920009180DDF880094FF000010DF5196444F045
:1029300001020B4612F0F6F84FF0080500954FF033
:10294000020601964FF00007029703970497DDF8FF
:102950008009DDF87C194FF448724FF4F07312F0DF
:1029600005F8DDF88009DDF87C1912F007F940F26E
:102970000004CAF2810404F53B2000F5006706AEAE
:102980004FF0010523460DF11B0104F5C864A04674
:1029900093F800C04FEACC0E0EF0F80E5A7802F011
:1029A00007004FEAC00040EA5C104FEA800002F0E6
:1029B000F8024EEA5E1C01F803CC40EA901001F8E0
:1029C000020C42EA521201F8012C03F1020093F8C2
:1029D00002C04FEACC0E0EF0F80EDB7803F00702CF
:1029E0004FEAC20242EA5C124FEA820203F0F803A5
:1029F0004EEA5E1C01F803CB42EA921201F8022C67
:102A000043EA531301F8013C00F1020301F1030111
:102A10004345BDD1CDF87869DDF880090DF6781110
:102A20002A4612F079F9BC42ACD10DF51B6454F87A
:102A3000300D4FF0000112F0B9F820460DF67C1170
:102A400012F09EF90DF518600DF67C114FF00002A2
:102A50000FF054FADDF88419DDF888090860DDF814
:102A60008C0901E04FF000000DF51B6DBDE8F08111
:102A700030B4034658B940F22844C1F2000447F686
:102A80009012C0F206020FCA84E80F003FE0B0F9CE
:102A9000004040F22842C1F200021460B0F9020086
:102AA0005060B3F90050B3F904106D1805F1FF310F
:102AB0009160B3F90250B3F90630EB1803F1FF331C
:102AC000D360002C06DA40F22842C1F200024FF037
:102AD00000041460002806DA40F22842C1F2000225
:102AE0004FF000005060B1F5487F06DB40F228420D
:102AF000C1F2000240F21F319160B3F5F07F06DBB6
:102B000040F22843C1F2000340F2DF10D86030BC2D
:102B1000704700BF30B585B040F20005CAF28105AC
:102B200028464FF000014FF46E42C0F2020209F055
:102B3000CDF94FF00000FFF79BFF40F21844C1F2BF
:102B40000004256041F6D470C0F206008368C3F526
:102B5000487101EBD173C268C2F5F07101EBD1721B
:102B60004FEA620100916FF00042019202924FF031
:102B7000FF0103914FF000010A464FEA6303FFF79C
:102B8000E7F8104820604FF00003009340F2D42291
:102B9000C1F2000201924FF05001029147F68810F5
:102BA000C0F206004FF0870143F67522C0F2020220
:102BB00021F0B0FC40F23C43C1F20003186005B0C4
:102BC00030BD00BF00B88CA030B440F22842C1F242
:102BD000000214685168956805F101052D1BD26843
:102BE00002F10102521A048041808580C28030BC0B
:102BF000704700BF70B4056840F22844C1F2000479
:102C00002668B54209DAAD1B14686619166040F2F1
:102C10002845C1F200052C6804600E6840F2284582
:102C2000C1F200056C68A64209DA351B1E687419EA
:102C30001C6040F22845C1F200056E680E60006815
:102C400040F22844C1F20004A4681568451904F153
:102C50000106B54203DD201A00F101001060096889
:102C600040F22844C1F20004E0681D684C1900F1EC
:102C70000105AC4203DD411A01F10101196012683E
:102C8000002A05DD18680028D4BF0020012001E0DB
:102C90004FF0000070BC704730B484B00B4699B15F
:102CA000B1F900200092B1F90410541804F1FF3278
:102CB0000292B3F902100191B3F90630CC1804F175
:102CC000FF3203926B4603E040F22843C1F2000357
:102CD00001881A680CB2944205DA848809198A1AA4
:102CE00082801C68048041885A680CB2944205DADC
:102CF000C48809198A1AC2805C684480048821B299
:102D00009A68914203DD4FF00002828008E0B0F93A
:102D1000045049198A4203DC02F10102141B848029
:102D200041880AB2DB689A4203DD4FF00003C3809A
:102D300008E0B0F906401219934203DC03F10103E5
:102D4000591AC180B0F90420002A06DDB0F9060046
:102D50000028D4BF0020012001E04FF0000004B0A3
:102D600030BC704708B5B1F5F07F36DC0029BCBF38
:102D70005B180021B3F5F07F88BF4FF4F073CA18D9
:102D8000B2F5F07FC8BFC1F5F07340F21C40C1F24C
:102D900000000268914204DA40F21C40C1F20000D7
:102DA0000160CB1803F1FF3140F24042C1F2000252
:102DB0001068814204DD40F24043C1F20003196013
:102DC00040F2D021C1F200010A6832B940F23C4021
:102DD000C1F20000006821F065FB08BD00B583B0BA
:102DE000C0F3C401C0F38522C0F3C4409DF8043091
:102DF00061F304038DF80430BDF8041062F34A1146
:102E0000ADF804104FEA112260F3C7028DF80520D7
:102E1000BDF8041040F21840C1F20000006841EA19
:102E200001414FF46E42C0F2020209F04FF84FF038
:102E3000000001464FF0FF321346FFF793FF03B047
:102E400000BD00BF08B540F21F339942A8BF194624
:102E500021EAE171A3F5A0739A42A8BF1A4622EABB
:102E6000E27240F23843C1F200031B7883420DD175
:102E700040F22043C1F200031B688B4206D140F2AE
:102E80002443C1F200031B68934216D040F238433A
:102E9000C1F20003187040F22040C1F2000001604E
:102EA00040F22441C1F200010A604FF000000146E7
:102EB0004FF0FF321346FFF755FF08BD08B5012854
:102EC00008D140F2D021C1F200010A6802F10102EA
:102ED0000A601BE090B940F2D020C1F20000016806
:102EE00001F1FF32026040F21443C1F2000318689E
:102EF00003280BD952B921F039FC07E040F2D02366
:102F0000C1F200034FF000021A600FE040F2D0233C
:102F1000C1F200031868B0F1FF3F01D108F074FF5F
:102F200040F2D021C1F200010A6832B940F23C43BC
:102F3000C1F20003186821F0B5FA08BD10B50446C7
:102F40004FF00000FFF794FD1CB14FF00000FFF7B9
:102F500045FF4FF00200FFF7B1FF4FF000000146C0
:102F60004FF0FF321346FFF7FDFE10BD70B48FB077
:102F7000CCB2C3B2E41A02FB04F448F28103C8F2F3
:102F8000800383FB04652E194FEAE474C4EBE61555
:102F900046198DF80460C1F30725C0F307242E1BE2
:102FA00006FB02F483FB04652E194FEAE474C4EBBC
:102FB000E616C0F3072555FA86F48DF80540C1F3EF
:102FC0000746C0F30745741B04FB02F483FB04654A
:102FD0002D194FEAE474C4EBE514C0F3074555FA24
:102FE00084F48DF806404FEA1064C4EB116101FBD4
:102FF00002F283FB021083184FEAE272C2EBE31184
:1030000054FA81F38DF8073001980FB070BC704707
:10301000F0B583B004464FF00001C4F2BE3131F088
:10302000C9FE28B320464FF00001C4F2DC3131F074
:103030008FFEE8B1204631F0F9FB4FF000024FF46B
:103040000043C4F27B0331F0E3FE01F10046314658
:103050004FF000024FF00003C4F24E0332F0D4F8F8
:1030600031F000FC07464FF07E554FF00006C9E0F6
:1030700020464FF00001C4F2DC3131F09BFE10B36A
:1030800020464FF00001C4F2F53131F061FED0B1BD
:10309000204631F0CBFB4FF000024FF40043C4F266
:1030A0007B0331F0B5FE4FF000024FF00003C4F295
:1030B000490332F0A9F831F0D5FB06464FF07E55B2
:1030C0004FF000079EE020464FF00001C4F2F531BA
:1030D00031F070FE08B320464FF00001C4F2FF311A
:1030E00031F036FEC8B1204631F0A0FB8CA3D3E905
:1030F000002331F08DFE01F100414FF000024FF04E
:103100000003C4F2340332F07FF831F0ABFB054624
:103110004FF07E564FF0000774E020464FF000015C
:10312000C4F2FF3131F046FEF8B120464FF0000105
:10313000C4F2114131F00CFEB8B1204631F076FBFB
:1031400077A3D3E9002331F063FE4FF000024FF480
:103150000043C4F2510332F057F831F083FB0746C5
:103160004FF000054FF07E564CE020464FF0000136
:10317000C4F2114131F01EFE28B320464FF48041C5
:10318000C4F2214131F0E4FDE8B1204631F04EFBBC
:103190004FF000024FF42053C4F2840331F038FEA4
:1031A00001F1004319464FF000024FF48043C4F28E
:1031B000500332F029F831F055FB06464FF0000578
:1031C0004FF07E571EE020464FF48041C4F221416B
:1031D00031F0F0FD60B120464FF00001C4F24341F0
:1031E00031F0B6FD48B94FF000052E462F4609E0F4
:1031F0004FF000052E462F4604E04FF000052E4606
:103200004FF07E5720464FF00001C4F22F4131F0BD
:10321000B9FD10B3204631F009FB02460B464FF0D2
:1032200000004FF4C041C4F2880131F0F1FD3EA32B
:10323000D3E9002331F032FF4FF000024FF00003DA
:10324000C4F2540331F0E0FF39A3D3E9002331F095
:10325000E1FD31F007FB044627E020464FF0000176
:10326000C4F2D23131F05CFDE8B1204631F0DEFA33
:1032700031A3D3E9002331F0CBFD2BA3D3E9002305
:1032800031F00CFF4FF000024FF00003C4F2440392
:1032900031F0BAFF26A3D3E9002331F0BBFD31F0B2
:1032A000E1FA044601E04FF07E543846214631F001
:1032B000ADFB4FF00001C4F27F3131F0A7FB31F0DC
:1032C000DDF907463046214631F0A0FB4FF0000102
:1032D000C4F27F3131F09AFB31F0D0F9064628462E
:1032E000214631F093FB4FF00001C4F27F3131F001
:1032F0008DFB31F0C3F94FF00003FFB267F3070312
:10330000F6B266F30F23C2B262F317439DF80700CB
:1033100060F31F63184603B0F0BD00BFAFF3008039
:103320000000000000E07F40666666666666E63F75
:10333000333333333333D33F0000000000C07740D2
:1033400082B0ADF8042040F22843C1F200031B68AC
:10335000834220DC40F22843C1F200039B6898427C
:1033600019DC40F22843C1F200035B688B4212DC97
:1033700040F22843C1F20003DB6899420BDC4FF4B2
:10338000487303FB010040F21841C1F200010B68D1
:1033900092B223F8102002B0704700BFF0B482B0A0
:1033A000072B6BD940F22844C1F200042468844200
:1033B00064DC40F22844C1F20004A468A0425DDC51
:1033C00040F22844C1F2000464688C4256DC40F2AA
:1033D0002844C1F20004E468A1424FDC4FF4487570
:1033E00005FB010040F21841C1F200010C6804EB3A
:1033F0004001EF2B2DD80F8807F01F0507F4FC665E
:1034000007F47841C2F3C4077F1B03FB07F7C7F338
:1034100004274FEA521C0CF4FC6CC6EB0C0C03FBAB
:103420000CFC4FEA1C2C0CF4FC6C4FEA122202F448
:103430007842521A03FB02F34FEA132202F4784354
:1034400066447D193543591845EA010224F81020D5
:1034500014E00192C2F38525C2F3C44605F00703C8
:10346000C2F3C40242EA431304F81030487820F053
:10347000070242EAD50366F3C7034B7002B0F0BC03
:10348000704700BFF0B482B0ADF80420072B58D9C4
:1034900040F22842C1F200021268824251DC40F23E
:1034A0002842C1F20002926890424ADC40F228426F
:1034B000C1F2000252688A4243DC40F22842C1F263
:1034C0000002D26891423CDCBDF80420092B38D9B7
:1034D0004FF4487404FB010140F21840C1F20000AF
:1034E000046804EB4100EF2B29D8078807F01F057B
:1034F00007F4FC6607F4784002F01F077F1B07FB08
:1035000003F7C7F3042702F4FC6CC6EB0C0C0CFBAE
:1035100003FC4FEA1C2C0CF4FC6C02F47842121AE7
:1035200002FB03F34FEA132303F4784266447D1948
:103530003543101845EA000324F8113001E024F85F
:10354000112002B0F0BC70472DE9F04F87B007465C
:103550000C4600929B46109DC5F3C400C5F385211F
:10356000C5F3C4429DF8143060F304038DF81430A1
:10357000BDF8140061F34A10ADF814004FEA1021B1
:1035800062F3C7018DF815104FEA15655C4505DD3E
:1035900022465C4693463B46009F009338462146B0
:1035A000059A2B46FFF76EFF0098C21B46BF52429A
:1035B0004FF0FF360126BBEB040A27D1002A00F0AA
:1035C0002781934602F1FF3101F00108BF19384607
:1035D0002146059A2B46FFF755FFBBF1010B40F042
:1035E0001A8115E1BF1938462146059A2B46FFF787
:1035F00049FF0BF1FF3BBF1938462146059A2B4680
:10360000FFF740FFBBF1010BECD101E132BB0AF146
:10361000FF3606F0010604F1010438462146059AFA
:103620002B46FFF72FFFBAF1010A40F00481EFE0CB
:1036300004F1010438462146059A2B46FFF722FF84
:103640000AF1FF3A04F1010438462146059A2B4657
:10365000FFF718FFBAF1010AEAD1D9E0524529D1A2
:103660000AF1FF3E0EF00108BF1904F101043846CB
:103670002146059A2B46FFF705FFBAF1010A40F0F3
:10368000EA80C5E0BF1904F1010438462146059AD5
:103690002B46FFF7F7FE0AF1FF38BF1904F10104CA
:1036A00038462146059A2B46FFF7ECFEB8F1010A91
:1036B000E8D1ADE0524554DA4FEA022191FBFAF02D
:1036C000C3B20193BAF1010ACDF808A000F09B80C3
:1036D00048F2810AC8F2800A029A02F1FF3808F023
:1036E00001099846002B40F0C980C6E0CDF80CB027
:1036F000DDF808B003E0CDF80CB0DDF808B0019AB1
:1037000008EB020E5FFA8EF9C14598BFBF1904F1AC
:103710000104C9F1FF0305FB03F38AFB0310C11881
:103720004FEAE372C2EBE11338462146059ADBB259
:10373000FFF7A8FE05FB09F08AFB00121318B81961
:103740002146059AC3F3C713FFF79CFE0BF1FF3B1D
:10375000019909EB010C5FFA8CF8C84500F2E4808E
:10376000E1E04FEA0A4ABAFBF2FA5FFA8AF1019104
:10377000531E029347D048F28108C8F2800803F133
:10378000FF3000F0010A8946002940F0F580F1E0A1
:10379000CDF80CB0DDF808B003E0CDF80CB0DDF8E2
:1037A00008B0019A09EB020E5FFA8EFACA4598BF7B
:1037B0000134BF19CAF1FF0305FB03F388FB0310B3
:1037C000C1184FEAE372C2EBE11338462146059A6D
:1037D000DBB2FFF757FE05FB0AF088FB0012131857
:1037E000384604F10101059AC3F3C713FFF74AFEF7
:1037F0000BF1FF3B01990AEB01095FFA89F9D14509
:1038000000F212810EE100985946059AFFF798FDE3
:1038100007B0BDE8F08FB8F1000F3FF4E3AEBF1979
:1038200038462146059A2B46FFF72CFEBBF1010BCB
:103830007FF4D8AEECE7002E3FF4FAAE04F10104B9
:1038400038462146059A2B46FFF71CFEBAF1010ABD
:103850007FF4EEAEDCE7B8F1000F3FF413AFBF1911
:1038600004F1010438462146059A2B46FFF70AFE6B
:10387000BAF1010A7FF406AFCAE7BF1904F10104E7
:10388000C8F1FF0005FB00F08AFB001319184FEA8E
:10389000E072C2EBE11338462146059ADBB2FFF72E
:1038A000F1FD05FB08F08AFB00121318B819214638
:1038B000059AC3F3C713FFF7E5FD0299481E02906E
:1038C000A1D0B9F1000F3FF411AF019A08EB020C3F
:1038D0005FFA8CF9C14598BFBF1904F10104C9F121
:1038E000FF0305FB03F38AFB0310C1184FEAE372E1
:1038F000C2EBE11338462146059ADBB2FFF7C2FD61
:1039000005FB09F08AFB00121318B8192146059A25
:10391000C3F3C713FFF7B6FDC8460299481E0290CD
:103920007FF4E9AE6FE7BF1904F10104C8F1FF00AD
:1039300005FB00F08AFB001211184FEAE073C3EB9D
:10394000E11338462146059ADBB2FFF79BFD05FBE4
:1039500008F08AFB00121318B8192146059AC3F320
:10396000C713FFF78FFDBBF1010B7FF4C8AEDDF885
:103970000CB048E704F10104BF19C9F1FF0305FBCE
:1039800003F388FB0312D1184FEAE370C0EBE11395
:1039900038462146059ADBB2FFF774FD05FB09F0B6
:1039A00088FB00121318384604F10101059AC3F38D
:1039B000C713FFF767FD0299481E02903FF423AF3B
:1039C000BAF1000F3FF4E4AE019A09EB020C5FFA82
:1039D0008CFACA4598BF0134BF19CAF1FF0305FB31
:1039E00003F388FB0310C1184FEAE372C2EBE11343
:1039F00038462146059ADBB2FFF744FD05FB0AF085
:103A000088FB00121318384604F10101059AC3F32C
:103A1000C713FFF737FDD1460299481E02907FF485
:103A2000BCAEF0E604F10104BF19C9F1FF0005FBCB
:103A300000F088FB001211184FEAE073C3EBE113AA
:103A400038462146059ADBB2FFF71CFD05FB09F05D
:103A500088FB00121318384604F10101059AC3F3DC
:103A6000C713FFF70FFDBBF1010B7FF49AAEDDF832
:103A70000CB0C8E62DE9F04383B040F2D027C1F284
:103A8000000740F21445C1F20005DFF8B88120F0CC
:103A9000D7FC3B6823B12B6803F101032B60F6E7E9
:103AA0004FF00000286040F21C41C1F200010A689A
:103AB000002A06DA40F21C44C1F200044FF000066E
:103AC000266040F24043C1F200031868B0F5F07F71
:103AD00006DB40F24041C1F2000140F2DF120A6011
:103AE00040F21C44C1F2000424684FF4C86340F261
:103AF0004046C1F200063068011B01FB03324FEA69
:103B0000920603FB04F404EB86004FF43843C0F242
:103B10000B03984201D908F077F940F20001CAF28C
:103B20008101081908EB0401324605F0DDFE40F280
:103B30003844C1F200042278002A73D040F21846BB
:103B4000C1F2000640F20000CAF28100306040F28B
:103B50002443C1F200031C6840F21C41C1F2000181
:103B60000E68B4422BDB40F24042C1F20002106802
:103B7000844224DC4FF0FF3300934FF000002146D5
:103B800040F21F322346FFF7DFFCB4F5EF7FD4BFCE
:103B9000013404F1FF3440F22441C1F200010C6011
:103BA00040F22444C1F2000423684FF07F420092A7
:103BB0004FF00000194640F21F32FFF7C5FC40F2FB
:103BC0002040C1F20000046840F24043C1F200030B
:103BD000D3F800904FF0FF31009120463146224645
:103BE0004B46FFF7B1FC40F21E329442D4BF013481
:103BF00004F1FF3440F22040C1F20000046040F2C2
:103C00002044C1F2000422684FF07F430093104625
:103C100031464B46FFF798FC40F21846C1F20006C9
:103C2000C6F8008040F21C41C1F200016FF0004272
:103C30000A6040F24040C1F200004FF0000404600E
:103C400025E700BF00B88CA02DE9F04F8BB007909E
:103C5000069105920493149C0894C4F3C40600963C
:103C6000C4F385260296C4F3C4454FEA14649DF854
:103C70005430002B00F08E8007A806A905AA04ABDB
:103C8000FEF7B8FF002800F09381DDF818B0049922
:103C90000BEB01039B4580F28B814FF4487707FBC8
:103CA0000BF6039640F21848C1F20008CDF804B0B4
:103CB000009E029FCDF80080079B05981A1893423A
:103CC0005ADADDF80CC00CEB03014FEA41029DF813
:103CD000240066F304008DF82400BDF8241067F377
:103CE0004A11ADF824104FEA112065F3C7008DF892
:103CF0002500BDF82410092C35D9DDF800C0DCF80A
:103D0000000000EB020CEF2C2CD8BCF800A00AF04D
:103D10001F080AF4FC690AF4784C01F01F0BC8EB89
:103D20000B0A04FB0AFBCBF3042A01F4FC6BC9EB7E
:103D30000B0B04FB0BFB4FEA1B2B0BF4FC6B01F48E
:103D40007841CCEB010104FB01F14FEA112101F4B0
:103D50007841D944D04449EA08088C4448EA0C0127
:103D6000815200E0815203F1010302F10202059940
:103D7000079841189942AADC019800F101000190CE
:103D8000039B03F5487203920499069B5A188242DA
:103D900092DC0DE1069F049839188F4280F28180F1
:103DA00040F22841C1F2000140F21842C1F2000283
:103DB00001924B68BB426ADCC868B84267DB079B6C
:103DC000059A9818834262DA4FF4487606FB073268
:103DD0004FEA42020868984250DC8E689E424DDBF2
:103DE0009DF82400009E66F304008DF82400BDF8C1
:103DF0002400029E66F34A10ADF824004FEA10201A
:103E000065F3C7008DF82500BDF82400092C35D9CD
:103E1000DDF804C0DCF8006006EB020CEF2C2CD8B7
:103E2000BCF800A00AF01F080AF4FC690AF4784CF8
:103E300000F01F0BC8EB0B0A04FB0AFBCBF3042AB0
:103E400000F4FC6BC9EB0B0B04FB0BFB4FEA1B2BC9
:103E50000BF4FC6B00F47840CCEB000004FB00F0AA
:103E60004FEA102000F47840D944D04449EA0809C8
:103E7000604449EA0000B05200E0B05203F101038F
:103E800002F102020598079E30189842A2DC049ABB
:103E9000012A06D002F1FF33FF1806981218BA4221
:103EA00087DC079F05997B189F4280F2818040F252
:103EB0002841C1F2000140F21840C1F20000019017
:103EC0000A68BA426ADC8B68BB4267DB069B0498CF
:103ED0001A18934262DA4FF4487606FB03704FEAF1
:103EE00040024E689E4250DCC86898424DDB9DF807
:103EF0002400009E66F304008DF82400BDF8240021
:103F0000029E66F34A10ADF824004FEA102065F3D4
:103F1000C7008DF82500BDF82400092C35D9DDF83F
:103F200004C0DCF8006006EB020CEF2C2CD8BCF8C7
:103F300000A00AF01F080AF4FC690AF4784C00F0AB
:103F40001F0BC8EB0B0A04FB0AFBCBF3042A00F49B
:103F5000FC6BC9EB0B0B04FB0BFB4FEA1B2B0BF4AD
:103F6000FC6B00F47840CCEB000004FB00F04FEA5F
:103F7000102000F47840D944D04449EA080960444C
:103F800049EA0000B05200E0B05203F1010302F52B
:103F9000C8620498069E30189842A2DC059A012A4D
:103FA00006D002F1FF33FF1807981218BA4287DCD7
:103FB0000BB0BDE8F08F00BF2DE9F04F83B0044691
:103FC0000D460C9F002A62DD002B60DD00EB02082D
:103FD00008F1FF3801EB030B184630F013FA0246E4
:103FE0000B4639A1D1E9000131F00EF930F03AFC6D
:103FF00081465D454BDA6FEA050606EB0B0000F0E3
:1040000001064FF00000494630F06AFC824630F06D
:1040100035FBC2B238460D99FEF7A8FF0090204646
:10402000294642462B46FFF78FFA05F10105AB45BD
:1040300030DC2CE05046494630F052FC824630F0ED
:104040001DFBC2B238460D99FEF790FF0090204646
:10405000294642462B46FFF777FA05F101052E4621
:104060005046494630F03CFC824630F007FBC2B275
:1040700038460D99FEF77AFF0090204629464246C1
:104080002B46FFF761FA05F10105AB45D2DC03B021
:10409000BDE8F08F002ECDD05046494630F020FCD0
:1040A000824630F0EBFAC2B238460D99FEF75EFF59
:1040B00000902046294642462B46FFF745FA05F177
:1040C0000105AB45B6DCE2E70000000000E06F4010
:1040D00038B530B340F24444C1F2000424682046AD
:1040E0004FF0000130F034FE28B140F24C40C1F2F4
:1040F0000000006838BD40F28445C1F200052D681B
:1041000040F28043C1F200031868294630F0E6FB14
:104110000146204630F07AFC0146284630F0E0FBAC
:1041200038BD40F25043C1F200031C6820464FF0F6
:10413000000130F00DFE28B140F24C42C1F2000205
:10414000106838BD40F28440C1F20000056840F2BA
:104150008041C1F200010868294630F0BFFB0146EA
:10416000204630F053FC0146284630F0B9FB38BDFC
:1041700008B540F27C43C1F200031868B0B140F2C8
:10418000F401C1F20001087840F24C42C1F2000291
:10419000116804F05DFF4FF0000000F0ABF940F251
:1041A0004843C1F200034FF00000187008BD00BF83
:1041B00010B582B040F25443C1F20003186848B30E
:1041C00040F2F401C1F200010C784FF00000FFF75B
:1041D0007FFF0146204604F03BFF40F24843C1F216
:1041E00000034FF001021A7040F27C40C1F200005F
:1041F000016879B14FF000030093019340F25840F9
:10420000C1F200004FF0FF0244F27113C0F202034A
:1042100020F022FF02B010BD10B4044628B140F2D5
:104220004440C1F200000068206029B140F25040D3
:10423000C1F20000006808602AB140F25441C1F2A6
:104240000001086810602BB140F27C42C1F200020C
:104250001168196010BC70470246C8B140F248436B
:10426000C1F200031878012808D002280DD140F2CD
:104270004443C1F200031868106009E040F2504165
:10428000C1F200010B68136002E04FF00001116001
:1042900040F24842C1F200021078704730B583B056
:1042A00040F2F403C1F200031878052852D040F21E
:1042B0004841C1F200010C781CB94FF0010000F038
:1042C00019F940F2F402C1F2000215784FF0010032
:1042D000FFF7FEFE0146284604F0BAFE40F24843CE
:1042E000C1F200034FF00200187040F25441C1F2D5
:1042F0000001096881B14FF000000090019040F288
:104300005840C1F200004FF0FF0244F2B113C0F276
:10431000020320F0A1FE1FE040F27C42C1F2000245
:10432000116881B14FF000030093019340F25840AF
:10433000C1F200004FF0FF0244F27113C0F2020319
:1043400020F08AFE08E040F25840C1F2000020F060
:10435000DDFD01E04FF00004204603B030BD00BF9A
:1043600010B540F24444C1F20004206040F25040D5
:10437000C1F20000016040F25441C1F200010A6044
:1043800040F27C42C1F200021360FFF787FF10BDCC
:1043900010B540F2F404C1F20004207040F28040F5
:1043A000C1F20000016040F24C41C1F200010A601C
:1043B00040F28442C1F2000213604FF07E5049F691
:1043C0009A11C3F699614FF078024FF41673FFF714
:1043D000C7FF10BD10B54CF2C403C4F20F031A6836
:1043E00042F00100186047F60821C0F206010C688F
:1043F00048F20803C2F208031C6047F60022C0F22C
:10440000060210684CF2B811C4F20F0108604CF2B9
:104410008814C4F20F042368C3F38102C3F381201C
:10442000904208DC02F1010262F38B234CF2881106
:10443000C4F20F010B6047F60424C0F206042168A1
:1044400047F6A410C0F20600A0F1040400F15400E5
:1044500004F104026368196002F1040452681160F7
:104460008442F5D14CF20811C4F20201086840F40C
:1044700000730B6047F60C24C0F20604226848F271
:104480000001C2F208010A6047F6FC10C0F2060003
:10449000046848F20403C2F208031C6048F21001E9
:1044A000C2F2080140F20002CAF281020A6047F635
:1044B000A010C0F20600036848F21804C2F2080413
:1044C000236048F22001C2F209010A6842F4006048
:1044D000086048F23C03C2F209034FF4006119601E
:1044E00042F2107022F01CFA226842F40060206050
:1044F00010BD00BF10B580B148F21804C2F2080424
:10450000216841F0010222604FF0640022F008FAB5
:10451000236843F40060206010BD48F21804C2F222
:10452000080423686FF3CB2323604FF0640022F06C
:10453000F7F920686FF30000206010BD08B503682C
:10454000196B4068884740F28840C1F200004FF084
:10455000000280F8642008BD2DE9F04F87B00546C1
:104560008B4601929A4640F2F043C1F200031C6868
:10457000E4B14FF00007B846B9464FF6FF76B542B2
:1045800003D020680188A9420CD1226893684BB1FE
:1045900005A804A903AA984705988144049988446A
:1045A000039ABF186468002CE9D103E04FF00007BC
:1045B000B846B946BBF1000F01D0CBF80090019B83
:1045C0000BB1C3F80080BAF1000F01D0CAF8007037
:1045D00007B0BDE8F08F00BF2DE9F04105460F465A
:1045E000904640F2F043C1F200031C68A4B14FF0C2
:1045F00000024FF6FF76B54203D020680188A94239
:1046000006D12368996A19B138468847024628B905
:104610006468002CEFD101E04FF00002B8F1000F08
:1046200001D0C8F800202046BDE8F08108B54FF061
:10463000020047F66031C0F2060146F23162C0F274
:10464000020221F0B1F808BDF0B591B004468569C9
:10465000436943B14FF0000141616A68002A00F0EC
:10466000C9809047C6E0C068002800F0C3804FF0C2
:104670000001E160206869464FF0400221F0A4FB90
:104680000246AB681BB1204669469847B2E0A5696F
:10469000BDF80400012840F0AD8000998A4240F046
:1046A000A9804FF0000EC5F804E0C5F81CE0C5F87D
:1046B00020E0C5F80CE005F124066F460FCF0FC6C9
:1046C00097E80F0086E80F00C5F844E042F20102C7
:1046D000A5F84A2005F1500071464FF014023AF057
:1046E000F9FB6B8D41F20900834277D01CD841F26F
:1046F00004018B423ED009D841F20202934275D0A8
:1047000076D802F1FF30834254D159E041F20601DC
:104710008B4233D030D301F101018B4230D001F113
:1047200001018B4246D12DE049F60102934237D078
:1047300012D841F20C00834226D004D800F1FF3198
:104740008B4237D14CE041F20D02934221D002F16D
:10475000070293422ED121E049F603018B4223D078
:1047600020D301F102018B4220D001F10B018B42D9
:1047700020D11DE020492BE0204929E0204927E0F5
:10478000204925E0204923E02048A8604FF000019F
:1047900027E01F4BAB604FF0000122E01D4917E0FE
:1047A0001D4915E01D4913E01D4911E01D490FE0A9
:1047B0001D490DE042F20502A5F84A201B4907E019
:1047C0001B4905E042F21900A5F84A00174900E02C
:1047D00081B12068224621F09DFA0BE0154900E0E6
:1047E000154995F86430002BECD1F1E71349EFE758
:1047F0001349EDE711B0F0BDF14E0200395F020040
:10480000894802003D4D02005D5D020071530200C7
:10481000C152020099620200F14A0200F54F020003
:10482000795C0200255A0200F9490200454802005D
:10483000A1630200594C0200BD62020069490200F6
:104840005949020070B50646946904F14405636C49
:1048500003F10C0363644FF0030284F848204FF027
:10486000000084F84900E26AE2648B4201D907F053
:10487000CBFA30462946626C3AF0F8FA4FF0000164
:10488000E162606C70BD00BF2DE9F04383B08046EB
:1048900089461746966940F25D53C1F200031878C5
:1048A000F8B1326B40F26051C1F200010B8843F461
:1048B00080318A421ED040F26054C1F200044FF0B1
:1048C000000310F0010F34D003F101052B4685429F
:1048D00005D234F8021F41F48031914232D1834233
:1048E00008D1306BB0F1FF3F04D042F20803A6F8C4
:1048F0004A3016E0726B02F1FF3313F1030F04D854
:1049000042F21402A6F84A200BE0308E4FF000016C
:104910000A4601ABFFF720FE4FF0040171640198D5
:104920003065404649463A46FFF78CFF03B0BDE884
:10493000F08303F1010334F8021F41F48031914206
:10494000C2D1CCE705F1010334F8021F41F48031F4
:104950009142B9D1C3E700BF10B593694FF000048D
:104960001C60FFF76FFF10BD38B593691C682CB150
:1049700042F21E05A3F84A501C6501E01C6B1C6046
:10498000FFF760FF38BD00BF2DE9F84380460E46B3
:1049900091460A9D2C686CB30F68006822189742F4
:1049A00003D80899CA19904204D30898C7193760E8
:1049B000BDE8F883C71B0898C11B8C4228BF0C4672
:1049C000099A32B1D9F800001018D91922463AF0E4
:1049D0004DFA2B68191B2960D8F800201019C8F867
:1049E0000000D9F800301919C9F800103268BF1852
:1049F0003C193460BDE8F883F0B58DB005460591EB
:104A0000164694694FF000030B93E3614FF6FF7075
:104A1000216B07AAFFF7E0FD079848B942F20903A6
:104A2000A4F84A30284605993246FFF70BFF35E0D7
:104A30004FF0100108914FF00202ADF8242049F622
:104A40001006ADF82660E76A0A9704F1200704F122
:104A50001C064FF00C030093019505A80290384600
:104A600031460BAA08ABFFF78FFF0599A9B14FF0AC
:104A7000000206924FF004030093019505A80290EE
:104A8000384631460BAA06ABFFF77EFF059921B1E8
:104A900045F28522C0F2020262600B980DB0F0BDB3
:104AA000F0B5A5B01C78ADF811406CB14FF0000422
:104AB00004F1010413F8015F24AF07EB440626F864
:104AC0007F5C002DF4D101E04FF0000404F10104FB
:104AD00024AB03F8804D4FEA440404F10104009430
:104AE0002A9C01942B9C0294FFF74EFF25B0F0BD49
:104AF000F0B58BB00746059194694FF0000306931B
:104B0000E3614FF01C0007904FF00201ADF8201058
:104B100049F60102ADF82220E56A099504F1200664
:104B200004F11C054FF00C030093019705A80290B7
:104B30003046294606AA07ABFFF726FF059900294C
:104B400000F086804FF0060207924FF004030093B6
:104B5000019705A802903046294606AA07ABFFF741
:104B600013FF0599002973D04DF60142ADF81C20C2
:104B70004FF002030093019705A8029030462946A2
:104B800006AA07ABFFF700FF0599002960D04DF694
:104B90000242ADF81C204FF002030093019705A8D4
:104BA00002903046294606AA07ABFFF7EDFE0599AD
:104BB00000294DD04DF60342ADF81C204FF0020302
:104BC0000093019705A802903046294606AA07AB34
:104BD000FFF7DAFE059900293AD04DF60442ADF808
:104BE0001C204FF002030093019705A80290304665
:104BF000294606AA07ABFFF7C7FE059941B34DF654
:104C00004142ADF81C204FF002030093019705A824
:104C100002903046294606AA07ABFFF7B5FE059974
:104C2000B1B14DF64442ADF81C204FF002030093A1
:104C3000019705A802903046294606AA07ABFFF760
:104C4000A3FE059921B145F28522C0F202026260FD
:104C500006980BB0F0BD00BFF0B58BB006460591CD
:104C600094694FF000030993206A0B283BD84FF654
:104C7000FF70216B04F11402FFF7AEFC206165693F
:104C800025B10268516A09B193693BB942F2090141
:104C9000A4F84A104FF00003A36108E028469847A3
:104CA000A061206905686A6A606990476061A069CF
:104CB00000F10C0006904FF00205ADF81C5041F2D7
:104CC0000902ADF81E20E16A08914FF00C03009331
:104CD000019605A8029004F1200004F11C0109AA24
:104CE00006ABFFF751FE6569ADB1059F236AA3F1DD
:104CF0000C03A2690092019605A9029104F120001B
:104D000004F11C0109AAEB18FFF73EFE05983F1AB3
:104D1000A369DA1BA261099909B1059850B1236909
:104D20001A68D16B09B16069884745F28520C0F2E5
:104D30000200606009980BB0F0BD00BF2DE9F04F94
:104D40008DB00746059195694FF000030B93EB6119
:104D5000D5F830C01FFA8CF440F25D50C1F200006B
:104D600090F800E0BEF1000F1CD040F26051C1F29B
:104D700000010B88A34221D040F26051C1F2000132
:104D80004FF000031EF0010F00F0A28003F10100BC
:104D90000346704504D231F8026FA64240F0A0806D
:104DA00073450BD1BCF1FF3F08D042F20800A5F8D3
:104DB0004A0038460599FFF745FD86E0696B01F129
:104DC000FF3313F1030F08D842F21401A5F84A107B
:104DD00038460599FFF736FD77E020464FF0000191
:104DE0000A4607ABFFF7B8FB079A02F104024FEA45
:104DF000820008904FF00201ADF8241041F2070341
:104E0000ADF82630EA6A0A9205F1200805F11C097E
:104E10004FF00C000090019705A9029140464946C9
:104E20000BAA08ABFFF7B0FD059B002B4CD04FF051
:104E300004020092019705A80290404649460BAA39
:104E400007ABFFF7A1FD059900293DD040F2F046E0
:104E5000C1F200063668002E2DD04FF0040BA2469A
:104E60004FF6FF739A4503D03268108850451FD122
:104E70003168CB68E3B19847044617E03268116A9D
:104E8000204688470690CDF800B0019705A802900B
:104E9000404649460BAA06ABFFF776FD059B9BB142
:104EA0003268116921B1204688470446002CE5D1BB
:104EB0007668002ED4D10B9808B1059B23B145F23A
:104EC0008522C0F202026A600B980DB0BDE8F08F37
:104ED00003F1010331F8020FA0427FF457AF5FE7FF
:104EE00000F1010331F8020FA0427FF44FAF57E702
:104EF0002DE9F04F8BB08146059196694FF0000384
:104F00000693F36140F25D50C1F20000017801F1B7
:104F100004014FEA810207924FF00207ADF82070BA
:104F200041F20403ADF82230F06A099006F120073F
:104F300006F11C084FF00C010091CDF8049005AA71
:104F400002923846414606AA07ABFFF71DFD059BB6
:104F5000002B49D040F25D50C1F20000017807916A
:104F60004FF004020092CDF8049005AB029338464E
:104F7000414606AA07ABFFF707FD0598002833D086
:104F800040F25D51C1F200010A7822B3184D4FF092
:104F900000044FF0010B40F25D539A46C1F2000A43
:104FA00035F8020FADF81C00ADF81EB04FF004014B
:104FB0000091CDF8049005AA02923846414606AA0F
:104FC00007ABFFF7E1FC059B73B104F101049AF80C
:104FD0000000A042E4D8069909B1059A22B145F231
:104FE0008523C0F20203736006980BB0BDE8F08F12
:104FF0005E0500102DE9F0418EB0054605919469DB
:105000004FF000030693E361208EA0F55C4101F1AF
:10501000FF33432B4BD8DFE813F05300F400F400C8
:10502000F7004A004A004A004A004A004A0053007A
:105030004A004A004A004A004A004A004A004A0020
:105040004A004A004A004A004A004A004A004A0010
:105050004A004A004A004A004A004A004A004A0000
:105060004A004A004A004A004A004A004A004A00F0
:105070004A004A004A004A004A004A004A004A00E0
:105080004A004A004A004A004A004A004A004A00D0
:105090004A004A004A004A004A0044004A004A00C6
:1050A00047004FF01A060DE04FF00B060AE04AF6F3
:1050B0000101A4F84A1028460599FFF7C3FBA6E0B2
:1050C0004FF00E0606F10C0207924FF00207ADF802
:1050D000207007F51840ADF82200E16A099104F14B
:1050E000200804F11C074FF00C030093019505AA5A
:1050F00002924046394606AA07ABFFF745FC0598E1
:1051000000287CD0218EA1F55C4303F1FF304328B9
:1051100064D8DFE800F0222B374063636363636386
:105120005B63636363636363636363636363636357
:10513000636363636363636363636363636363633F
:10514000636363636363636363636363636363632F
:105150006363636363634963635207A847F6182177
:10516000C0F20601324639F081FE37E007A847F663
:105170007C31C0F20601324639F078FEA28EADF8DD
:1051800021202BE007A847F65431C0F20601324631
:1051900039F06CFE22E007A847F62821C0F206018C
:1051A000324639F063FE19E007A847F6D431C0F261
:1051B0000601324639F05AFE10E007A847F6B8312A
:1051C000C0F20601324639F051FE07E007A847F663
:1051D000C431C0F20601324639F048FE009601950E
:1051E00005A902914046394606AA07ABFFF7CCFB5A
:1051F000059B23B145F28520C0F20200606006984D
:1052000005E04FF00C065DE74FF012065AE70EB0CE
:10521000BDE8F0812DE9F84380460E4691460A9D8F
:105220002C686CB30F6800682218974203D808995D
:10523000CA19904204D30898C7193760BDE8F883AB
:10524000C71BD9F800100898421A944228BF144688
:10525000099820B1C0195918224639F007FE2B6869
:10526000191B2960D8F800201019C8F80000D9F8D7
:1052700000301919C9F800103268BF183C193460A1
:10528000BDE8F88310B58469626C02F10C026264B7
:105290004FF0030384F848304FF0000184F84910C0
:1052A000E36AE364006804F1440120F057FD94F8D8
:1052B000640000B9E0624FF00002A260626010BDBD
:1052C000F8B5064684693F2A8CBF00270127E369A9
:1052D00023B901F10C01A2F10C0500E0154620698B
:1052E0000268936B60692A46984768B92269136817
:1052F000196B6069884742F20C00A4F84A00E26921
:105300005319E36127B329E0002F2BD022691368DA
:1053100099696069884740F2F442C1F20002136A59
:10532000984209D023691868016B6069884742F286
:105330000702A4F84A2004E020690168CA6B60698A
:1053400090474FF000036361E0694119E16105E0B6
:10535000B4F84A1042F20100814207D03046FFF70C
:1053600091FFF8BDE1694819E061F1E7F8BD00BFC0
:105370002DE9F04F8BB005908A46164684694FF0B0
:105380000003099347F64429C0F2060940F2185B6E
:10539000C1F2000B40F2F440C1F20000049048E07A
:1053A000E2684FEA021009EB00054FF00003079393
:1053B00019F8001002297AD001290BD19BF800209E
:1053C0004FEA420008906968884205D9431A07935A
:1053D000089101E06F680897AA68B2F1FF3F14BF17
:1053E0005A44002204F1200804F11C07009601929F
:1053F00008A802904046394609AA5346FFF70AFF1B
:1054000000964FF00001019107AB029340463946E8
:1054100009AA5346FFF7FEFE0898079A111841B9EA
:10542000EB6813B143F001000047E36803F10103A7
:10543000E36009998E42B3D8402E38D1CCE0DBF836
:10544000082004990A62F0E7BBF8010040B34FF06E
:105450000003FF2888BF3F20049A985403F10103FA
:10546000BBF80310002940F0BA801BE0FF2988BF79
:105470003F21195403F1010213460BEB4201B1F82D
:10548000011079B1FF2988BF3F21815402F1010346
:105490000BEB4302B2F80110002940F0A28001E0BA
:1054A0004FF000034FF00000049AD054BDE74FF0D6
:1054B00000036361208E06A91A46FFF74DF840F2FB
:1054C000F441C1F20001086A069A904204D942F2FE
:1054D0000C03A4F84A307CE0268E04F1140840F254
:1054E000F045C1F200052D689DB14FF0000140F27A
:1054F000F447C1F200072B681888B04205D1DA6A78
:105500001AB138469047014628B96D68002DF2D18E
:1055100001E04FF00001B8F1000F00D06161616956
:1055200021B142F21D01A4F84A1052E0268E40F249
:10553000F445C1F20005D5F820A040F2F043C1F2D5
:1055400000031D68B5B14FF0000140F2F449C1F20B
:1055500000090F4628680288B24207D1436B2BB17D
:10556000484651463A469847014628B96D68002D8D
:10557000F0D101E04FF00001B8F1000F00D06161FF
:105580002561606920B942F20C02A4F84A2020E0AB
:1055900029680A6A02B19047B4F84A1042F201033E
:1055A000994216D1228EA4F850204FF000014FF0FE
:1055B000010384F8523084F8531084F8541084F8AE
:1055C000551084F8561084F85710A0654FF00C0061
:1055D00060640598FFF756FE0BB0BDE8F08F0498A5
:1055E00044E71F2B7FF442AF5CE700BF2DE9F04199
:1055F00088B0804640F2F045C1F200054FF000044B
:1056000040F25C57C1F200074FF001062B6853B11E
:105610001A7A1AB11C721868016C19B95B68002BF0
:10562000F6D100E03BB940F25C51C1F200014FF00D
:1056300000020A7028E03E701A68136C0DF1030036
:1056400001A998479DF80300012809D010B102284C
:10565000DCD102E044F2030304E044F2070301E07A
:1056600044F202034FF0100202924FF00401ADF831
:105670000C10ADF80E304FF0FF300490019B0593F5
:10568000404602A920F06AFB08B0BDE8F08100BFE7
:1056900008B543692BB14FF0000141610078FFF775
:1056A000A5FF08BD10B514464DF6044398422BD013
:1056B00009D84DF6024188421CD020D801F1FF32B2
:1056C00090423DD111E04DF64143984221D004D89B
:1056D0004DF60B41884233D12AE04DF644429042C8
:1056E0001CD0B0F1FF3F2BD130E04FF001034FF061
:1056F000040028E04FF001034FF0020023E04FF0D8
:1057000001034FF002001EE04FF001034FF00800CC
:1057100019E04FF001034FF0100014E0084639F093
:10572000A3FC4FEA400000F103004FF001030AE040
:105730004FF00003184600F1040003F1010302E0FA
:105740004FF0000318465CB1236010BD084639F0E5
:105750008BFC4FEA400000F123004FF00603EAE71C
:1057600010BD00BF2DE9F0438BB007460E469046B2
:105770009946A0F55C4404F1FF34432C75D8DFE86A
:1057800004F0222C314074747474747471747474E1
:1057900074747474747474747474747474747474C9
:1057A00074747474747474747474747474747474B9
:1057B00074747474747474747474747474747474A9
:1057C00074745174745F0A6913681888ADF818000E
:1057D0004FF00101ADF81A1047E04FF44051ADF819
:1057E000181042E0086901684A691AB170690DF140
:1057F000170190479DF8173003F00100ADF818002D
:1058000033E00D692C68A3692BB1486998470446B9
:105810004FF0000503E04FF000044FF00005CDE924
:10582000064522E006A84FF000014FF0100239F0C3
:1058300051FB33691868016A70698847069014E063
:105840000B691868C169706988470346CDF80090F4
:10585000129A019206F1200006F11C014246FFF760
:105860001FF918E04FF000020692384648F6A06192
:10587000C0F206014FF00002FFF714FF0090CDF8D0
:105880000490129A029206F1200006F11C01424691
:1058900006ABFFF779F80BB0BDE8F083F0B585B043
:1058A00005466446CCF80010A080A0F55C4303F1E7
:1058B000FF30432861D8DFE800F022272C316060F8
:1058C00060606060406060606060606060606060F8
:1058D00060606060606060606060606060606060C8
:1058E00060606060606060606060606060606060B8
:1058F000606060606060606060603660603B4FF078
:105900000601ACF806101CE04FF00400ACF80600ED
:1059100017E04FF00403ACF8063012E04FF0080730
:10592000ACF806700DE04FF00A02ACF8062008E073
:105930004FF6FF71ACF8061003E04FF00606ACF826
:105940000660216A04F11C0604F114074FF00802F6
:105950000092A3690193029701F1200001F11C015B
:1059600032462346FFF710F8606930B1216AA36917
:10597000009728463246FFF7F5FE05B0F0BD00BFA0
:1059800038B56446DCF820301A691068016A586935
:105990008847054623699A68B2F1FF3F09D16069DB
:1059A00068B938BDA4464DF60B402946FFF776FF8F
:1059B00038BDA44690B22946FFF770FF38BDA44613
:1059C0004DF601402946FFF769FF616941B3A446DE
:1059D0004DF602402946FFF761FF636903B3A44611
:1059E0004DF603402946FFF759FF6269C2B1A4464C
:1059F0004DF604402946FFF751FF606980B1A44687
:105A00004DF641402946FFF749FF616941B1A4467F
:105A10004DF644402946FFF741FF6369002BC1D191
:105A200038BD00BF70B590B015460C900B919369CE
:105A30000E934FF000040D94DC610E9B03F13002D5
:105A40000A921A6A0B2A03D94FF00C01D961C3E0FC
:105A5000DA6B3AB14AF60702A3F84A202A46FEF763
:105A6000F1FE07E11A6C3AB14AF60802A3F84A209F
:105A70002A46FEF7E7FEFDE05A6B3AB142F2140205
:105A8000A3F84A202A46FEF7DDFEF3E0986B48F6BD
:105A9000A061C0F2060105AAFFF704FE059850B9FF
:105AA0004AF601000E9BA3F84A000C980B992A466F
:105AB000FEF7C8FEDEE04FF000010E9B99610A9AE6
:105AC000116819B34FF6FF700E9A02F11402FEF737
:105AD00083FD0E9A10610E9B586948B942F2090283
:105AE000A3F84A200C980B992A46FEF7ABFEC1E0BA
:105AF0000A9CA46819690A68D36998470146204638
:105B000005AAFFF7CFFD0E99886141E04FF0000034
:105B1000059040F2F041C1F200010A680E9B1A6143
:105B20000E980069002833D04FF000040168CA685D
:105B3000002A25D090470E9B58611DE095690A9E6A
:105B4000B66811690B68DA6990470146304604AAC5
:105B5000FFF7A8FD40190E998861049B059AD0189B
:105B600005900E990B691A68136923B14869984723
:105B70000E99486100E04C610E9A50690028DDD111
:105B80000E980269536803610E9908690028CDD107
:105B90000E99059800F102028B6903EBC200069092
:105BA0004FF00202ADF81C2049F60503ADF81E3097
:105BB000C86A08904FF00C0200920C9B01930BA84E
:105BC000029001F1200001F11C010DAA06ABFEF7C5
:105BD000DBFE0B9900294CD0059806900E994FF0EA
:105BE000040300930C9A01920BA8029001F120008B
:105BF00001F11C010DAA06ABFEF7C6FE0B990029A8
:105C000037D00A9B1A683AB10DF1180CFFF7B8FEAD
:105C10000B9A002A2DD022E040F2F040C1F20000A1
:105C200001680E9B19610E9A1369C3B11868C168A7
:105C300069B188470E9B586105E00DF1180CFFF71C
:105C40009FFE0B99A9B10E9A50690028F5D10E9BC1
:105C50001A69506818610E990B69002BE6D10D98EE
:105C600008B10B9929B145F285220E9BC0F20202C0
:105C70005A600D9810B070BDF0B58DB00646059114
:105C8000154694694FF000010B91E161226A0B2ADD
:105C90004CD84FF6FF70216B04F11402FEF79CFC08
:105CA0002061616939B942F20900A4F84A004FF055
:105CB0000002A26115E0A78E0068C26908469047FD
:105CC000014638464FF00002FFF7ECFCA06140B9F6
:105CD0004AF60103A4F84A304FF00001A161616166
:105CE00001E063692BB9304605992A46FEF7AAFD03
:105CF00032E0A16901F10C0106914FF00200ADF80C
:105D00001C0049F60302ADF81E20E36A08934FF029
:105D10000C010091019605A8029004F1200004F105
:105D20001C010BAA06ABFEF72FFE02E04FF00C039E
:105D3000E36162693AB1A08E05AB009321460BAADC
:105D40003346FFF70FFD0B9808B1059921B145F2D5
:105D50008522C0F2020262600DB0F0BD2DE9F0476D
:105D600096B006460591174694694FF000031593C7
:105D70008DF81B30E3614FF6FF70216B07AAFEF729
:105D80002BFC0546079848B942F20900A4F84A00DE
:105D9000304605993A46FEF755FDCAE02A68D169B2
:105DA00088478146286847691FB107980DF11B0194
:105DB000B847484639F058F900F123004FEA40034C
:105DC00008934FF00202ADF8242041F20801ADF82B
:105DD0002610E06A0A9004F1200804F11C074FF035
:105DE0000C030093019605AA02924046394615AA73
:105DF00008ABFEF7C9FD0599002900F099802868D5
:105E0000B0F800A09DF81B5005F00105836913B19F
:105E10000798984701E04FF00000ADF820A04FF040
:105E20000102ADF822204FF44051ADF82410ADF836
:105E300026500A904FF00000ADF82C00ADF82E006F
:105E4000ADF83000ADF83200ADF83400ADF83600F2
:105E5000ADF83800ADF83A00ADF83C00ADF83E00C2
:105E6000ADF84000ADF84200ADF84400ADF8460092
:105E7000ADF84800BDF84A3060F30F03ADF84A3082
:105E8000139014904FF034020092019605A90291EC
:105E90004046394615AA08ABFEF776FD059800285E
:105EA00046D0009605AB01934046394615AA4B46AD
:105EB000FEF7F6FD059A002A3AD04FF000018DF862
:105EC00020104FF001000090019605AB0293404670
:105ED000394615AA08ABFEF757FD059A42B34FF0B5
:105EE00000018DF820104FF001000090019605ABE5
:105EF00002934046394615AA08ABFEF745FD059AC0
:105F0000B2B14FF000018DF820104FF00100009069
:105F1000019605AB02934046394615AA08ABFEF739
:105F200033FD059A22B145F28521C0F2020161607C
:105F3000159816B0BDE8F0872DE9F04190B0054600
:105F4000059194694FF000030F93E36140F25D50B7
:105F5000C1F2000090F800E0BEF1000F21D0266BE6
:105F600040F26051C1F200010B8843F48030864258
:105F700020D040F26051C1F200014FF000031EF04A
:105F8000010F00F0B38003F101000346704506D213
:105F900031F8027F47F48037B74240F0B180734553
:105FA00008D142F20800A4F84A0028460599FEF7F5
:105FB00049FC98E0B6F1011F14D040F2F042C1F262
:105FC000000213689BB1B6B21F683988B14201D193
:105FD0007F6887B95B68002BF6D147F68837C0F237
:105FE000060708E047F68837C0F2060703E047F6E1
:105FF0008837C0F20607384639F036F800F101025A
:106000000D9200F11F004FEA400006904FF002068B
:10601000ADF81C6041F20501ADF81E10E36A08936B
:1060200004F1200804F11C064FF00C0200920195C7
:1060300005A80290404631460FAA06ABFEF7A4FC25
:10604000059900294ED0208E0EA90DAA4FF000030D
:10605000FEF782FA4FF000034FF00302ADF818206C
:106060004FF00100ADF81A00ADF81C300D99CDF8D5
:106070001E10CDF822300E9ACDF82620CDF82A3009
:106080004FF0FF33ADF82E30ADF830304FF01A003E
:106090000090019505A90291404631460FAA06AB32
:1060A000FEF772FC059AEAB1009505AB01934046F4
:1060B00031460FAA3B46FEF7F3FC059890B10095D8
:1060C00005A90191404631460FAA47F69C33C0F21C
:1060D0000603FEF7E5FC059A22B145F28523C0F2DE
:1060E000020363600F9810B0BDE8F08103F1010373
:1060F00031F8020F40F48030B0427FF444AF4EE7F5
:1061000000F1010331F8020F40F48030B0427FF417
:106110003AAF44E7F0B58DB005460591164694694F
:106120004FF000030B93E06800287BD1E061216A07
:10613000C1B947F62C30C0F20600FBF7C7F9606121
:1061400048B942F20A00A4F84A00284605993246A6
:10615000FEF778FB9BE0FAF7AFFFA0616069FAF702
:10616000C1FF6061A26902F11A0208924FF00206B3
:10617000ADF8246041F21407ADF82670E36A0A9383
:1061800004F1200704F11C064FF00C00009001956B
:1061900005A90291384631460BAA08ABFEF7F4FB7D
:1061A000059A002A6AD04DF20543ADF8203044F23A
:1061B0000200ADF822004FF000018DF824104FF0DE
:1061C00005020092019505AB0293384631460BAAB1
:1061D00008ABFEF7D9FB059800284FD04FF000011F
:1061E00007914FF004020092019505AB02933846E7
:1061F00031460BAA07ABFEF7C7FB059800283DD038
:106200004FF004010091019505AA029238463146EB
:106210000BAA04F11803FEF7B7FB059B002B2DD04A
:106220001C4EE660059F079704F1200704F11C0649
:106230006369A1690091019505AA02923846314629
:106240000BAAFEF7A1FB0598079B1A1A0792616932
:106250008B186361A1698A1AA26178B14FF00000BE
:106260008DF820004FF001030093019505A90291DC
:10627000384631460BAA08ABFEF786FB0B9808B1EF
:10628000059A22B145F28523C0F2020363600DB086
:10629000F0BD00BF2462020038B593691C6B4DF25B
:1062A0000545AC4202D1FFF735FF38BD42F21B0471
:1062B000A3F84A40FEF7C6FA38BD00BFF0B587B074
:1062C00007460E46154694694FF000038DF80F30CF
:1062D000216BB1F1FF3F04D142F20600A4F84A005D
:1062E0003DE042F20902A4F84A204FF6FF7004F1A3
:1062F0001402FEF771F90146606980B311B10B68B1
:106300001A6B62B3216109684B691BB10DF10F0172
:10631000984700BB9DF80F00E8B921690B6804930A
:10632000606905904FF00802009247F63430C0F2E1
:1063300006004FF0070144F23D52C0F2020204ABE6
:106340001EF0FCF942F20101A4F84A104FF00103DB
:1063500084F8643003E042F20D02A4F84A20384683
:1063600031462A46FEF76EFA07B0F0BD10B582B08E
:106370000C4640F20012C0F2000292F8463092F849
:106380004720009247F64032C0F2060236F08AFA01
:1063900000F10100A04228BF204602B010BD00BF9E
:1063A0002DE9F04399B00546059194694FF000033B
:1063B0000793E361206A0B282AD89B4838F054FEE3
:1063C00006464FF000004FF04001FFF7CFFF3218B4
:1063D0004FEA420606F1C50608964FF00203ADF8F3
:1063E000243041F20100ADF82600E16A0A914FF035
:1063F0000C020092019505AB029304F1200004F118
:106400001C0107AA08ABFEF7BFFA059818B907E107
:106410004FF00C01E16147F61026C0F2060608AA0B
:106420003068716803C204F1200804F11C064FF0C3
:1064300008010091019505AB02934046314607AA39
:1064400008ABFEF7A1FA0598002800F0E9804FF0AC
:1064500000098DF820904FF001070097019505AFD6
:1064600002974046314607AA08ABFEF78DFAADF811
:1064700020904FF00202009201950297404631466B
:1064800007AA08ABFEF780FA0599002900F0C8803A
:1064900018AF4FF0120347F8403D09A847F6F42122
:1064A000C0F206014FF0240238F0E0FC4FF0280063
:1064B0000090019505AA02924046314607AA3B4644
:1064C000FEF762FA0599002900F0AA8018AF4FF094
:1064D000030347F8403D09A840F2F801C1F200016A
:1064E0004FF0060238F0C2FC4FF00A000090019510
:1064F00005AA02924046314607AA3B46FEF744FAF7
:106500000599002900F08C8018AF4FF0010347F87F
:10651000403D09A847F61831C0F206014FF00202CB
:1065200038F0A4FC4FF006000090019505AA0292F5
:106530004046314607AA3B46FEF726FA0599002950
:106540006ED0CDF820904FF004000090019505AA80
:1065500002924046314607AA08ABFEF715FA0599A4
:1065600000295DD018AF4FF0040347F8403D09A85B
:1065700047F63C21C0F206014FF0080238F076FCE5
:106580004FF00C000090019505AA0292404631465A
:1065900007AA3B46FEF7F8F90599002940D0009577
:1065A00005AB01934046314607AA47F6A833C0F22F
:1065B0000603FEF775FA0598002831D0009505AA64
:1065C00001924046314607AA174BFEF769FA059932
:1065D00031B308A84FF04001FFF7C8FE009505ABA6
:1065E00001934046314607AA08ABFEF759FA0598D1
:1065F000B0B108A84FF020014A461FF0E9FB18AAE5
:10660000111801F8409C009505A8019040463146BC
:1066100007AA08ABFEF744FA059A0AB1034961607C
:10662000079819B0BDE8F0831601000085520200FA
:1066300000B583B00378A12B4AD1407866284AD0B0
:10664000672820D0642802D04FF002004EE0062ACE
:1066500044D10A8844F201039A4242D1D1F802108F
:1066600040F28840C1F20000C26A91423CD1204B06
:106670004FF0000159601F481FF0C2F81FF0CCFA1C
:106680004FF0010032E040F28840C1F20000C26ADF
:106690006AB940F28843C1F2000393F8641042F2F1
:1066A000190042F20103002918BF034601E042F23B
:1066B00019034FF00402ADF80420ADF806304FF096
:1066C00000000DEB02011FF049FB4FF003000DE04D
:1066D0004FF002000AE04FF0010007E04FF0020027
:1066E00004E04FF0020001E04FF0020003B000BDF3
:1066F00088040010F07B060010B5044640F2F04319
:10670000C1F200031B68002B31D0026811881868A1
:1067100002888A4214BF00220122A34208D110BD80
:10672000186802888A4214BF002201229C4226D0A7
:106730005B68A2B9002BF3D119E005F065FB40F2CC
:106740005D53C1F200031A782068008840F260515E
:10675000C1F2000121F8120002F101021A7040F2A8
:10676000F043C1F200031A6862601C6010BD40F281
:106770005D51C1F200010A78032AE0D9DDE710BDBE
:1067800008B54FF00103037240F25C50C1F2000003
:10679000017839B947F61C30C0F206001FF030F816
:1067A000FEF724FF08BD00BF40F27053C1F20003A2
:1067B0001868A0F10300704747F64440C0F2060095
:1067C000704700BF4FF6FD70704700BF4FF6FD7376
:1067D00098420CBF18460020704700BF4FF6FD736B
:1067E000984214BF02200020704700BF4FF6FD738F
:1067F0000B604FF000010170704700BF08B540F218
:106800000010C1F20000FFF777FF08BD08B540F2A5
:106810000010C1F20000FFF7B3FF47F65840C0F286
:1068200006004FF0070146F63502C0F202021DF0E5
:1068300091FF08BD2DE9F047C2B041F288301DF04C
:10684000C7FF4FF00000FAF7EBFF05464FF00000DE
:10685000FAF7FAFF00EB050A40F26853C1F20003B1
:106860001868C1787E290ED047F67043C0F206033F
:1068700000934FF00000014652464FF0FF33FBF704
:1068800025F9AA44BAE047F69442C0F20602009203
:106890004FF00000014652464FF0FF33FBF716F968
:1068A0004FF0000001464FF0FF321346FCF75AFA52
:1068B0000AEB0504A2461DF059FF21F0C3FC98B96C
:1068C00047F6B042C0F206020092014622464FF05F
:1068D000FF33FBF7FBF84FF0000001464FF0FF32AB
:1068E0001346FCF73FFA89E047F6C043C0F20603BF
:1068F00000934FF00000014622464FF0FF33FBF7B4
:10690000E5F84FF0000001464FF0FF321346FCF768
:1069100029FA04EB050A1DF029FF40F27050C1F27C
:1069200000000168042925D94FF482744FF0040354
:1069300040F26858C1F200084FF040073E4E40F266
:106940007059C1F2000900E00446D8F8002002A8FE
:10695000D1183A4602F0C8FF02A831194FF48072EC
:1069600003F08AFA30B904F580702346D9F8001094
:10697000A142E9D840F26852C1F20002106800F169
:10698000040040F20001C0F2010140F27053C1F274
:1069900000031A6835F096FCB0B147F6E041C0F24A
:1069A000060100914FF00000014652464FF0FF33C0
:1069B000FBF78CF84FF0000001464FF0FF32134612
:1069C000FCF7D0F9AA4419E047F6F040C0F20600FF
:1069D00000904FF00000014652464FF0FF33FBF7A6
:1069E00075F84FF0000001464FF0FF321346FCF7F8
:1069F000B9F94FF0010022F08BFD1AE047F6FC4098
:106A0000C0F2060000904FF00000014652464FF0E1
:106A1000FF33FBF75BF84FF0000001464FF0FF3209
:106A20001346FCF79FF942F210701DF0D1FE05F0FD
:106A3000EBF942B0BDE8F087FCFE000038B5144623
:106A400040F26853C1F200031B68D3B140F27052A8
:106A5000C1F200021068251840F26C52C1F2000227
:106A60001268954210D81818224638F0FFF940F203
:106A70007051C1F200010B68E4180C604FF0010086
:106A800038BD4FF0000038BD4FF0000038BD00BFEA
:106A900000B583B040F26853C1F200034FF000022A
:106AA0001A604FF02E0136F0DFFA002848D047F682
:106AB0001C51C0F2060135F03BFF002840D122F006
:106AC00027FD40F20000C0F20100214B181A40F2ED
:106AD0006C52C1F20002106007F0FEFA40F26851F9
:106AE000C1F20001086058B34FF00100FCF726FA2C
:106AF0004FF00000FAF7A8FE024647F62450C0F215
:106B0000060000904FF0000001464FF0FF33FAF707
:106B1000DDFF40F26C53C1F200031A6840F2685185
:106B2000C1F2000108684FF0FF314FEA920205F010
:106B3000CDF940F27050C1F200004FF00303036042
:106B400040F26852C1F20002106803B000BD00BFFD
:106B5000080002004FF0FF3303600B604FF00000AD
:106B60001060704740F27453C1F200031868704718
:106B700047F69850C0F20600704700BF4FF6FE700F
:106B8000704700BF4FF6FE7398420CBF18460020B6
:106B9000704700BF4FF6FE73984214BF02200020DA
:106BA000704700BF2DE9F00F84B040F28453C1F26A
:106BB00000031868002800F0018140F27453C1F20C
:106BC0000003186810181860002A00F0FA8040F2DC
:106BD0008454C1F20004256802950E46891840F2DB
:106BE0007853C1F200034FF0000247F64857C0F255
:106BF0000607009740F20009C0F2000940F2000ABF
:106C0000C5F2000A40F20000C5F28000019040F297
:106C10000004CAF20004039416F8015B1C79A5F184
:106C20004107F8B2052803D8A5F13700C7B208E03C
:106C3000A5F13007FFB2092F03D9002C40F08F8057
:106C4000174693F809C047EA0C105FFA80FC83F8F6
:106C500009C0D87900F10100C0B2D87110F0010864
:106C60000AD193F808B0E34483F808B093F806B06B
:106C70000BF1FF3B83F806B0062C05D8DFE804F0E3
:106C8000060D1B2440565E00104663E0532D58D17C
:106C90004FF00100187110465FE0DDF800C01CF8ED
:106CA000070000285BD05F711A721A604FF0020073
:106CB0001871104651E0022845D183F806C04FF004
:106CC00003001871104648E01D6847EA05171F6069
:106CD0005D79DDF800B01BF80550B0EB450F34D1FD
:106CE0009879012804D14FF005001871104634E05E
:106CF0004FF004051D7107F1FF371F60104629E0B2
:106D0000B8F1000F23D11D6805F101051D60587908
:106D100000F1FF35E8B202288CBF002001209D79E8
:106D2000012D17D14FF005041C7116E0022810D177
:106D3000187AFF2813D11A7110460EE04FF00200A6
:106D400008E0104606E0104604E0104602E0104657
:106D500000E010461D79A5420BD0DA7109E040F23F
:106D60007851C1F200014FF006030B714FF00000A3
:106D70002CE0022828D001281AD1186848450DD3E4
:106D800040F20004C0F20804A04207D85C7AC9EBC4
:106D90000000DDF808C00CF8004009E0504507D3BA
:106DA000019CA04204D8CAEB00005C7A039D4455C4
:106DB0008E427FF431AF4FF0010007E04FF000004A
:106DC00004E04FF0010001E04FF0000004B0BDE826
:106DD000F00F704708B540F20C10C1F20000FFF749
:106DE0008BFC08BD08B547F6A850C0F206004FF06E
:106DF000070146F60162C0F202021DF0ABFC08BDBD
:106E00002DE9F04184B002AF41F68462C0F206027F
:106E100041F6D473C0F20603981A20F0030101F181
:106E20000A0121F00702ADEB020D0DF1080841F255
:106E300088301DF0CDFC1EF07BFC4FF00000FAF70F
:106E400047FC47F65800C0F20600FAF73FFB00285F
:106E500000F0AE804FF00000FAF7E2FC04464FF07D
:106E60000000FAF7F1FC05192E4640F20003C0F2CB
:106E7000000340F20010C0F20000C21A40F2845138
:106E8000C1F2000108684CF6DE63CEF6A5538258C5
:106E90009A4274D14FF00000FAF748FB00286ED0F8
:106EA00047F6C056C0F2060600964FF000000146B5
:106EB0002A464FF0FF33FAF709FE4FF00000014673
:106EC0004FF0FF321346FBF74DFF2E191DF04EFC1D
:106ED00040F20003C5F20003184640F20001C5F27B
:106EE0008001C91A07F104023B462DF0DDF847F690
:106EF000DC50C0F2060000904FF000000146324620
:106F00004FF0FF33FAF7E2FD4FF0000001464FF07B
:106F1000FF321346FBF726FF36191DF027FC786871
:106F200040F20001CAF200013A682DF085F847F6F8
:106F3000F852C0F2060200924FF0000001463246BD
:106F40004FF0FF33FAF7C2FD4FF0000001464FF05B
:106F5000FF321346FBF706FF36191DF007FC41F61A
:106F60008463C0F206034046194641F6D472C0F26B
:106F70000602D21A37F07AFF08F10108C04747F637
:106F8000FC41C0F2060100914FF00000014632467C
:106F90004FF0FF33FAF79AFD4FF0000001464FF033
:106FA000FF321346FBF7DEFE42F210701DF010FCBC
:106FB00004F02AFF07F10807BD46BDE8F08100BFD5
:106FC00070B58AB004463D4D03A847F61061C0F283
:106FD00006012A4635F07CFC204603A935F0A8FCC2
:106FE000064603A847F61861C0F206012A4635F0A6
:106FF0006FFC204603A935F09BFC08B1002E55D14B
:107000004FF0000022F084FA40F27850C1F2000004
:107010004FF000014FF00C0237F05CFF40F200032C
:10702000C0F2000340F20004C0F20804E41A204653
:1070300007F052F840F28451C1F200010860A8B391
:107040004FF00100FBF77AFF4FF00000FAF7FCFB6E
:10705000024647F62060C0F2060000904FF00000A4
:1070600001464FF0FF33FAF731FD40F28452C1F28E
:10707000000210684FF0FF314FEA940204F026FF3F
:1070800040F20000CAF2000040F20003CAF280039E
:107090001A1A4FF0FF314FEA920204F017FF40F244
:1070A0007451C1F200014FF00000086040F28453B7
:1070B000C1F2000318680AB070BD00BF16010000DD
:1070C0002DE9F00F82B04FF0000301930093019B74
:1070D0004FF00102019202606FF001034360026809
:1070E000012A0BD14FF0020303606FEA03024260F2
:1070F00002689A4204D15300F6D101E04FF0010337
:107100000093009A002A40F0CD804FF002070197CB
:10711000091A21FA07F707F1FF3212F0010F00F008
:10712000D3804FF001034FF0AA3440F823404FEAD8
:1071300043031342F9D1BBE003F1FF3440F824507C
:1071400000EB830650F82340B4F1AA3F04D023E0BB
:107150004FF001034FF055354FEA43031A42EBD18C
:10716000B9E000EB850640F825800368B3F1AA3F3B
:1071700012D1634650F82340B4F1AA3F01D09D429A
:107180000AD14FEA43031342F4D1C6F800904FEA04
:1071900045051542E5D102E0002E40F086804FF013
:1071A00003020192C1F17F4909F58019002F6ED0C9
:1071B00009EB07084B466FEA090404EB080202F0EA
:1071C0000102044644F8049B03F10103434540F0E7
:1071D000C5800CE0224642F8043B03F101031D4642
:1071E000636003F1010302F104044345F2D1036833
:1071F00099454FD100F1040A52464D4603464FF0DF
:10720000000617F0010F09D18BE01346144654F81D
:1072100004CBA346AC4500F092803EE06FEA050443
:107220001C6005F1010506F10106BE42EDD10268C0
:107230006FEA090991452FD14FF00103CFF6107382
:10724000591A6FEA01016FEA080803464FF000007F
:10725000C8EB010212F0010F13D055E0534652461D
:1072600052F8046B154601F1FF348E4215D1CAF86D
:1072700000001346DAF8045002F1040AA5424DD08A
:107280000BE018604145E9D14FF0000305E04FF0F5
:10729000000302E0034600E00346D3F1010038BFDB
:1072A00000202DE04FF000002AE04FF0000027E022
:1072B0004FF05533036003604368B3F1AA3F18BF32
:1072C000061D7FF469AF43E74FF0553303604FF07D
:1072D000AA32026063E706464FF0AA3346F8043B41
:1072E0004FF0553343600368B3F1AA3F7FF454AFC6
:1072F0004FF00105AC464FF0AA394FF0553838E74A
:1073000002B0BDE8F00F7047186053465AF8044BBE
:1073100001F1FF328C42C0D11146B2E704F1FF31D6
:10732000AFE76FEA0904046009F1010406F1010600
:10733000534652F8045BA5423FF470AFADE76FEAE5
:107340000C0515600CF1010C06F101062346556889
:1073500004F1040265453FF461AF9EE7002A3FF463
:1073600039AF44F8043B03F1010343457FF432AFE6
:107370003DE700BF11B1012916D108E040F2181114
:10738000C1F200010B7813704FF00000704748F213
:107390009400C2F20900016881F48033C3F3004015
:1073A00010704FF0000070474FF01400704700BF9E
:1073B00010B5144611B1012921D115E044F2400164
:1073C000C4F202010A6812F4003F44F24003C4F21E
:1073D00002031868C0F3100018BF40422CF0FAFFF7
:1073E00020604FF0000010BD40F28850C1F2000054
:1073F00000682DF01FF820604FF0000010BD4FF026
:10740000140010BD684620F007018D4601B440F21B
:107410000002C4F209021368136003F01000C1B245
:1074200000293ED040F29852C1F20002136883B99D
:1074300040F22C00C4F20900016840F28C52C1F203
:107440000002116040F28853C1F200034FF00000C7
:10745000186040F29851C1F200010A68B2F5006F5D
:107460000FD140F22C03C4F20903186840F28C518A
:10747000C1F200010A68801A40F28853C1F2000389
:10748000186040F29851C1F200010A68B2F5006F2D
:1074900007D840F29850C1F20000036803F10103DD
:1074A000036001BC8546704708B54FF4005047F6AD
:1074B0007861C0F2060140F29C52C1F2000220F055
:1074C000A1FF08BD38B514464FF000031370002922
:1074D00040F0978040F29050C1F20000016800290E
:1074E00040F092804FF0000000F004FC4CF2C40524
:1074F000C4F20F052A6842F480032B6047F67460DB
:10750000C0F2060001684CF2C815C4F20F052960EC
:107510004CF2EC03C4F20203186840F29452C1F238
:107520000002106047F65C61C0F206010D681D6044
:1075300047F65463C0F20603186840F27002C4F2C2
:107540000902106047F65861C0F206010D684CF25E
:107550003C13C4F202031D6047F6B060C0F206009F
:10756000026840F22801C4F209010A6047F6AC65DE
:10757000C0F2060528684CF23813C4F20203186002
:107580004FF0000540F20C02C4F20902156040F20F
:107590001401C4F209010D6040F20400C4F20900B4
:1075A00047F6B463C0F206031A68026047F65061FA
:1075B000C0F206010B68036047F66060C0F2060087
:1075C0004FF0070147F26962C0F202021DF0C2F8F3
:1075D00040F29052C1F20002106047F20540C0F242
:1075E00002004FF00F014FF0030204F02BFD4FF0AB
:1075F000010040F21811C1F2000108702070284605
:1076000038BD4FF0140038BD4FF0000038BD00BF4A
:1076100070B540F29853C1F200034FF000021A60B7
:107620001DF0CCFD054643F2D30440F29856C1F25A
:1076300000061DF0C3FD401BA04209D940F21810FE
:10764000C1F200004FF0050202704FF0000070BD63
:107650001DF08CF83168B1F5006FEAD940F288531B
:10766000C1F20003186870BD70B54FF0000001460C
:1076700003F0FAF8FFF7CCFF064640F21813C1F208
:1076800000031878012840F0EA8030462CF0DAFE3A
:1076900004460D4684A3D3E900232DF043FF38B9F7
:1076A0002046294682A3D3E900232DF057FF38B1A5
:1076B00040F21811C1F200014FF002030B70CEE04E
:1076C000FFF7A6FF044640F21811C1F200010A7844
:1076D000012A40F0C480864294BFC6EB0006C0EB8E
:1076E0000606012E55D9FFF793FF054640F2181301
:1076F000C1F200031878012840F0B180AC4294BF79
:10770000C4EB0504C5EB0404012C3FD9FFF780FF4F
:10771000044640F21811C1F200010A78012A40F033
:107720009E80854294BFC5EB0005C0EB0505012D89
:107730002FD9FFF76DFF054640F21813C1F2000381
:107740001878012840F08B80AC4294BFC4EB05044C
:10775000C5EB0404012C1BD9FFF75AFF044640F285
:107760001811C1F200010A78012A78D1A84234BF69
:10777000C0EB0505C5EB0005012D0AD940F2181430
:10778000C1F200044FF00203237068E02C4600E0D1
:107790002C4620462CF056FE04460D4646A3D3E95F
:1077A00000232DF0BFFED0B143A1D1E90001224654
:1077B0002B462DF02DFB02460B46204629462DF088
:1077C00023FD4FF000024FF00003C3F6E0732DF0ED
:1077D00021FB2CF0F1FF04464FF001051AE0204692
:1077E000294635A3D3E900232DF012FB02460B46B0
:1077F00031A1D1E900012DF007FD4FF000024FF05B
:107800000003C3F6E0732DF005FB2CF0D5FF044612
:107810004FF00005B4F5003F0AD340F21813C1F24F
:1078200000034FF004021A704FF000052C460AE0E6
:107830002846214603F018F840F21810C1F2000063
:107840004FF0000101702846214603F023F830B9BB
:1078500040F21814C1F200044FF0030020704FF002
:10786000000440F22802C4F20902146020464FF0DE
:107870000F014FF0030204F0E5FB40F29450C1F217
:10788000000001684CF2EC03C4F20203196040F2FC
:107890009052C1F2000214604FF0010000F02AFA89
:1078A00070BD00BFAFF3008000000000EE0D63412B
:1078B00000000000B217634100000000D0126341D5
:1078C000F8B515461C464FF00003237021BB40F26B
:1078D0009050C1F20000016809BB10462DF06AFE0D
:1078E000074628462CF0CAFE0646D7F1010038BFED
:1078F0000020314602F0CEFF28462DF05BFED0F18D
:10790000010038BF0020314602F0AEFF4FF0010207
:1079100022704FF00000F8BD4FF01400F8BD4FF09A
:107920000000F8BD4FF0000303600B604FF0010052
:107930001060704740F2C453C1F200031868A0F50C
:107940008030704740F2C453C1F200031A68A2F5B8
:107950008033984206D141B14FF0000008704FF0DB
:10796000030070474FF0020070474FF0030070476C
:1079700040F2C053C1F200031868704740F2C4538C
:10798000C1F200031868A0F58030704740F2C4537C
:10799000C1F200031968A1F58032824218BF0020AD
:1079A000704700BF4FF00000704700BF08B540F2BD
:1079B0001C10C1F20000FEF79FFE4FF44A43C0F2D4
:1079C000080340F2C052C1F20002136008BD00BFBC
:1079D00008B540F2C453C1F200031A68A2F580331F
:1079E0000B6040F2B851C1F200010B780370BBB9D3
:1079F00002F10102B2F57A7F40F2C450C1F20000F8
:107A000028BF0022026040F2B851C1F200014FF0DD
:107A100001020A7040F21C10C1F20000FEF7B0FE35
:107A200008BD00BF08B540F2BC53C1F2000318689E
:107A300008B107F04BFF4FF44A40C0F2080040F293
:107A4000C052C1F20002106040F2B851C1F2000110
:107A50004FF000030B7040F21C10C1F20000FEF763
:107A60008FFE08BD08B540F2C050C1F200004FF4CF
:107A70004A43C0F208030360FAF7E6FE40F2BC5145
:107A8000C1F20001086008BD10B540F2A854C1F26F
:107A9000000420464FF00D0147F6FC62C0F20602DA
:107AA00040F2C453C1F200031B6834F0FBFE2046D1
:107AB00010BD00BF48F23403C2F20903196811F087
:107AC000020F17D040F2D551C1F200010A78002A06
:107AD0004BD138B148F2B801C2F209014FF00202AD
:107AE0000A60704748F2BC00C2F209004FF002037E
:107AF0000360704740F2D552C1F200021378A3BB75
:107B0000D0B140F2D451C1F200010A7842BB47F62D
:107B10005873C0F20603196840F23C02C4F209022D
:107B2000116047F64C73C0F20603196840F2040274
:107B3000C4F20902116013E047F66071C0F2060159
:107B40000A6840F20403C4F209031A6047F654714C
:107B5000C0F206010A6840F23C03C4F209031A604D
:107B600040F2D453C1F200031870704740F2D4536E
:107B7000C1F200031878704738B515461C46002935
:107B80004FD140F2D550C1F200000178002942D116
:107B900040F20403C4F209031A7822F001001870BD
:107BA00028464FF00001C4F2C8212DF0EBF8E0B1F7
:107BB00028464FF00001C4F2FA512DF0B1F8A0B1FF
:107BC000284629462CF08CFE01464EF2C010C4F621
:107BD000E4402CF085FF2CF051FD40F22402C4F269
:107BE000090210604FF0000208E040F22401C4F2E4
:107BF00009014CF286730B604FF0160240F204004C
:107C0000C4F20900017841F001030370017841F0EA
:107C10000203037001E04FF0000222704FF00000F9
:107C200038BD4FF0000323704FF0140038BD00BF83
:107C300010B584B048F23403C2F20903186810F09A
:107C4000020F3FD14CF2C401C4F20F010A6842F4A2
:107C500080040C6047F61473C0F20603186840F203
:107C60007001C4F20901086047F65C72C0F20602B6
:107C7000146840F21403C4F209031C604FF00004BE
:107C8000009401944FF0030202924FF005004FF070
:107C90000101234601F0ECFB40F22400C4F209008C
:107CA0004CF28671016040F20C02C4F209021460C9
:107CB00047F65073C0F20603186840F20401C4F29C
:107CC0000901086004B010BD08B5FFF7B1FF47F621
:107CD0000C70C0F2060021F0DFFA4FF0140047F6F6
:107CE0001871C0F2060140F2C852C1F2000220F041
:107CF00089FB08BD08B548F23403C2F209031968CC
:107D000011F0020F1AD140B140F2D550C1F200007B
:107D100002789AB1FFF78CFF08BD40F2D550C1F24E
:107D20000000027852B94FF00000FFF7C3FE40F2A6
:107D3000D553C1F200034FF00101197008BD00BF17
:107D400030B400F2671292B240F2CE239A4210D9B8
:107D500046F2B704CBF20B6484FB00452B184FEAC4
:107D6000E074C4EB23254FF4B47303FB150423B272
:107D700000E00346002BBCBF03F5B4731BB2A3F1B4
:107D80005B05ACB2B3F5877F08DDA3F5877347F6D3
:107D90006875C0F2060535F8133015E0B42B08DD20
:107DA000C3F5877347F66875C0F2060535F81330DA
:107DB0000AE05A2BCCBF5A3BC3F15A0347F6687509
:107DC000C0F2060535F81330B22C9CBF5B429BB263
:107DD000CB800B8040F2CE239A420FD946F2B702F5
:107DE000CBF20B6282FB00231B184FEAE072C2EB5E
:107DF00023234FF4B47202FB130000B20028BCBF6F
:107E000000F5B47000B2B0F5877F0ADDC0F5B4723A
:107E100047F66873C0F2060333F81220B42816DC64
:107E200018E0B42808DDA0F1B40047F66872C0F28B
:107E3000060232F810200AE05A28C8BFC0F1B40088
:107E400047F66873C0F2060333F8102002E0C2F16F
:107E5000000082B24A80C2F100038B8030BC7047C0
:107E600070B4039C1D88491B5E88B21A0DB216B20D
:107E7000B0F90210B0F9062002FB06F201FB052260
:107E800002F18002B0F90010B0F9040006FB00F620
:107E900005FB016101F180014FEA212121804FEAB8
:107EA000222262801888091821805B889A1A6280D1
:107EB00070BC70472DE9F04186B007460E46144667
:107EC0001D46B2F90010B2F9022005AB009333460B
:107ED000FFF7C6FFA18820880918B4F9022004AB77
:107EE0000093384609B23346FFF7BAFFB4F90010E1
:107EF000E2886088121803AB0093384612B233460A
:107F0000FFF7AEFFA18820880918E288648812195B
:107F100002AB0093384609B212B23346FFF7A0FF16
:107F2000BDF91070BDF914108F42B4BF3846084631
:107F3000BDF90C60B042A8BF3046BDF90840A04270
:107F4000A8BF204680B28F42ACBFB8468846BDF974
:107F500012C0BDF91670BC45B4BF63463B46BDF9BF
:107F60000E108B42A8BF0B46BDF90A209342A8BF52
:107F700013469BB2BC45A8BF674628806B80B045BE
:107F8000A8BF4646A642ACBFC0EB0600C0EB04004B
:107F9000A8808F42A8BF39469142ACBFC3EB010312
:107FA000C3EB0203EB8006B0BDE8F0812DE9F04F92
:107FB000ABB005461646349C9DF8D480CDF83C8085
:107FC000B3F90000B2F90020871A0D97B3F9020047
:107FD000B6F90230C21A1592B1F800A0CDF808A087
:107FE000B1F80680CDF80C80B1F802A0B1F804B069
:107FF0004FF00007ADF8A070ADF8A270A868ADF81A
:10800000A400EB68ADF8A6300846314628AA26AB96
:10801000FFF750FF002C50D0BDF89810DDF83490D9
:1080200009FA81F2BDF89A80DDF854C00CFA88F3A1
:10803000B4F800C00FFA8CF0824209DA871ABFB296
:108040007918ADF89810BDF89C10CF1BADF89C7056
:10805000678839B28B420CDAC3EB01091FFA89F940
:10806000C844ADF89A80BDF89E80C9EB0809ADF808
:108070009E90B4F8048000FA88F0BDF99C90914479
:10808000484504DAC444C2EB0C02ADF89C20E288F7
:1080900001FA82F1BDF99E00C018814203DAD219BB
:1080A000D31AADF89E30BDF99C10002940F33384FB
:1080B000BDF99E00002840F32E84BDF89A703BB2B3
:1080C000BDF99E20D118994240F32584DDF808803F
:1080D0000FFA88F4DDF80CC00FFA8CF00FFA8AFA68
:1080E0000FFA8BFB00FB04F20BFB1A2141F30F226A
:1080F0000B924FEA00201C90CBF100084FEA082CAD
:10810000CDF87CC0CAF1000A4FEA0A2BCDF878B04E
:108110004FEA04241D9448F28108C8F28008CDF883
:10812000388047F66471C0F206011B910297AA4697
:108130003546BDF898400FFA84FBBDF99C200BEB47
:108140000200834580F294831C9EDDF82C9096FB00
:10815000F9F739B203911F9A92FBF9F006B205962E
:108160001E9F97FBF9F10AB206921D9890FBF9F653
:1081700037B20797DDF8548043440C9357462A885A
:108180006888A11A0BB2029EC6EB000C0FFA8CF1A4
:10819000DDF814A001FB0AF9039E03FB069808F121
:1081A000800ADDF81C8008FB01FC069E06FB03C369
:1081B00003F1800312B20AEB022900B2C3EB002ADA
:1081C000C9F30F23CAF30F2219B2B1F1FF3FC0F276
:1081D000418310B2B0F1FF3FC0F23C8318B2B968DE
:1081E000884280F237830FFA82F8CDF80480FE6867
:1081F0000496B04580F22E835FFA89F95FFA8AF619
:10820000C9F5807EC6F5807808FB0EFCCCF30F2AFA
:10821000CDF820A00FFA89F909FB08F8C8F30F2C54
:10822000CDF824C036B206FB0EFECEF30F2ACDF8F1
:1082300028A006FB09F94FEA19291FFA81FAD7F895
:1082400004C048F68808C44540F0AD8007F1180E18
:108250000FFA8AFC019E0CFB060C0EEB8C0813F443
:10826000004F0BD112F4004F40F02D835EF82C60CC
:10827000219600F1010088420BDB0EE04FF0000E6A
:10828000CDF884E000F10100814206DD12F4004FD8
:1082900003D1D8F80460229602E04FF00002229247
:1082A00013F4004F0BD1019B03F10103049A9A428E
:1082B00005DD0FFA8AF358F82320239202E04FF0ED
:1082C0000006239681420DDD019800F1010004991A
:1082D000814207DD0FFA8AF303F1010358F82320E6
:1082E000249202E04FF00006249608980FFA80FAD4
:1082F000DDF824C00FFA8CF0DDF828800FFA88F141
:108300000FFA89F39DF887609DF88B2000FB02F23D
:108310000AFB06229DF88F6001FB06229DF8936000
:1083200003FB06224FEA22268DF897609DF88460B1
:108330009DF8882002FB00F206FB0A229DF88C6063
:1083400006FB01229DF8906006FB03224FEA2226DD
:108350008DF894609DF885609DF8892002FB00F2FD
:1083600006FB0A229DF88D6006FB01229DF89160B4
:1083700006FB03224FEA22268DF895609DF88620A1
:108380009DF88A6006FB00F002FB0A029DF88E0051
:1083900000FB01219DF8926006FB03134FEA2322A4
:1083A0008DF896207BE248F26556B44540F02A816C
:1083B00007F1180C0FFA8AFEDDF804800EFB0806A0
:1083C00006EB460E0CEB0E0813F4004F1ED112F410
:1083D000004F40F05C821CF80E6006F01F0CCDF8D8
:1083E0004CC098F8012002F0070E4FEACE0C4CEA80
:1083F000561ECDF850E04FEAD20298F802C0CDF8F0
:1084000048C000F1010088420CDB62E200F101008B
:10841000814244DD12F4004F4FD14FF0000214921C
:108420001392129298F803C00CF01F06189698F851
:1084300004E00EF007064FEAC60646EA5C1CCDF8DB
:1084400068C04FEADE0ECDF840E098F805C0CDF8E0
:1084500064C013F4004F3ED1019B03F10103049E5D
:108460009E4241DD0FFA8AF303EB430608EB060355
:1084700018F806C00CF01F0ECDF858E093F801E094
:108480000EF007064FEAC60646EA5C1CCDF844C06B
:108490004FEADE0ECDF85CE093F802E02CE04FF0FE
:1084A000000214921392129210921A921892199238
:1084B00096461792119216921EE04FF00002149207
:1084C0001392129210921A9218921992964617923B
:1084D0001192169210E04FF0000ECDF85CE0CDF84E
:1084E00044E0CDF858E007E04FF0000ECDF85CE036
:1084F000CDF844E0CDF858E081421FDD019901F14B
:108500000101049888421FDD0FFA8AF303F1010389
:1085100003EB430108EB010618F8013003F01F08D4
:10852000707800F0070A4FEACA0C4CEA531ACDF8EB
:1085300004A04FEAD0010491B6780AE04FF000069B
:1085400004960196B04604E04FF0000604960196AA
:10855000B046089B0FFA83FA099800B2DDF828C0EC
:108560000FFA8CF10FFA89F3DDF8649000FB09F93A
:10857000DDF848C00AFB0C9901FB0E9E03FB06E6E2
:108580004FEA26268DF89760DDF860C00CFB00F6F8
:10859000DDF84CE00EFB0A66DDF858C00CFB016606
:1085A00008FB03664FEA26264FEAC6068DF894605C
:1085B000DDF8688008FB00F6DDF850E00EFB0A6687
:1085C000DDF844C00CFB0166DDF8048008FB03669F
:1085D0004FEA26264FEA86068DF89560109E06FB28
:1085E00000F002FB0A02DDF85CA00AFB0120DDF8C6
:1085F00010E00EFB03014FEA21234FEAC3068DF87A
:1086000096604CE140F265518C4540F01F8107F1C6
:1086100018010FFA8AFE019E0EFB060801EB480CBA
:1086200013F4004F0FD112F4004F40F05D8131F888
:108630001820ADF8842000F10100B96888421FDBE2
:108640004FF0FF082AE09DF884106FF304018DF8C5
:108650008410BDF884606FF34A16ADF884604FEA69
:1086600016216FF3C7018DF8851000F10100BE6877
:10867000B0420EDA12F4004F0ED14FF0000801E0C4
:108680004FF0FF08BCF80260ADF888604FF0FF0EB5
:1086900018E04FF0000801E04FF000089DF88860F6
:1086A0006FF304068DF88860BDF888206FF34A12D6
:1086B000ADF888204FEA12216FF3C7018DF88910B9
:1086C0004FF0000E13F4004F0FD1019A02F1010296
:1086D000FB689A4209DA0FFA8AF13CF81160ADF8AA
:1086E0008C604FF0FF02049214E09DF88C106FF341
:1086F00004018DF88C10BDF88C606FF34A16ADF84C
:108700008C604FEA16226FF3C7028DF88D204FF070
:1087100000030493BB68834210DD019800F101005F
:10872000F96888420ADA0FFA8AF000F101003CF891
:108730001010ADF890104FF0FF0213E09DF890601C
:108740006FF304068DF89060BDF890206FF34A1225
:10875000ADF890204FEA12236FF3C7038DF89130E4
:108760004FF00002089E0FFA86FA099B18B2DDF856
:1087700028C00FFA8CF10FFA89F300FB0EF60AFB02
:108780000866DDF8108001FB086603FB02624FEA11
:1087900022268DF897609DF8842002F01F069DF830
:1087A000882002F01F0202FB00F206FB0A269DF859
:1087B0008C2002F01F0202FB01629DF8906006F01F
:1087C0001F0606FB03224FEA22264FEAC6028DF857
:1087D0009420BDF88460C6F34516BDF88820C2F326
:1087E000451202FB00F206FB0A26BDF88C20C2F3FC
:1087F000451202FB0162BDF89060C6F3451606FB08
:1088000003224FEA22264FEA86028DF895209DF832
:1088100085604FEAD6029DF889604FEAD60606FBCE
:1088200000F002FB0A029DF88D004FEAD00606FB1D
:1088300001219DF891204FEAD20000FB03134FEA7B
:1088400023264FEAC6018DF8961028E01B9B1A6874
:10885000259224E004F10104A4B20FFA84FBBDF9CF
:108860009820BDF99C0011188B45FFF688ACBA46DC
:10887000029B03F101039AB2029213B2BDF99A006E
:10888000BDF99E1042189342FFF653AC43E000F14D
:1088900001004FF0000214921392129219E09DF819
:1088A00097000F9901FB00F0DDF838E08EFB0086A1
:1088B00033180D9E06EB0B000C99259AC3F3C713D2
:1088C000FAF76CFDC6E74FF00002219200F10100BB
:1088D000E3E44FF0000ECDF840E0CDF868E0CDF8CD
:1088E00060E0CDF864E0B7E59DF884206FF3040202
:1088F0008DF88420BDF884106FF34A11ADF8841010
:108900004FEA11266FF3C7068DF8856000F101006C
:108910004FF00008C2E62BB0BDE8F08F40F2E45300
:10892000C1F20003196848F22800C0F2060082680C
:108930000A6040F2E053C1F200031A6848F22401D1
:10894000C0F206010B68136040F2D852C1F2000277
:108950001168C068086040F2DC53C1F20003196876
:1089600048F22002C0F206021068086048F20003D4
:10897000C2F2090319686FF3D751196048F21C005D
:10898000C2F209004FF080620260704708B54FF0F4
:108990001C014FF0000201F015F908BD08B50146B1
:1089A0004FF000004FF01C0201F07EF840F2E4535B
:1089B000C1F200034CF26002C4F202021A6040F2FB
:1089C000D850C1F200004CF26401C4F2020101600F
:1089D00040F2E053C1F200034CF25C02C4F2020226
:1089E0001A6040F2DC50C1F200004CF26801C4F29F
:1089F00002010160FFF792FF08BD00BFF8B5044611
:108A00000D4648F21403C2F20903186810F4000F6F
:108A100040F0D780002C00F0D780002900F0D780EC
:108A200040F2E451C1F200010F6848F22002C0F2A6
:108A3000060216683E6040F2E053C1F20003186877
:108A4000066040F2D851C1F200010F6848F22802D6
:108A5000C0F20602D3683B6040F2DC50C1F2000075
:108A600001680E6048F20007C2F209073A686FF326
:108A70009A623A603B6843F400003860396841F01C
:108A800080723A6048F21807C2F209074FF080730B
:108A90003B6048F21C00C2F209004FF40001016083
:108AA0004FF019001BF094FE4FF0000222604FF0CF
:108AB000030000F07DFB074620604FF0030000F04C
:108AC00077FBC71927604FF0030000F071FBC7194F
:108AD00027604FF0030000F06BFBC31948BF03335E
:108AE0004FEAA307276040F2E454C1F20004206873
:108AF00048F22801C0F206018A68026040F2E053A1
:108B0000C1F200031C68266040F2D850C1F2000098
:108B100001680E6040F2DC52C1F2000213681E6070
:108B200048F20004C2F2090420686FF3D7502060B5
:108B3000216841F000722260236843F08060206069
:108B400048F21804C2F209044FF00071216048F2A3
:108B50001C03C2F209034FF080621A604FF0190043
:108B60001BF036FE4FF0000028604FF0020000F0CE
:108B70001FFB044628604FF0020000F019FB0419A7
:108B80002C604FF0020000F013FB04192C604FF032
:108B9000020000F00DFB011948BF03314FEAA104A8
:108BA0002C60FFF7BBFE4FF019001BF011FE48F2DE
:108BB0001403C2F209031A6882F40000C0F3C05023
:108BC000F8BD4FF00000F8BD4FF00100F8BD4FF0C8
:108BD0000100F8BDF8B540F20403C4F202031A68BC
:108BE00042F400211960044628B34FF47A751E46FA
:108BF00000F1FF3000F0010728461DF091FE3368B8
:108C000003F00812082A19D11BE028461DF088FE3F
:108C1000336803F00812082A10D104F1FF34284603
:108C20001DF07EFE316801F00810082806D117E01B
:108C30004FF00100F8BD4FF00100F8BD4FF000000B
:108C4000F8BD013CF4D0002FDFD028461DF068FEAF
:108C5000316801F008100828F0D1013CD5D1E7E7D0
:108C6000013CD2D1E4E700BF684620F007018D4601
:108C700019B548F2B803C2F209034FF002021A60B4
:108C80004FF47A742046FFF7A5FF0028FAD003F0CE
:108C9000AFF8BDE819408546704700BF10B54CF2EB
:108CA000C803C4F20F031A6842F00800186048F2C3
:108CB0003801C0F206010C6840F20003C4F202035E
:108CC0001C604FF064001DF02BFE48F23C02C0F225
:108CD0000602106840F20401C4F2020108604CF27E
:108CE00050301DF01DFE4FF03200FFF773FF88B9C2
:108CF00000F03CFC48F2B804C2F209044FF0020351
:108D000023604FF4FA742046FFF764FF0028FAD07E
:108D100003F06EF84FF0170003F0E0F948F66944ED
:108D2000C0F2020420464FF00F014FF0170203F08B
:108D300089F940F20400C4F20200026842F4002102
:108D400001604FF0290003F0C9F920464FF00F01F0
:108D50004FF0290203F076F910BD00BF02469CF8DF
:108D6000043043B1DCF8000040B140F21061C1F2C0
:108D7000000141F82200DCF8000050B940F2106315
:108D8000C1F2000353F8220049F64042002808BF10
:108D9000104670474FF46063C0F22773B3FBF1F1E4
:108DA00010B1012819D10CE044F21802C4F20102FA
:108DB000116044F20C00C4F201004FF000030360A4
:108DC000704748F21800C4F20100016048F20C0339
:108DD000C4F201034FF000011960704710B582B072
:108DE00000918DF80420052814D1EC464FF00000C6
:108DF000FFF7B4FF01464FF00000FFF7CBFFEC4652
:108E00004FF00100FFF7AAFF01464FF00100FFF706
:108E1000C1FF0CE048F20413C0F206031C5CEC46F0
:108E20002046FFF79BFF01462046FFF7B3FF02B045
:108E300010BD00BF10B448F28803C0F2060300EB77
:108E400080004FEA80001A18148A1B5C012B1CD189
:108E500069B18C420ED944F21800C4F201000068D6
:108E600004F1FF3300FB0131B1FBF4F404E04FF0F7
:108E7000000401E04FF6FF745068046093681968BD
:108E8000D26841EA0200186026E0022B24D103F5E3
:108E90007F70844218D849B18C420AD9C1EB812134
:108EA00004F1FF304318B3FBF4F404E04FF0000486
:108EB00001E040F2FF344CF20001C4F208010A68FC
:108EC00064F38F120A6007E04CF20003C4F2080357
:108ED0001A6861F38F121A6010BC704708B54FF022
:108EE00000000146FFF7A6FF4FF001004FF0000120
:108EF000FFF7A0FF4FF002004FF00001FFF79AFFCD
:108F00004FF003004FF00001FFF794FF4FF0040013
:108F10004FF00001FFF78EFF4FF0030343F4807121
:108F20004CF23002C4F2020211604CF23403C4F27B
:108F3000020319604FF0010141F480704CF26002AD
:108F4000C4F2020210604CF26401C4F20201086033
:108F500048F20C10C0F2060003684CF28802C4F21A
:108F6000020213604CF28C01C4F202010B604CF25D
:108F70009400C4F2020003604CF29802C4F20202B0
:108F800013604CF2AC01C4F202010B6008BD00BFDB
:108F900010B54CF2C404C4F20F04236843F020005F
:108FA0002060216841F040022260FFF797FF4FF0F8
:108FB00005004FF000010A46FFF710FF44F21403CA
:108FC000C4F20103186840F00201196048F214036A
:108FD000C4F201031A6842F00200186048F28001EE
:108FE000C0F206010A6844F24C03C4F201031A609D
:108FF00048F24C00C4F201004FF00001016048F259
:109000001012C0F20602136844F20400C4F2010018
:10901000036048F20401C4F201010B60226842F4CB
:109020008053236048F24000C0F20600016844F219
:109030000002C4F20302116040F2E850C1F20000E5
:1090400048F20011C0F2060117F010F910BD00BF80
:109050002DE9F0410E4644F21803C4F201031968E9
:1090600048F28803C0F2060300EB80004FEA80025A
:109070009F189B5C012B5AD108462BF0E3F902465E
:109080000B464FF000004FF00001C3F6F0712CF0DA
:10909000BBF84FF000024FF00003C3F6E0732BF073
:1090A000FDFF2BF0DFFB804631462BF06BFE78BBDB
:1090B00030462BF0BBFB04460D4640462BF0B6FB7A
:1090C00002460B464FF000004FF00001C3F6F0716E
:1090D0002BF09EFE02460B46204629462CF006FA4F
:1090E000C8B944F21800C4F2010000682BF0A2F9DC
:1090F00031462BF08BFC2BF099FB4FF000024FF028
:109100000003C3F6E0732BF085FE2BF055FB04E063
:109110004FF0000001E04FF6FF707B681860B86800
:109120000168FA6841EA02030360BDE8F081022B9E
:1091300033D130462BF07AFB04460D4618A3D3E911
:1091400000232CF0EFF9D8B92046294616A3D3E91D
:1091500000232CF0CBF9B0B930464FF44041C4F2B3
:109160007F412BF053FC2BF061FB4FF000024FF0DE
:109170000003C3F6E0732BF04DFE2BF01DFB04E063
:109180004FF0000001E040F2FF304CF20001C4F269
:1091900008010A6860F38F120A60BDE8F08100BF21
:1091A0009A9999999999A93F666666666666EE3FAF
:1091B00010B50446032839D840F2E850C1F2000047
:1091C0004FF0000117F06AF844F20001C4F2030105
:1091D0000B6848F24402C0F2060204EB44004FEA76
:1091E00080041019125944F20404C4F203042468E0
:1091F0001468406860F307034FF0010464F31A63D6
:109200000B601168002907DB44F20000C4F2030080
:1092100003681368002BFBDA1268C2F30B1440F2E8
:10922000E850C1F2000017F049F901E04FF0FF34B7
:10923000204610BD10B50446FFF7BAFF04EB440109
:1092400048F24403C0F2060303EB8104228902FBC7
:1092500000F040F20111C0F21001A1FB0023C01A7E
:1092600003EB5002C2F3CF2010BD00BF08B5FFF7DB
:109270009FFF2BF0DFF84FF47041C4F27F512BF0C9
:109280002FFC08BD0000000038B548F28803C0F28A
:10929000060300EB80004FEA80015A185B5C012B4B
:1092A00011D15468206844F21805C4F201052D68F4
:1092B0002BF0C0F8044628462BF0BCF801462046A7
:1092C0002BF00EFC38BD022B10D14CF20000C4F282
:1092D00008000168C1F389102BF094F806A3D3E9C4
:1092E00000232BF091FF2BF0BDFA38BD4FF00000AA
:1092F00038BD00BFAFF300800000000000F88F40D1
:109300004FF0000303604FF000007047F8B572B6ED
:1093100042F210701DF004FB4CF2A013C4F20F03D4
:109320001A7842F02000187019460C6814F0400FAB
:10933000FBD04CF20005C4F20F052E684FF0050774
:1093400067F30F362E6048F22013C0F206031A6846
:109350004CF20411C4F20F010A6048F22810C0F266
:10936000060004684CF20812C4F20F02146048F2BE
:109370001415C0F206052F684CF28006C4F20F06E1
:1093800037604CF28C03C4F20F034FF0AA041C6048
:109390004FF0550018604CF20C15C4F20F052F6801
:1093A00047F001072F6048F22415C0F206052F6828
:1093B0004CF28405C4F20F052F6048F21C15C0F270
:1093C00006052D6835601C60186048F21816C0F25A
:1093D000060636684CF2A403C4F20F031E604CF27A
:1093E000A003C4F20F031D604CF2AC03C4F20F03E0
:1093F0001C60186008684FF0010363F30400086004
:1094000011684FF0020060F3040111604CF2A812E1
:10941000C4F20F0213604CF28801C4F20F010B6812
:1094200013F4806FFBD04CF2A800C4F20F00026866
:1094300012F4806FFBD04CF20411C4F20F010B68E0
:1094400043F4807008604CF20813C4F20F031A68EA
:109450004FF0020161F309221A604CF20000C4F2DD
:109460000F0003684FF0040262F30F330360F8BD8E
:10947000F0B49DF810609DF814504FF00004032ADA
:1094800011D1069A62F3020448F21C22C0F20602CD
:10949000925D62F3C40444F02004003518BF012536
:1094A00065F3492416E06FF3020448F21C27C0F26A
:1094B0000607BE5D66F3C40444F02004003518BFFF
:1094C000012565F34924022A04D16FF3C71444F43B
:1094D000803401E044F08004012B14BF00230123F9
:1094E00063F38A2448F21C33C0F2060353F82000C9
:1094F00040F82140F0BC704748F28423C0F20603D4
:1095000053F820100A6848F2C413C0F2060353F857
:1095100020100A4048F2D423C0F2060353F820007A
:10952000824214BF00200120704700BF48F2AC13F4
:10953000C0F2060353F820004069704748F2C41394
:10954000C0F2060353F8203039B148F23C11C0F2A2
:10955000060151F820201360704748F22C22C0F217
:10956000060252F820000360704700BF70B548F251
:109570001823C0F2060319684CF20010C4F202006E
:10958000C16248F28022C0F2060214684CF2002543
:10959000C4F202052C6548F23016C0F206063368A4
:1095A000EB6448F29011C0F206010A686A6548F25D
:1095B0001424C0F2060426684CF20003C4F202032D
:1095C0005E6548F27421C0F206010A68AA6648F294
:1095D0002C14C0F206042668DE6448F2A411C0F21E
:1095E00006010A684CF28006C4F20206B26448F230
:1095F0002424C0F206042168296448F29C12C0F2B7
:1096000006021468746048F23811C0F206010A6854
:109610009A6448F2A014C0F206042168A96548F2D1
:109620002822C0F206021468EC6548F2D021C0F28C
:1096300006010A685A6448F23414C0F2060421682C
:10964000716348F29412C0F206021468EC6648F2A4
:109650008811C0F206010A68F26148F27C26C0F265
:1096600006063468446048F28C10C0F206000268B6
:109670004CF28021C4F202014A6048F21026C0F286
:1096800006063468DC6548F27820C0F206000268FD
:109690009A6648F20C21C0F206010E681E6648F276
:1096A0008414C0F206042068586648F2A812C0F27A
:1096B00006021168A96448F2CC26C0F20606346896
:1096C0006C6448F22025C0F206052868186548F247
:1096D0009812C0F20602116899654FF00000014629
:1096E000FFF72CFF48F20004C2F20904236843F498
:1096F000802626604FF001004FF00001FFF71EFFAB
:1097000048F28005C2F20905286840F480022A6008
:109710004FF002004FF00001FFF710FF296841F4FD
:1097200000032B604FF003004FF00001FFF706FF2E
:10973000266846F4003020604FF004004FF000012E
:10974000FFF7FCFE48F22006C2F20906326842F436
:10975000005131604FF005004FF00001FFF7EEFEC1
:109760002B6843F0006028604FF006004FF00001C6
:10977000FFF7E4FE326842F0800131604FF00700ED
:109780004FF00001FFF7DAFE48F24003C2F209038E
:10979000186840F002021A604FF008004FF0000114
:1097A000FFF7CCFE48F2A001C2F209010B6843F0BA
:1097B000020008604FF009004FF00001FFF7BEFE05
:1097C000226842F4000121604FF00A004FF00001CE
:1097D000FFF7B4FE236843F0806020604FF00B0079
:1097E0004FF00001FFF7AAFE226842F0807121606D
:1097F0004FF00C004FF00001FFF7A0FE236843F08C
:10980000007020604FF00D004FF00001FFF796FE52
:109810002A6842F4802129604FF00E004FF00001C9
:10982000FFF78CFE2B6843F4003028604FF00F00E8
:109830004FF00001FFF782FE226842F480112160A0
:109840004FF010004FF00001FFF778FE236843F45B
:10985000800020604FF0010015F022FB70BD00BFBA
:1098600008B5FFF783FE08BD48F2C413C0F2060333
:1098700053F8203048F28422C0F2060252F8201039
:109880000968194048F2D422C0F2060252F820209A
:10989000914207BF48F22C22C0F2060248F23C1265
:1098A000C0F2060252F820000360704708B54CF27F
:1098B000C403C4F20F031A6842F00050186048F263
:1098C0004831C0F206010A6840F23003C2F20803D0
:1098D0001A6040F21860C1F2000048F25431C0F240
:1098E000060116F0C3FC08BD2DE9F843074688467B
:1098F0001646002A52D040F21860C1F200004FF024
:10990000000116F0CBFC40F22813C2F208034FF01E
:1099100000021A6048F24430C0F20600016840F2CA
:109920002C14C2F20804216048F24035C0F206054A
:10993000D5F8009048F23833C0F206031D6840F6AF
:10994000FF7C40F2201EC2F2080E40F22410C2F248
:10995000080040F22C11C2F2080140F23014C2F2A9
:109960000804664534BF33466346CEF8008007607E
:109970000A6863F30B020A60C4F80090F61A4FEA13
:1099800083039844FF1822681542FCD1002EE8D1C9
:1099900040F21860C1F2000016F090FDBDE8F883B7
:1099A000F0B41746002A41D048F23432C0F2060221
:1099B000166840F21015C2F208052C682642FCD148
:1099C00040F20012C2F20802116040F20411C2F229
:1099D0000801086040F20810C2F208004FF00002CF
:1099E000026048F25031C0F20601086840F20C12E1
:1099F000C2F208021060116867F30B01116048F2AF
:109A00003C30C0F20600016840F21012C2F20802B7
:109A100011605BB148F24C33C0F20603186840F2A3
:109A20001011C2F208010A681042FCD1F0BC704764
:109A30004FF000034FF0020262F307034FF00700FC
:109A400060F30F234FF0050161F3174340F29002DA
:109A5000C0F22002136040F29403C0F220034FF4DE
:109A6000A0701860704700BF03685868C0F57C603C
:109A7000704700BFF0B405686C688768C66806FB6D
:109A800007454768ED1969181960B1F57C6F07D271
:109A9000521804F57C64A2428CBF0020012001E032
:109AA0004FF00000F0BC70472DE9F04F91B0074631
:109AB0000D469046002A6BD040F2840BC0F2200B7A
:109AC00040F2800AC0F2200A48F26033C0F2060376
:109AD000D3F8009040F28C04C0F2200407F03F015C
:109AE000781AC1F14006464528BF4646CBF800002B
:109AF000CAF80090402E26D0226800922368019375
:109B000020680290226803922368049320680590DD
:109B100022680692236807932068089022680992B9
:109B200023680A9320680B9022680C9223680D9397
:109B300020680E9022680F92284600AB59183246D2
:109B400035F094F91FE022682A6023686B60216871
:109B5000A9602068E86022682A6123686B61216837
:109B6000A9612068E86122682A6223686B62216823
:109B7000A9622068E86222682A6323686B6321680F
:109B8000A9632068E863BF19AD19B8EB0608A5D131
:109B900011B0BDE8F08F00BF30B583B015461C464C
:109BA0001A4601ABFFF766FF38B1019829462246F5
:109BB000FFF77AFF4FF0000001E04FF01F0003B005
:109BC00030BD00BF2DE9F04F93B0804616460D46DC
:109BD00000297AD040F2840AC0F2200A48F2643B9D
:109BE000C0F2060B40F28003C0F22003019306F09E
:109BF0003F07C7EB0609C7F14004AC4228BF2C461B
:109C0000402C05D0484602A94FF04002FFF74CFF18
:109C100002AAD71938464146224632F053FBC0B259
:109C200000284ED038464146224635F01FF9CAF882
:109C30000090DBF80010019B196040F28800C0F230
:109C40002000029A026003990160049B0360059A58
:109C5000026006990160079B0360089A02600999F7
:109C600001600A9B03600B9A02600C9901600D9BD6
:109C700003600E9A02600F990160109B0360119AB5
:109C8000026040F6E870C0F220004FF0FF31016042
:109C90004FF032001CF044FECAF8009048F25C33EA
:109CA000C0F206031868019A10604FF032001CF0F1
:109CB00037FE40F6E071C0F220010B6813F0805FC0
:109CC000FBD03619A0442D1B91D113B0BDE8F08F05
:109CD00030B583B015461C461A4601ABFFF7CAFEE5
:109CE00038B128462146019AFFF76CFF4FF000007B
:109CF00001E04FF01F0003B030BD00BF08B50346C0
:109D00000A4640F24060C1F2000048F26831C0F2F9
:109D100006011EF03DFC08BD10B540F25064C1F2D2
:109D200000044FF03A03236041F6F172C1F6FF726E
:109D3000204621469047206848B940F26460C1F24D
:109D4000000004F104014FF0100235F08FF810BD4F
:109D500008B572B648F20043C0F206031A684CF226
:109D60000410C4F20F00026048F2FC31C0F2060198
:109D70000A684CF20813C4F20F031A6048F2F83074
:109D8000C0F2060001684CF28002C4F20F021160BA
:109D90004CF28C03C4F20F034FF0AA0018604FF08E
:109DA000550119604CF20C13C4F20F031A686FF3DB
:109DB00000021A604CF2A010C4F20F00017821F0EA
:109DC0002003037040F25061C1F200014FF03902EC
:109DD0000A6041F6F173C1F6FF730846984708BD63
:109DE00070B572B640F28003C0F220034FF000025B
:109DF0001A6048F27434C0F20604256840F6E8762A
:109E0000C0F22006356048F27833C0F206034FEA0C
:109E100010301E5C4FEA11315D5C40F25064C1F2BB
:109E200000044FF0320222606660A56041F6F173D3
:109E3000C1F6FF73204621469847206880B9214625
:109E40004FF0340222606660A5604DF2C043C0F25C
:109E50000103E36041F6F172C1F6FF7220469047BC
:109E600062B640F25061C1F200010868002814BFD8
:109E70000220002070BD00BFF8B507460D4616460B
:109E800072B648F27833C0F206034FEA1132985C9A
:109E900089194FEA11341B5D40F25064C1F200048D
:109EA0004FF0320222606060A36041F6F173C1F6A8
:109EB000FF73204621469847206888B921464FF015
:109EC000330222606560A760E6604DF2C043C0F2D5
:109ED0000103236141F6F172C1F6FF7220469047FB
:109EE00040F25061C1F200010878002814BF02203E
:109EF000002062B6F8BD00BF08B540F26461C1F24F
:109F000000014FF0100234F0B1FF4FF0100008BD17
:109F100008B545F62040C1F2000046F22002C1F229
:109F20000002131A4FF0FF314FEAA30201F0CEFFF7
:109F300015F004FD02F096FB4FF0000008BD00BFD5
:109F4000BFF36F8F704700BF032826D8DFE800F00B
:109F5000020B141D4CF2C400C4F20F00026842F060
:109F60000201016070474CF2C400C4F20F000168A6
:109F700041F00403036070474CF2C401C4F20F01C6
:109F80000B6843F480020A6070474CF2C403C4F2C9
:109F90000F031A6842F400001860704711B10129DC
:109FA0002CD116E040F28463C1F200031968022943
:109FB00009D040F28460C1F200000368042B14BF92
:109FC0000023012301E04FF0010313704FF0000064
:109FD000704740F28461C1F200010B68012B07D188
:109FE00040F29C60C1F2000003684FF000019960EC
:109FF0004FF0010010704FF0000070474FF000006C
:10A0000010704FF014007047684620F007018D462D
:10A0100001B448F24443C0F20603186840F25012FB
:10A02000C2F2080211680842FCD140F29463C1F206
:10A03000000318680268026040F24C13C2F2080381
:10A0400018684FF0010161F30B00186040F25013E3
:10A05000C2F208031A680A431A6040F27462C1F23D
:10A060000002106840F28063C1F200031968401AD0
:10A0700040F27861C1F20001086012681A6040F293
:10A080008463C1F200034FF00200186001BC8546F2
:10A09000704700BF684620F007018D4601B440F2CA
:10A0A0009C63C1F2000318680268026040F2986184
:10A0B000C1F200010B681A690AB1006B00E0C06AC6
:10A0C00040F28461C1F200010B683BB940F2846246
:10A0D000C1F200024FF00303136011E040F280620E
:10A0E000C1F200021168431A40F27862C1F2000224
:10A0F000136040F28463C1F200034FF00401196061
:10A1000040F28061C1F20001086001BC85467047E1
:10A1100010B540F28463C1F200031968022904D02B
:10A12000042914D0012942D129E040F28463C1F20C
:10A1300000034FF0000440F27861C1F200011C609E
:10A1400008681A68002AFAD12AF074F910BD40F2A2
:10A150008463C1F200034FF0030440F27861C1F25E
:10A1600000011C6008681A68032AFAD12AF062F913
:10A170004EF2C011C4F6E4412AF0B2FC10BD68B141
:10A1800040F29C63C1F2000319684FF0000001F136
:10A19000080101F03DFE2AF04DF910BD40F29C602F
:10A1A000C1F20000026890682AF044F910BD4FF037
:10A1B000000010BD10B5144611B1012910D107E0FF
:10A1C0004FF00000FFF7A4FF20604FF0000010BD2B
:10A1D0004FF00100FFF79CFF20604FF0000010BD22
:10A1E0004FF0140010BD00BFF0B585B040F29C6385
:10A1F000C1F200031A6848F21441C0F206010D686A
:10A20000556040F29463C1F200031A685560054638
:10A21000002800F03E8140F29860C1F2000003681F
:10A22000187999684FF0000400940194DA6802925A
:10A230004FF003022346FFF71BF940F28461C1F29D
:10A2400000010C6040F28060C1F200000460042D47
:10A2500023D140F29C61C1F20001086823464FF00F
:10A26000020262F3010340F29861C1F200010A6840
:10A27000116961F38303036744618462C46048F237
:10A280008842C0F206021168416040F28460C1F267
:10A2900000004FF001030360FBE0052D3DD140F2CB
:10A2A0009C65C1F200052C6840F29865C1F200057A
:10A2B000286803684AF29500C0F202004FF00F01CF
:10A2C00048F24C42C0F20602D25601F0BBFE48F200
:10A2D0004841C0F20601086820674FF0000363613F
:10A2E0002A68116911B101290DD106E048F2AC428A
:10A2F000C0F206021168A16205E048F2A840C0F26F
:10A3000006000368A3624FF00000E06048F28C434F
:10A31000C0F206031A686260BBE040F29C64C1F2BE
:10A320000004266840F29467C1F200073C684FF0D1
:10A3300000034FF0020262F3010340F29861C1F2A0
:10A3400000010868076967F3830333674FF0000370
:10A350007361B362F360336148F25042C0F20602A7
:10A360001768776040F25011C2F208010B6040F2AA
:10A370004810C2F20800036048F2B043C0F206037E
:10A38000196840F24C12C2F20802116006F1080688
:10A3900040F24010C2F20800066040F24416C2F2D9
:10A3A000080640F27463C1F20003336048F2A4412E
:10A3B000C0F206010A6840F27C60C1F20000066843
:10A3C000032E2FD8DFE806F0020D18234CF2C41339
:10A3D000C4F20F03196841F0010018604FF0000348
:10A3E00022E04CF2C413C4F20F03196841F00400D8
:10A3F00018604FF0020317E04CF2C413C4F20F03CD
:10A40000196841F0100018604FF004030CE04CF2A2
:10A41000C413C4F20F03196841F4804018604FF070
:10A420000E0301E04FF0000363F3450240F25011C8
:10A43000C2F208010A604AF20900C0F202004FF0BD
:10A44000000148F24C42C0F20602925701F0FAFDB8
:10A4500048F24046C0F206063068206748F2A04342
:10A46000C0F20603196861614FF00006A66248F267
:10A470000442C0F2060252F825004EF2C011C4F6A2
:10A48000E4412AF0C3FA2AF0F9F8A061E6602661F7
:10A49000676005B0F0BD00BF10B54FF000041C7040
:10A4A00049B9052A0AD84FF0010119701046FFF783
:10A4B0009BFE204610BD4FF0140010BD4FF016005B
:10A4C00010BD00BF08B54FF00000FFF78DFE08BDBE
:10A4D00038B504460D4640F29861C1F2000148F2D9
:10A4E0001840C0F206000860012D03D1012A01D1F5
:10A4F000122B01D001F088FC40F27C63C1F2000312
:10A500001C6048F29040C0F2060050F8252040F24E
:10A510009C61C1F200010A6050F8240040F294638B
:10A52000C1F2000318602846FFF70EFD2046FFF732
:10A530000BFD4CF2020048F25441C0F2060140F219
:10A540008862C1F200021DF05DFF38BD4CF280133D
:10A55000C4F20F03186840F2A062C1F200024FF08B
:10A5600000011170C3B203F00400C2B23AB140F26C
:10A57000A061C1F200014FF020020A702DE003F04B
:10A580001001C8B238B140F2A063C1F200034FF02D
:10A590000100187021E013F0010F07D040F2A06114
:10A5A000C1F200014FF080020A7016E003F00202CF
:10A5B000D1B239B140F2A063C1F200034FF04000C4
:10A5C00018700AE003F00803D8B230B140F2A0617D
:10A5D000C1F200014FF002020A704CF28013C4F283
:10A5E0000F034FF0FF30186045F61441C1F200012F
:10A5F0000A6840F2A463C1F200031A60704700BF0A
:10A6000040F2A063C1F200031878704730B444F2FE
:10A610001402C4F2020244F21805C4F202051368DF
:10A620002C6811688B42FAD129688C42F7D103F06B
:10A630003F020260C3F305214160C3F3044282601C
:10A64000C3F30263836104F01F01C160C4F30322FA
:10A6500002F1FF330361C4F30B44A4F26C74446150
:10A6600030BC704700B58BB0014601A84FF0240202
:10A6700034F0FCFB01A833F005FD44F20803C4F2FA
:10A6800002031A7822F001001870197841F00202D2
:10A690001A7044F22000C4F202000199016044F2F1
:10A6A0002400C4F20200029A026044F22801C4F2BB
:10A6B00002010398086044F23001C4F20201079AD3
:10A6C0000A6044F22C00C4F2020004990160059A69
:10A6D00002F1010244F23800C4F20200026006995D
:10A6E00001F26C7244F23C00C4F20200026019787C
:10A6F00041F001021A70187820F0020119700BB0B5
:10A7000000BD00BF10B582B04CF2C403C4F20F0309
:10A710001A6842F40070186044F20801C4F20201A1
:10A720000B6813F0010F00F0888044F20802C4F2B5
:10A730000202106810F0020F7FD144F20C01C4F243
:10A7400002010A6848F2E443C0F206031868824234
:10A7500073D144F21001C4F202010A68002A6CD1DC
:10A7600044F23C03C4F20203186840F2D9718842F3
:10A7700051D862E001996FEA0104A0420FD148F27A
:10A78000DC42C0F20602136844F20801C4F202017E
:10A790000B6044F24004C4F20204206010E048F26E
:10A7A000E042C0F20602106844F20803C4F2020359
:10A7B000186044F24001C4F202014FF000040C6042
:10A7C0004FF0000444F20C00C4F20200046044F2B2
:10A7D0001002C4F20202146048F2B840C0F206004F
:10A7E000FFF740FF44F24403C4F202031C6044F24A
:10A7F0004801C4F202010C6044F24C00C4F20200B1
:10A80000046044F25002C4F20202146044F25403A1
:10A81000C4F202031C6044F20001C4F202014FF0D2
:10A82000FF30086048F2E442C0F20602116844F2C8
:10A830000C03C4F20203196014E048F2E844C0F2C9
:10A840000604226844F20803C4F202031A60F5F712
:10A8500007FD69464FF00802FFF726F90098002827
:10A8600088D19CE702B010BD4FF0000361F31003E4
:10A8700060F3514344F24002C4F20202136048F212
:10A88000B440C0F20600016844F20803C4F20203B7
:10A890001960704700B583B04FF00003009360F378
:10A8A00041038DF80230009861F3100000906FEAC8
:10A8B00000010191F5F7D4FC024668464FF008010B
:10A8C000FFF780F94FF0010003B000BD48F2EC4300
:10A8D000C0F20603195C48F2DC52C0F206024FF0E7
:10A8E0002C0000FB0123996848F2D852C0F20602FE
:10A8F00010680860704700BFF8B548F2DC57C0F236
:10A90000060748F2EC44C0F20604255C4FF02C0622
:10A9100006FB05FE07EB0E0547F2E004C0F27204E9
:10A92000B4FBF1F14FF08004EE68346057F80E602C
:10A930008FB237606E68C1F307213160E9694FF06B
:10A94000F0060E606FF3C714A3F1050363F301046F
:10A950009DF8183013F1FF3118BF012161F3820413
:10A96000131C18BF012363F3C30448F2D051C0F293
:10A9700006018A5C62F30514EB681C60FFF7A6FF12
:10A98000F8BD00BF38B548F2EC43C0F206031B5CCB
:10A9900003EB830440F2A862C1F2000202EBC4029E
:10A9A00082F8211014693CB140F2A865C1F200059B
:10A9B0001346D2699B69A04738BD00BFF8B506466B
:10A9C0000F4648F2EC43C0F206031D5C05EB850020
:10A9D00040F2A864C1F2000404EBC004D4F810C033
:10A9E000BCF1000F07D0E2698A4204D030464FF034
:10A9F0000001A369E047E76163695BB105EB85008E
:10AA000040F2A862C1F2000202EBC00230463946B1
:10AA10009269984794F8201079B127696FB105EBD6
:10AA2000850540F2A863C1F2000303EBC50530467B
:10AA300094F82110E269AB69B847F8BD38B505460E
:10AA400040F2A862C1F2000200EB80034FEAC300AB
:10AA500014184FF0000184F8221013584BB148F23B
:10AA6000CC52C0F20602505DA169984794F82200CA
:10AA700040B9636833B148F2CC51C0F20601485D79
:10AA8000A169984738BD00BF2DE9F8430446074641
:10AA900048F2DC55C0F206054FF02C0303FB0055CD
:10AAA000A868026812F0010F42D104EB840140F261
:10AAB000A868C1F2000808EBC1082E693168C2F32A
:10AAC000420648F2CC59C0F20609CBB2C3F3800269
:10AAD00003F00800C1B211B142F00202D2B203F099
:10AAE0000203D8B208B142F0040206F1FF33052B8D
:10AAF0001ED8DFE803F01A03031D1D03D8F808C0B1
:10AB0000BCF1000F08D02868036819F80700D9B213
:10AB1000D8F81830E04701E029680B682A69116805
:10AB200011F0010FD1D1BDE8F8832046FFF786FF71
:10AB3000BDE8F883684620F007018D4601B54FF067
:10AB40000400FFF7A1FFBDE801408546704700BF44
:10AB5000684620F007018D4601B54FF00300FFF76E
:10AB600093FFBDE801408546704700BF684620F06E
:10AB700007018D4601B54FF00200FFF785FFBDE8E4
:10AB800001408546704700BF684620F007018D46AA
:10AB900001B54FF00100FFF777FFBDE801408546A2
:10ABA000704700BF684620F007018D4601B54FF0A1
:10ABB0000000FFF769FFBDE801408546704700BF10
:10ABC00010B582B08DF8071048F2EC43C0F20603CE
:10ABD000185C48F2DC51C0F206014FF02C0202FB77
:10ABE000001421690B6813F0200FFBD0246802A920
:10ABF00011F8012D226000EB800040F2A863C1F241
:10AC0000000303EBC004A08C4FF001021BF0A0FE78
:10AC1000A08404F1200402B010BD00BF30B583B0A1
:10AC20008DF8071048F2EC43C0F206031B5C48F2B3
:10AC3000DC51C0F206014FF02C0202FB03F288182F
:10AC400003EB830540F2A864C1F2000404EBC504E1
:10AC50004FF0010584F822500069046814F0200FB9
:10AC60001DBF8A589DF807101160002503EB830370
:10AC700040F2A861C1F2000101EBC304A08C0DF108
:10AC800007014FF001021BF063FEA08404F12004D1
:10AC9000284603B030BD00BF38B5054601F062F963
:10ACA000044648F2EC43C0F20603585DFFF7C6FEC7
:10ACB000204601F061F938BD2DE9F041064648F221
:10ACC000EC43C0F206031C5C04EB840040F2A86570
:10ACD000C1F2000505EBC00501F044F9804695F886
:10ACE0002010002900F08F8048F2DC57C0F20607E0
:10ACF0004FF02C0202FB0474236A4FF000071F6020
:10AD0000606807603846394694F9242001F09AF9C2
:10AD1000216A0A6867F3C7120A6030463946FFF7AE
:10AD200031FE06F1FF33042B63D8DFE803F0031B89
:10AD300033624B004CF2C403C4F20F0318686FF384
:10AD4000C300186048F2D452C0F2060211684CF2F7
:10AD50000803C4F2020319604CF20C00C4F20200B2
:10AD6000016046E04CF2C400C4F20F0001686FF3CA
:10AD70005961016048F2D453C0F2060318684CF2DE
:10AD80000002C4F2020210604CF20401C4F202019B
:10AD900008602EE04CF2C403C4F20F031A686FF38C
:10ADA00004121A6048F2D450C0F2060001684CF256
:10ADB0003C03C4F2020319604CF24002C4F20202E6
:10ADC000116016E04CF2C400C4F20F0001686FF38A
:10ADD0001861016048F2D452C0F2060213684CF2C6
:10ADE0002800C4F2020003604CF22C01C4F20201FC
:10ADF0000B60EB681BB13046E969AA6998474FF0D0
:10AE0000000285F82020404601F0B6F8BDE8F08148
:10AE10002DE9F04782B006468A469146984648F2A8
:10AE2000EC43C0F20603185C00EB800140F2A8641A
:10AE3000C1F2000404EBC10448F2DC55C0F206057F
:10AE40004FF02C0202FB005501F08CF8074606F18A
:10AE5000FF33042B68D8DFE803F0031B33674B0094
:10AE60004CF2C400C4F20F00036843F00801016013
:10AE700048F2FC42C0F2060210684CF20803C4F229
:10AE8000020318604CF20C01C4F2020108604BE0AE
:10AE90004CF2C403C4F20F03196841F000721A6047
:10AEA00048F20850C0F2060003684CF20001C4F2F8
:10AEB00002010B604CF20402C4F20202136033E0A0
:10AEC0004CF2C401C4F20F010A6842F0100008609D
:10AED00048F2FC43C0F2060319684CF23C02C4F28B
:10AEE000020211604CF24000C4F2020001601BE05B
:10AEF0004CF2C400C4F20F00016841F0807202609D
:10AF000048F20053C0F2060318684CF22801C4F25C
:10AF10000201086048F2FC42C0F2060210684CF2DE
:10AF20002C03C4F2020318609DF8282000929DF8BB
:10AF30002C000190304651464A464346FFF7DCFC60
:10AF40002B6A196841F080021A600C9820600E9BF1
:10AF5000A3600D9961600F9AE2601098A061A86AE1
:10AF60004FF00F0195F9242001F06CF86B6848F25E
:10AF70000451C0F206010A681A604FF0010084F81B
:10AF80002000384600F0F8FF02B0BDE8F08700BFAF
:10AF900048F2EC43C0F20603185C00EB800340F279
:10AFA000A860C1F2000000EBC30319615A61704749
:10AFB00048F2EC43C0F20603185C00EB800340F259
:10AFC000A862C1F2000202EBC3008160704700BFBB
:10AFD00048F2F443C0F20603185C00EB400148F26B
:10AFE0000C52C0F2060202EB01107047062812D87C
:10AFF00048F2EC43C0F20603185C00EB800140F21B
:10B00000A862C1F2000202EBC1034FF6FF70988400
:10B010004FF0010070474FF00000704706280ED82F
:10B0200048F2EC43C0F20603185C00EB800140F2EA
:10B03000A862C1F2000202EBC103988C70474FF086
:10B040000000704708B54BF2D100C0F202004FF08B
:10B050000F014FF0010200F0F5FF4CF2C403C4F2FF
:10B060000F031A6842F00200186048F2C461C0F28F
:10B0700006010A6844F27003C4F200031A6048F241
:10B08000B860C0F20600016844F21402C4F2000283
:10B09000116044F21803C4F2000345F6C050186072
:10B0A00044F20C01C4F200014FF000020A6048F2C1
:10B0B000C063C0F20603186844F20401C4F2000140
:10B0C000086048F2BC62C0F2060213680B6008BD5B
:10B0D000684620F007018D4601B544F20003C4F232
:10B0E00000031A7842F0010018701AF077F8BDE8F2
:10B0F00001408546704700BF0B4601B3032816D8B0
:10B10000DFE800F0020B0211082913D9102914D925
:10B1100020298CBF4023202311E040F2FF329342CC
:10B1200028BF13460BE0402B28BF402307E04FF019
:10B13000000304E04FF0080301E04FF0100318464D
:10B14000704700BF4FF000034CF20822C2F2080221
:10B150004FF0100111604FF0050262F30F2360F30E
:10B1600017434CF21020C2F2080003604CF2002199
:10B17000C2F208010B6813F0100FFBD0704700BF3C
:10B1800038B50D464FF00004FFF7DCFF4CF2082302
:10B19000C2F208034FF010021A604FF0010060F392
:10B1A0000F2465F317444CF21021C2F208010C6021
:10B1B0004CF20022C2F20802136813F0100FFBD009
:10B1C00038BD00BF38B505464FF00004FFF7BAFFA1
:10B1D0004CF20823C2F208034FF020021A604FF02D
:10B1E000020060F30F2465F317444CF21021C2F201
:10B1F00008010C604CF20022C2F20802136813F03E
:10B20000200FFBD04CF21420C2F20800006838BDB9
:10B210002DE9F84F4CF20023C2F20803D3F800B036
:10B220004CF23020C2F208000768002F53D041F2E0
:10B230005021C1F200010A78012A4CD94FF00004D4
:10B240004FF001054CF2382AC2F2080A41F2C04917
:10B25000C1F2000941F25C28C1F200083D4233D03E
:10B26000CAF800504FEA540619F806304FF04C0067
:10B2700000FB03864CF20021C2F208010A6812F0BA
:10B28000200FFBD04CF21423C2F208031868C0F35D
:10B29000800114F0010F0BD0F36B2BB1306A4FF02B
:10B2A00000011AF0D9FC07E04FF00100706303E0E1
:10B2B0004FF00102F2623163F16A09B9726B1AB19F
:10B2C00006F1100013F0CCF904F10104E4B24FEAE6
:10B2D0004505202CC2D14CF20823C2F20803C3F862
:10B2E00000B00BF00800C1B2002971D04FF0FE0091
:10B2F000FFF768FFC4B204F01002D3B26BB141F2A1
:10B300005220C1F200004FF00101017041F22422ED
:10B31000C1F20002106819F0C5F814F0010F36D020
:10B3200004F00800C1B2002952D004F00402D3B2E4
:10B33000B3B141F25121C1F200014FF001030B7092
:10B3400041F2BD40C1F200004FF00002027041F234
:10B350002421C1F20001086819F0A4F8BDE8F88FB3
:10B3600041F25120C1F200004FF00001017041F2A2
:10B37000BD43C1F200034FF001021A7041F22420D4
:10B38000C1F20000006819F08DF8BDE8F88F04F0F4
:10B390000203D8B2E0B141F25021C1F2000191F9AB
:10B3A0000020002A14DB41F25123C1F200034FF0C8
:10B3B0000100187041F2BD41C1F200014FF00002DE
:10B3C0000A7041F22423C1F20003186819F06AF8E8
:10B3D000BDE8F88F684620F007018D4689B500AFBB
:10B3E000FFF716FFBD46BDE889408546704700BFA0
:10B3F00070B50B46A1B34CF20822C2F208024FF41A
:10B40000807111604CF24424C2F2080425684FF0A8
:10B41000010606FA00F646EA050222604CF24821CF
:10B42000C2F2080108604CF24C20C2F2080003602E
:10B4300019F0C4FE4CF20024C2F20804C0F1040565
:10B44000236813F4807F04D119F0B8FE2A18F92A72
:10B45000F6D94CF23421C2F20801086806430E60A6
:10B4600070BD00BF10B54FF04C0303FB00F041F27C
:10B470005C21C1F200014418405828B3226A4FEA07
:10B48000420303F0FE00E168FFF7B2FF216A4FEAD2
:10B49000410000F10102D0B2A168FFF7A9FF41F21B
:10B4A0005023C1F200031978081F18BF0120606201
:10B4B0004FF00102A2624FF00003E3622363636373
:10B4C00004F1100013F0CCF810BD00BF4CF2C01313
:10B4D000C4F20F031A6860F3DF721A60704700BF8E
:10B4E00010B541F2C043C1F200031A5C40F2707320
:10B4F000C1F200031B8843FA00F010F0010F30D0B6
:10B5000041F25C23C1F200034FF04C0000FB023318
:10B5100011B1986818B927E0DA68002A27D01C6AA8
:10B520004FEA440300290CBF1946591C4CF2C014C1
:10B53000C4F20F0422686FF3DF722260C8B2FFF713
:10B5400041FE236843F000412160C0B200F00202D6
:10B55000D3B27BB900F0010100290CBF0220032007
:10B5600010BD4FF0000010BD4FF0000010BD4FF0B7
:10B57000000010BD4FF0010010BD00BF10B54CF22F
:10B58000C014C4F20F0423686FF3DF7323604FF01D
:10B59000410048F2D461C0F206010978FFF7F0FDDE
:10B5A000206840F00042226010BD00BF38B54CF268
:10B5B000C014C4F20F0423686FF3DF7323604FEAF3
:10B5C000400000F1010545F04001CDB2284648F2A7
:10B5D000E462C0F206021178FFF7D2FD284648F275
:10B5E0000073C0F206031978FFF7CAFD206840F027
:10B5F0000041216038BD00BF38B503464FEA400026
:10B6000000F10100C0B24CF2C014C4F20F0425686E
:10B610006FF3DF7525604CF20824C2F20804256838
:10B6200045F0800525604FF0020463F385044CF279
:10B630002823C2F208031C604CF22423C2F2080340
:10B640001A604CF20022C2F20802136813F0800F55
:10B6500012D101F104014CF21C24C2F208044CF294
:10B660000022C2F2080251F8043C2360136801F181
:10B67000040113F0800FF6D0FFF764FD4FF0FA00DD
:10B68000FFF760FD4CF2C011C4F20F01086840F0F2
:10B6900000420A6038BD00BFF0B583B04FEA400EEB
:10B6A0005FFA8EFC4CF2C013C4F20F031C686FF3F8
:10B6B000DF741C604CF20827C2F208073B6843F0B5
:10B6C00040043C604FF0010760F385074CF22820EE
:10B6D000C2F2080007604CF22027C2F208073B685C
:10B6E00013F4006FFBD04CF22020C2F20800076870
:10B6F0004FEA87534FEA9357BA4238BF17464CF286
:10B700000020C2F20800036813F0400F31D1032A71
:10B710002FD901F104034CF21825C2F208054CF2AE
:10B720000026C2F20806A2F10401C1F380042868D1
:10B73000194643F8040CA2F10402306810F0400FDF
:10B740005AD016E02C68194643F8044CA2F10404C0
:10B750002246306810F0400F0BD103F104032A6831
:10B76000194643F8042CA4F10402346814F0400F85
:10B7700057D04CF20023C2F20803186810F0400FB3
:10B780001ED1EAB14CF21824C2F2080420680190DC
:10B790004FF0000302F1FF3404F00104C85403F138
:10B7A000010393421ED10BE001A8185CC85403F1B9
:10B7B000010301A8C05CC85403F101039342F3D113
:10B7C0006046FFF7BFFC4FF0F200FFF7BBFC4CF206
:10B7D000C011C4F20F010A6842F000430B60384602
:10B7E00003B0F0BD002CDFD001A8185CC85403F1F1
:10B7F00001039342D8D1E3E703F10403032AB8D944
:10B80000002C9FD02868194643F8040CA2F10402CA
:10B81000306810F0400FACD103F10403032A91D833
:10B82000A7E703F10403032A8CD8A2E710B54FF071
:10B830000000FFF717FE4FF00100FFF713FE4FF077
:10B840000200FFF70FFE4FF00300FFF70BFE4FF073
:10B850000400FFF707FE4FF00500FFF703FE4FF06F
:10B860000600FFF7FFFD4FF00700FFF7FBFD4CF26E
:10B87000C014C4F20F0423686FF3DF7323604FF02A
:10B88000D8004FF00101FFF77BFC206840F0004139
:10B89000216010BDF8B5054641F25C23C1F20003FA
:10B8A000186800284AD0634C41F25C21C1F20001C3
:10B8B000CA6C002A77D004F14C0441F25C26C1F234
:10B8C0000006D6F89870002F70D004F14C0441F2B5
:10B8D0005C23C1F20003D3F8E400002869D004F12E
:10B8E0004C0441F25C21C1F20001D1F83021002A60
:10B8F00062D004F14C0441F25C26C1F20006D6F895
:10B900007C71002F5BD004F14C0441F25C23C1F246
:10B910000003D3F8C801002854D004F14C0441F2CC
:10B920005C21C1F20001D1F81422002A4DD004F1AB
:10B930004C0400F069FA4FF0080705E04FF00007EB
:10B9400041F25C24C1F200042E7A36B348F2E86377
:10B95000C0F2060353F82660317848B2B0F1FF3FD9
:10B960001ED040F27072C1F2000210884BB240FA51
:10B9700003F111F0010F0DD006F101031E4613F87B
:10B98000012B51B2B1F1FF3F0AD040FA01F111F0A1
:10B99000010FF3D196F900601AE04FF0000617E0AE
:10B9A00000F032FAF6E74FF00107CDE74FF002075B
:10B9B000CAE74FF00307C7E74FF00407C4E74FF0AB
:10B9C0000507C1E74FF00607BEE74FF00707BBE7E3
:10B9D00040F27070C1F200004FF0010303FA06F369
:10B9E000028813430380287A6989FFF785FBA060EA
:10B9F000287AA989FFF780FBE06041F2C041C1F2DB
:10BA000000018F55274647F8205B38464FF000016C
:10BA10004FF01C0233F05EFA26626868A06304F1FE
:10BA200010004FF006012A683B4612F0F9FD30463F
:10BA3000F8BD00BFA812001038B54FF0000360F346
:10BA4000060363F07F04032915D14CF2C015C4F23C
:10BA50000F0528686FF3DF7028604FF0D000214693
:10BA6000FFF78EFB4FF0D0002146FFF789FB2968D6
:10BA700041F000422A6038BD70B584B0002879D00A
:10BA80004CF2C401C4F20F010C6844F000450D6093
:10BA90004CF6F476C2F208064FF0FF33336048F2FA
:10BAA000E062C0F2060210684CF6F871C2F20801BA
:10BAB0000C680440A042FBD14FF003054CF2101675
:10BAC000C2F2080635604FF064001AF029FF4CF608
:10BAD000F473C2F208031A686FF3C3021A604FF0DE
:10BAE0000004009401944FF00106029620464FF0A6
:10BAF0001F012A462346FDF7BBFC009401940295E2
:10BB000020464FF00E012A462346FDF7B1FC009473
:10BB100001944FF00200029030464FF01E012A4679
:10BB20002346FDF7A5FC4BF2D530C0F202004FF0E2
:10BB30000F014FF0180200F085FA4FF0FF314CF280
:10BB40003823C2F2080319604CF20822C2F208023C
:10BB500011604CF20420C2F208004FF00C010160A9
:10BB600020462946FFF768FF4FF0FE003146FFF7F9
:10BB700007FB15E04FF000044FF0FE002146FFF7F1
:10BB8000FFFA20464FF00F014FF0180200F05AFA6A
:10BB90004CF2C403C4F20F031A6842F0004018606C
:10BBA00004B070BDF8B54CF2C403C4F20F031A68B8
:10BBB00042F40060186048F60C01C0F206010C68FF
:10BBC0004CF22005C2F209052C604CF20406C2F2C8
:10BBD0000906376817F0010FFBD148F20473C0F271
:10BBE00006031A684CF20000C2F2090002604CF22F
:10BBF0000011C4F20F014FF001040C6048F6040577
:10BC0000C0F206052E684CF20807C2F209073E6032
:10BC100048F21873C0F20603196848F22070C0F2A7
:10BC20000600A0F1040500F1DC0005F104026C68D7
:10BC3000216002F10405566831608542F5D14CF26D
:10BC4000A017C4F20F073B7843F001013970387830
:10BC500020F002023A703C7824F004053D7048F66A
:10BC60000806C0F2060633684CF20017C2F2090754
:10BC70003B604FF001044CF23001C2F209010C604C
:10BC80004CF23400C2F209004FF0040202604FF09F
:10BC900008054CF23806C2F2090635604CF23C0346
:10BCA000C2F209031C604CF24001C2F209010D60AE
:10BCB0004FF002064CF24400C2F2090006604CF25A
:10BCC0004802C2F209024FF00D0313604CF24C011E
:10BCD000C2F209010D604CF25000C2F20900056089
:10BCE0004FF003054CF25402C2F2090215604CF207
:10BCF0005803C2F209031D6048F60001C0F20601B4
:10BD000008684CF20415C2F2090528604CF22802BA
:10BD1000C2F2090214604CF2DC13C4F20F0340F6C5
:10BD20000521196048F21070C0F2060005684CF257
:10BD30000002C2F20902156048F20873C0F206035D
:10BD400019684CF22005C2F2090529604FF0320053
:10BD50001AF0E6FD48F20C70C0F2060002682A6094
:10BD60004FF064001AF0DCFD2B6866F3C8132B60FB
:10BD700020461AF0D5FD4CF22406C2F209063460C2
:10BD800020461AF0CDFD4FF07501316020461AF0C3
:10BD9000C7FD286864F3C810286048F21472C0F226
:10BDA0000602138840F20006CAF2000646EA033192
:10BDB0000B6820461AF0B4FD48F21C70C0F2060071
:10BDC00002682A603B6843F4002139604FF47A70BE
:10BDD0001AF0A6FD3046054A931B48BF03334FF0C7
:10BDE00000014FEAA30200F071F8F8BD030000A1C2
:10BDF00048F61003C0F206031A684EF60C50CEF255
:10BE000000000260FEE700BF08B5FFF7F1FF00BFCA
:10BE100051E8002FBFF35F8F41E80003012B3FF48F
:10BE2000F7AF1046704700BF13461A462DE9F00FD2
:10BE3000092AC0F00980B1E8F80FA0E8F80FA2F1D4
:10BE40000902092ABFF4F7AF4FF00C0303FB02F21B
:10BE50001D4B1A44974600F032B800BF00BF00BF28
:10BE600000BF0B68036000F02AB800BF00BF91E874
:10BE7000180080E8180000F022B891E8380080E847
:10BE8000380000F01CB891E8780080E8780000F0F5
:10BE900016B891E8F80080E8F80000F010B891E8D2
:10BEA000F80180E8F80100F00AB891E8F80380E8AA
:10BEB000F80300F004B891E8F80780E8F807BDE857
:10BEC000F00F70471346000056BE020013461A4694
:10BED0002DE9F00F0B460C460D460E460F468846E0
:10BEE00089468A468B46092AC0F00780A0E8F80FE9
:10BEF000A2F10902092ABFF4F9AF4FF0080303FBCE
:10BF000002F2144B1A44974600F020B800BF00BF5D
:10BF1000046000F01BB800BF80E8300000F016B8E5
:10BF200080E8700000F012B880E8F00000F00EB871
:10BF300080E8F00100F00AB880E8F00300F006B8ED
:10BF400080E8F00700F002B880E8F00FBDE8F00FDD
:10BF50007047134608BF0200EFF3118070474FF09F
:10BF6000000000BFEFF311804FF0800181F31188D2
:10BF700070474FF0000000BF80F31188704700BF8A
:10BF800030B440F20003C0F2000340F2E402C0F219
:10BF90000002D01AB0F5697F03D2274B934201D338
:10BFA00024E0FEE7254D264C621B22F003054FF0EE
:10BFB000000340F20002C1F2000240F20001C0F2B0
:10BFC000000105F10400C5F380045D589D5003F1A4
:10BFD0000403834226D109E05C589C5003F104031A
:10BFE0005C58D45003F104038342F5D14EF6085354
:10BFF000CEF2000340F20002C1F200021A604FF0DC
:10C00000B501CBF26B1145F62040C1F20000016092
:10C010004EF61453CEF200031A6842F01001196074
:10C0200030BC7047002CD7D05C589C5003F10403FF
:10C030008342D1D1DAE700BF000000000400000015
:10C04000E700000010B4034600283ED002F11004BF
:10C0500040F20000C1F2000040F82430002A0ADA61
:10C0600012F10C0F35DB02F10C024EF61850CEF235
:10C07000000011542DE04EF20014CEF200040F29FE
:10C080009CBF0901C9B24EF20043CEF20003D15465
:10C090001146002AB8BF02F11F014FEA611004EBFC
:10C0A00080014FF01F03C8F200031340002B05DA94
:10C0B00003F1FF3262F01F0303F1010358B24FF0A6
:10C0C000010202FA00F30B6003E0002AC8DB024C15
:10C0D000D5E710BC704700BF80E100E003460028B0
:10C0E000B8BF00F11F034FEA63114EF28022CEF277
:10C0F000000202EB81024FF01F03C8F2000303406D
:10C10000002B05DA03F1FF3060F01F0303F1010398
:10C1100058B24FF0010101FA00F31360704700BFFD
:10C120001EF0040F0CBFEFF30880EFF3098020E945
:10C13000F00F00F001B800BF10B5026845F6CC332F
:10C14000C1F200031A604168596082689A60C16850
:10C15000D96002691A614169596182699A61C1694C
:10C16000D961026A1A62416A5962826A9A62C16A34
:10C17000D962026B1A63416B5963826B9A63C16B1C
:10C18000D96300F1400018644EF62850CEF200004A
:10C1900002685A6435F01CFC002800F0DD8148F686
:10C1A0001400C0F2060035F02FFD4EF62C54CEF2EE
:10C1B00000042368002B05DA48F62400C0F20600CC
:10C1C00035F022FD4EF62C51CEF20001086810F039
:10C1D000020F05D048F63400C0F2060035F014FD19
:10C1E0004EF62852CEF200025478002C63D048F666
:10C1F0004C00C0F2060035F007FD4EF62853CEF293
:10C200000003597811F0010F05D048F65C00C0F228
:10C21000060035F0F9FC4EF62850CEF200004278C8
:10C2200002F00204E3B22BB148F67C00C0F2060033
:10C2300035F0EAFC4EF62851CEF20001487800F0C5
:10C240000402D4B22CB148F6A000C0F2060035F0CA
:10C25000DBFC4EF62853CEF20003597801F00800BB
:10C26000C2B22AB148F6C400C0F2060035F0CCFCD8
:10C270004EF62854CEF20004637803F01001C8B2E1
:10C2800028B148F6E400C0F2060035F0BDFC4EF6D9
:10C290002852CEF20002547804F08003D9B251B192
:10C2A0004EF63850CEF20000016848F60410C0F295
:10C2B000060035F0A9FC4EF62852CEF20002548852
:10C2C000A3B2002B5ED048F62410C0F2060035F071
:10C2D0009BFC4EF62851CEF20001488810F0010F69
:10C2E00005D048F63410C0F2060035F08DFC4EF64D
:10C2F0002852CEF20002548804F0020399B229B108
:10C3000048F66010C0F2060035F07EFC4EF628506C
:10C31000CEF20000428802F00404A3B22BB148F62A
:10C320008410C0F2060035F06FFC4EF62851CEF2B4
:10C330000001488800F0080294B22CB148F6C410FD
:10C34000C0F2060035F060FC4EF62853CEF2000332
:10C35000598801F4807082B22AB148F6F410C0F214
:10C36000060035F051FC4EF62854CEF200046388E6
:10C3700003F4007188B228B148F61020C0F206001C
:10C3800035F042FC4EF62852CEF200021478002C12
:10C3900054D048F62820C0F2060035F035FC4EF6A1
:10C3A0002853CEF20003197811F0010F05D048F69A
:10C3B0003820C0F2060035F027FC4EF62850CEF2A9
:10C3C0000000027802F00204E3B22BB148F65820D4
:10C3D000C0F2060035F018FC4EF62851CEF20001EE
:10C3E000087800F00802D4B22CB148F67020C0F2F0
:10C3F000060035F009FC4EF62853CEF200031978FA
:10C4000001F01000C2B22AB148F69420C0F2060032
:10C4100035F0FAFB4EF62854CEF20004237803F0F0
:10C420008001C8B250B14EF63452CEF2000211680B
:10C4300048F6B820C0F2060035F0E6FB45F6CC34ED
:10C44000C1F20004216A48F6E420C0F2060035F08B
:10C45000DBFB616A48F6F820C0F2060035F0D4FB39
:10C46000A16A48F60C30C0F2060035F0CDFBE16A57
:10C4700048F62030C0F2060035F0C6FB216848F6C9
:10C480003430C0F2060035F0BFFB616848F6483032
:10C49000C0F2060035F0B8FBA16848F65C30C0F287
:10C4A000060035F0B1FBE16848F67030C0F20600D6
:10C4B00035F0AAFB216948F68430C0F2060035F059
:10C4C000A3FB616948F69830C0F2060035F09CFB8A
:10C4D000A16948F6AC30C0F2060035F095FBE16981
:10C4E00048F6C030C0F2060035F08EFB216B48F6EE
:10C4F000D430C0F2060035F087FB216C48F6E830F6
:10C50000C0F2060035F080FB616B48F6FC30C0F2EB
:10C51000060035F079FBA16B48F62040C0F206001A
:10C5200035F072FB45F61443C1F200031A6848F671
:10C530004440C0F206001146126835F065FB40F633
:10C540005471C1F200010B6848F65C40C0F206006D
:10C5500019461A6835F058FBFFF756FC10BD00BFAE
:10C5600000B518F0A9FA002808BF5DF804FBEFF346
:10C570000981EFF3118221E9F40F5DF804EB41F832
:10C5800004ED094C2268002A18BF516018F006FB20
:10C590002268516851F804EBB1E8F40F82F3118876
:10C5A00081F3098870470000145C001008B54CF254
:10C5B0006150C0F202004FF0FF016FF00102FFF77F
:10C5C00041FD08BDF8B507460C461E460799089D73
:10C5D00014F0030F00D0FEE722B1A4EB8500A0F118
:10C5E000480401E004F14800012D01D8A16205E0F2
:10C5F0002A46FDF779F9A7EB8507A7624FF00003FC
:10C6000063604FF01130E0624FF0223121634FF050
:10C61000333262634FF04433A3604FF05530E06033
:10C620004FF0663121614FF0773262614FF088330D
:10C63000A3614FF09930E0614FF0AA3121624FF0D1
:10C64000BB3262624FF0CC33A363E663069820648A
:10C650004FF0807161646FF00202226005F11200F8
:10C66000F8BD00BF62B64EF60453CEF200031A685E
:10C6700042F08050186000BF2DE9F8430D46904607
:10C680001F46644627F0A6FE0646284627F0A2FE6F
:10C6900005463046616928F0B9F981462846216986
:10C6A00028F0B4F90146484628F01AF9E16828F064
:10C6B00017F9C8F800003046A16828F0A7F9064627
:10C6C0002846616828F0A2F90146304628F008F9AA
:10C6D000216828F005F93860BDE8F88341B940F2D7
:10C6E0008873C1F20003987E10704FF0000070470D
:10C6F0004FF01400704700BFF8B507460E460868B3
:10C7000028F094F810A3D3E9002328F0C7FC28F000
:10C71000A9F828F08BF804460D46384627F072FE3B
:10C720004FF000024FF00003C4F2340328F06CFD18
:10C7300002460B462046294628F06CFB28F092F86A
:10C740003060F8BDAFF30080666666666666EE3FF1
:10C7500008B54FF00100187071B940F27D73C1F255
:10C7600000031A7072B94FF0000001460246F6F756
:10C7700069FB4FF0000008BD4FF000021A704FF047
:10C78000140008BD4FF0000008BD00BF2DE9F04FB8
:10C790008DB040F28873C1F200031F68D3F8109087
:10C7A000D3F80C809E68D3F804A05D6938464946EA
:10C7B00028F02CF9044640464FF0000128F026F9F5
:10C7C000314628F023F90146204628F089F804462E
:10C7D00050464FF0000128F019F9294628F016F9C3
:10C7E0000146204628F07CF8044638464FF0000108
:10C7F00028F00CF90146284628F008F901462046A1
:10C8000028F06CF8044648464FF0000128F0FEF886
:10C810000146304628F0FAF80146204628F05EF836
:10C8200004464046514628F0F1F80146204628F0DB
:10C8300055F8044628464FF0000128F0E7F88346F3
:10C840004846594628F04AF8214628F049F90B9005
:10C8500030464FF0000128F0D9F80190514628F0F9
:10C860003DF8214628F03CF90A905046294628F028
:10C87000CDF882464846314628F0C8F80146504671
:10C8800028F02CF8214628F02BF90990584641460B
:10C8900028F024F8214628F023F908903846019919
:10C8A00028F01CF8214628F01BF907904046314635
:10C8B00028F0ACF806463846294628F0A7F8014685
:10C8C000304628F00BF8214628F00AF906900DF1C1
:10C8D000180C40F28B104FF0EB0104AA02ABFFF7EB
:10C8E000CBFE0DF1180C40F295104FF0F50105AAA2
:10C8F00003ABFFF7C1FE0498059927F0EFFF04464C
:10C9000004900298039927F0E9FF029020462EF048
:10C9100057F827F08BFF4FF000024FF00003C3F6EB
:10C92000E07328F077FA27F0DFFE40F2A871C1F239
:10C930000001086002982EF043F827F077FF4FF0CF
:10C9400000024FF00003C3F6E07328F063FA27F00B
:10C95000CBFE40F6FC02C1F2000210600DB0BDE853
:10C96000F08F00BF30B585B040F28874C1F200048A
:10C970002046FCF713F8258B4FF0000323834FF676
:10C98000FF7021464FF01C0219F0E2FFA84214BFCD
:10C9900000200120C1B2A07609B1FFF7F7FE4FF0E9
:10C9A0000003009340F2AC72C1F2000201924FF01A
:10C9B0005000029048F6A840C0F206004FF0060171
:10C9C0004DF2B932C0F2020217F0A4FD4FF00A0096
:10C9D00048F67441C0F2060140F6EC02C1F20002D2
:10C9E0001BF010FD05B030BD2DE9F04FC9B00D9220
:10C9F000002940F0C0844FF0140012904FF4C87129
:10CA000013914FF44374149415904FF0F00516955C
:10CA10004FF4E67617964FF07E5108464FF000022D
:10CA20001346F7F79DFC159F1298249025971399AC
:10CA300026912797149A28922997169B2A902B9330
:10CA40002C912D932E922F93179C309031943291EC
:10CA50003394349235944FF07F40F6F7BFF94FF09E
:10CA60000000F4F7F1FE00F1050548F6B046C0F20B
:10CA7000060600964FF000004FF005012A464FF0E1
:10CA8000FF33F5F723F84FF00000F4F7C9FE2A183A
:10CA900048F6C847C0F2060700974FF000004FF075
:10CAA00005014FF0FF33F5F711F84FF00000014694
:10CAB0004FF0FF321346F6F755F941F2883017F080
:10CAC00087FE40F27C70C1F200000178002900F07E
:10CAD00059844FF0320540F27C74C1F200042846BC
:10CAE00017F076FE2278002AF9D100F04BBC059DA4
:10CAF00055F8044F059548AA02EBC40353F8906C0F
:10CB000024AF0398C65153F88C4C39184C604FF041
:10CB10007F40F6F763F924AD039A56594FF0FF337F
:10CB200000934FF00107019706F1FF3004F1FF3148
:10CB30004FF002021346F7F787F84FF00000F4F7C2
:10CB400083FE04F10A010D184FF00000F4F772FEA5
:10CB500000EB40004219B2F5F07F88BFC0EB04053E
:10CB600048F6EC44C0F206040094049E56F8043FD4
:10CB7000049601934FF0000001462A464FF0FF3320
:10CB8000F4F7A4FF4FF0000001464FF0FF321346C8
:10CB9000F6F7E8F84FF032054FF0000710971197BD
:10CBA00099F8001031B1284617F012FE99F80000EC
:10CBB0000028F8D199F8002032B9284617F008FE6D
:10CBC00099F80040002CF8D040F27476C1F20006CB
:10CBD000306810A9FFF790FD40F27873C1F20003AE
:10CBE000186811A9FFF788FD1099119F084627F0D2
:10CBF0000DFF04463846394627F008FF0146204617
:10CC000027F06EFE06464FF0010740F6F804C1F229
:10CC100000044FF0000B3CE040F27473C1F20003DB
:10CC2000186810A9FFF768FD40F27871C1F20001A1
:10CC3000086811A9FFF760FD07F10107109802903D
:10CC4000DDF844A0014627F0E1FE804650465146FB
:10CC500027F0DCFE0146404627F042FE8046642F66
:10CC600016D9314628F08EF820B13046414627F0DB
:10CC700037FF03E04046314627F032FF27F0D6FD6C
:10CC80000DA3D3E9002328F069FCC8B9464600E0AB
:10CC9000064684F800B0217839B94FF00A084046BA
:10CCA00017F096FD20780028F9D099F80020002A86
:10CCB0003FF472AFB0E700BF1EA7E8482EFFEF3F7A
:10CCC00036AC029827F07CFC039AA050A518504679
:10CCD00027F076FC68604FF001001CF0E3FA03983F
:10CCE00000F108000390059F024B9F427FF4FFAEC6
:10CCF00002E000BF888D06004FF00004369E3046EB
:10CD000027F068FB214627F0EBFD8246379D284639
:10CD100027F060FB214627F0E3FD8146DDF8908097
:10CD2000404627F057FB214627F0DAFD8346259F32
:10CD3000384627F04FFB214627F0D2FD029006FB34
:10CD400006F027F047FB214627F0CAFD039005FBBC
:10CD500006F027F03FFB214627F0C2FD059005FBBA
:10CD600005F027F037FB214627F0BAFD049008FBB9
:10CD700006F027F02FFB214627F0B2FD069008FBB6
:10CD800005F027F027FB214627F0AAFD804607FB88
:10CD900006F027F01FFB214627F0A2FD079007FBB6
:10CDA00005F027F017FB214627F09AFD0890389CE4
:10CDB000204627F00FFB0146504627F091FD8246A2
:10CDC000399D284627F006FB0146484627F088FD96
:10CDD0008146269E304627F0FDFA0146584627F048
:10CDE0007FFD8346279F384627F0F4FA01460298D4
:10CDF00027F076FD029004FB04F027F0EBFA0146E1
:10CE0000039827F06DFD039005FB04F027F0E2FA8C
:10CE10000146059827F064FD059005FB05F027F015
:10CE2000D9FA0146049827F05BFD049006FB04F054
:10CE300027F0D0FA0146069827F052FD069006FB2F
:10CE400005F027F0C7FA0146404627F049FD804625
:10CE500007FB04F027F0BEFA0146079827F040FDD3
:10CE6000079007FB05F027F0B5FA0146089827F070
:10CE700037FD08903A9C204627F0ACFA0146504610
:10CE800027F02EFD82463B9D284627F0A3FA014657
:10CE9000484627F025FD8146289E304627F09AFA1D
:10CEA0000146584627F01CFD8346299F384627F047
:10CEB00091FA0146029827F013FD029004FB04F05A
:10CEC00027F088FA0146039827F00AFD039005FB36
:10CED00004F027F07FFA0146059827F001FD059040
:10CEE00005FB05F027F076FA0146049827F0F8FCD8
:10CEF000049006FB04F027F06DFA0146069827F02F
:10CF0000EFFC069006FB05F027F064FA0146404668
:10CF100027F0E6FC804607FB04F027F05BFA0146A9
:10CF2000079827F0DDFC079007FB05F027F052FA81
:10CF30000146089827F0D4FC08903C9C204627F036
:10CF400049FA0146504627F0CBFC09903D9D284602
:10CF500027F040FA0146484627F0C2FC0A902A9E74
:10CF6000304627F037FA0146584627F0B9FC834689
:10CF70002B9F384627F02EFA0146029827F0B0FC86
:10CF8000029004FB04F027F025FA0146039827F0ED
:10CF9000A7FC039005FB04F027F01CFA0146059856
:10CFA00027F09EFC824605FB05F027F013FA0146A8
:10CFB000049827F095FC059006FB04F027F00AFA88
:10CFC0000146069827F08CFC049006FB05F027F03C
:10CFD00001FA0146404627F083FC069007FB04F067
:10CFE00027F0F8F90146079827F07AFC079007FB2D
:10CFF00005F027F0EFF90146089827F071FC08903A
:10D000003E9F3F9CDDF8B080DDF8B49004FB07F054
:10D0100027F0E0F9514627F063FC8246384627F0B6
:10D02000D9F9099927F05CFC0646204627F0D2F989
:10D030000A9927F055FC0546404627F0CBF959469A
:10D0400027F04EFC0990484627F0C4F9029927F0D2
:10D0500047FC0A9007FB07F027F0BCF9039927F07B
:10D060003FFC834604FB04F027F0B4F9059927F050
:10D0700037FC029008FB07F027F0ACF9049927F081
:10D080002FFC049008FB04F027F0A4F9069927F080
:10D0900027FC069009FB07F027F09CF9079927F079
:10D0A0001FFC07905846314627F01AFD07465046A8
:10D0B000294627F015FD80465046314627F010FDE1
:10D0C00003900298294627F00BFD059004983146FD
:10D0D00027F006FD04900698294627F001FD0690EA
:10D0E0000798314627F0FCFC079009FB04F027F075
:10D0F00071F9089927F0F4FB294627F0F1FC089014
:10D1000030464FF00001C4F2A00127F0E9FC0646CA
:10D1100028464FF00001C4F2A00127F0E1FC029084
:10D1200009984FF00001C4F2A00127F0D9FC824613
:10D130000A984FF00001C4F2A00127F0D1FC81460B
:10D140003846314627F0CAFB09900598029927F026
:10D15000C5FB0A904046314627F0C0FB0B90039870
:10D16000029927F0BBFB0C9009980A9927F04EFC16
:10D1700004460B980C9927F049FC0146204627F0FD
:10D18000ADFB05460498514627F0A8FB0E90069883
:10D19000514627F0A3FB834640F28874C1F2000495
:10D1A0000A980E9927F032FC0F900C98594627F0F8
:10D1B0002DFC01460F9827F091FB294627F090FCA3
:10D1C00020600998594627F021FC83460B980E9958
:10D1D00027F01CFC0146584627F080FB294627F023
:10D1E0007FFC60600698314627F010FC834640467D
:10D1F000514627F00BFC0146584627F06FFB0146CD
:10D20000039827F003FC83463846514627F0FEFB7F
:10D2100082460498314627F0F9FB0146504627F034
:10D220005DFB0146059827F0F1FB0146584627F0C3
:10D2300057FB83464046049927F0E8FB8246384670
:10D24000069927F0E3FB0146504627F047FB0146CD
:10D25000029827F0DBFB0146584627F041FB2946A0
:10D2600027F03EFCA0600798494627F037FB83462D
:10D270000898494627F032FB82460A98594627F01B
:10D28000C5FB04900C98514627F0C0FB014604985A
:10D2900027F024FB294627F023FCE060099851463B
:10D2A00027F0B4FB82460B98594627F0AFFB0146A6
:10D2B000504627F013FB294627F012FC20610898FE
:10D2C000314627F0A3FB82464046494627F09EFBA5
:10D2D0000146504627F002FB0146039827F096FBD3
:10D2E00082463846494627F091FB814607983146E9
:10D2F00027F08CFB0146484627F0F0FA01460598D6
:10D3000027F084FB0146504627F0EAFA06464046DD
:10D31000079927F07BFB80463846089927F076FB73
:10D320000146404627F0DAFA0146029827F06EFBE4
:10D330000146304627F0D4FA294627F0D1FB606138
:10D340004FF0000525834FF00106A6764FF6FF70DB
:10D3500021464FF01C0219F0FBFA20832046FBF710
:10D3600015FBFFF713FA4FF07F40F5F737FD0D99E6
:10D370000E70284619E04FF000030D9A13704FF01D
:10D38000140012E048F67853C0F20603A3F1040635
:10D390000596074F04974FF00000039040F27C7110
:10D3A0008946C1F20009FFF7A2BB49B0BDE8F08F82
:10D3B000888D0600AFF300802DE9F04F85B04FF067
:10D3C000000303931D464FF0050411E0204617F0BB
:10D3D000FFF9039800F101000390B0F5FA6F07D14F
:10D3E00040F2A471C1F200014FF001020A700BE09B
:10D3F00028462946FBF702FB0028E7D104E04FF05E
:10D40000320017F0E5F90CE040F2887AC1F2000A28
:10D4100040F2A87BC1F2000B40F6FC06C1F2000608
:10D4200001964FF000000146FBF7E8FA0028E6D02D
:10D430004FF000042646254603E03E4645464FF0A1
:10D44000010403A802A9FBF7D9FA814604F10104FB
:10D45000E4B203982D18029BF61895FBF4F896FB9E
:10D46000F4F79AF81A10E9B14045B4BFC0EB0800D0
:10D47000C8EB0000BB42B4BFC3EB0703C7EB030319
:10D48000DBF8002090424CDC019801688B4248DCBC
:10D490004FF01E0017F09CF9B9F1000FC1D0042C19
:10D4A000CFD902E0B9F1000FBBD040F27474C1F2E1
:10D4B0000004C4F8008040F27875C1F200052F60C6
:10D4C00040F27C73C1F200034FF001061E7040F67B
:10D4D000F802C1F2000216701F78002FA1D04FF0A1
:10D4E000320940F27C74C1F2000440F27477C1F258
:10D4F000000740F27876C1F200061546484617F05C
:10D5000067F903A802A9FBF779FA2070039838603D
:10D51000029931604FF001032B702278002AEDD17F
:10D520007FE74FF01E0017F053F9B9F1000F84D1D7
:10D5300077E700BF2DE9F04705460C4640F2A4739B
:10D54000C1F20003187850B140F2A470C1F200009B
:10D550004FF0000303704FF00200BDE8F08740F287
:10D560007C71C1F20001087840F6F802C1F20002B5
:10D570001378A3B9002800F0B2802DB140F2807278
:10D58000C1F2000213682B60002C00F0A88040F26A
:10D590008471C1F200010A682260BDE8F08740F69C
:10D5A000F803C1F200034FF0000940F27C7CC1F2A5
:10D5B000000C40F27477C1F2000740F27871C1F2BA
:10D5C000000183F800909CF800603868D1F8008072
:10D5D0001A78002AF5D140F28873C1F20003997ECF
:10D5E000002966D026F0F6FE8146404626F0F2FE7F
:10D5F000804640F28877C1F200074846396827F034
:10D6000005FA82464046796827F000FA01465046FE
:10D6100027F066F9B96827F063F927F007F94FF0AA
:10D6200000024FF00003C3F6E07327F0F3FB27F08E
:10D630005BF8824640F28070C1F20000C0F800A0A2
:10D640004846F96827F0E2F981464046396927F0F3
:10D65000DDF90146484627F043F9796927F040F99A
:10D6600027F0E4F84FF000024FF00003C3F6E07338
:10D6700027F0D0FB27F038F8024640F28473C1F25D
:10D680000003186040F27D71C1F20001087880B19A
:10D690002EB14FF001005146F5F7D4FB0AE04FF0F0
:10D6A000000001460246F5F7CDFB4FF00000BDE853
:10D6B000F08786B12DB140F28072C1F2000213688A
:10D6C0002B605CB140F28471C1F2000108682060F7
:10D6D0003046BDE8F0873046BDE8F0873046BDE80B
:10D6E000F08700BF00F5E07003688B4203D8426802
:10D6F0009B18994202D380680028F5D1704700BF7B
:10D7000082B040F6D823C1F200031868F0B940F6A1
:10D71000D823C1F200034FF480529A605A604FF050
:10D72000FF31D9604FF4001018614FF000025A61C8
:10D7300040F60011C1F20001C1F8BC2101A880F03F
:10D74000553222F0070141F0080018604FF0010047
:10D7500002B0704701F1080313F0070F1ABF5B42D4
:10D7600003F007030023C918D21A8161C26042F096
:10D7700001034B6089184FF028024A6040F6D82315
:10D78000C1F200031969C161704700BF2DE9F04182
:10D7900004460D4640F6D823C1F20003186808B9C4
:10D7A000FFF7AEFF15F1410F55D8A169002955D0FB
:10D7B00005F12805E668B54257D240F6D822C1F2F5
:10D7C0000002D2F808802046FFF78CFF0746C168A8
:10D7D00011F0080F49D1464406F1FF335D1BB5FB3C
:10D7E000F8F000F1FF3208FB02F64FF6FE71C7F6C3
:10D7F000FF718E4288BFC8F100464FF00000F2F77B
:10D80000FDFC3D687B68ED1885422ED1C6F1000015
:10D81000F2F7F4FC06464FF00000F2F7EFFCB6F129
:10D82000FF3F22D0854220D92D1A1ED07B68581B7D
:10D830007860D4F8B021511BC4F8B011E3682046D9
:10D84000A1695A1BFFF786FF0AE04FF0FF31E16143
:10D850004FF0000504E04FF0000501E04FF0000537
:10D86000281C18BF0120BDE8F081E068E269904201
:10D87000EBD84FF00005F3E72DE9F84306460C46D8
:10D88000154601EB02084B6813F0010F40F0C6800B
:10D890000A6813F0030F00F071828C1AAD1800694A
:10D8A0008442C0F0B78071698C4200F0A0804FEADA
:10D8B000D2021F2A25D8A368E76806EBC20C0CF138
:10D8C000280C634506D0984200F24282D9688C4207
:10D8D00040F03E829F4208D14FF0010303FA02F26A
:10D8E000316821EA0201316098E0674506D0B8420C
:10D8F00000F23182B868844240F02D82DF60BB6064
:10D900008CE0D4F81890E768BC420DD0A368984228
:10D9100007D8DA68944200F0218202E0DF60BB6041
:10D920001FE0F2F799FC1CE004F11401676937B9B4
:10D9300004F11001276917B913E01F68194607F1B0
:10D9400014037A69002AF8D107F110033A69002A12
:10D95000F3D1884203D84FF00000086001E0F2F7ED
:10D960007BFCB9F1000F59D0E16901F14C0356F885
:10D97000232094420ED101F14C0146F82170CFB919
:10D98000E0694FF0010202FA00F2716821EA020137
:10D99000716043E03069814508D3D9F810108C429A
:10D9A0000CBFC9F81070C9F8147001E0F2F754FC0C
:10D9B000002F33D033699F4216D3C7F818902069DF
:10D9C00038B13269904202D33861876101E0F2F7E1
:10D9D00043FC616911B33369994202D379618F6164
:10D9E0001CE0F2F739FC19E0F2F736FC16E0D8F843
:10D9F000040000F00303032B10D1B560D8F8042015
:10DA000022F00101C8F8041045F001006060655182
:10DA1000BDE8F883F2F720FCBDE8F883316988455A
:10DA2000C0F09281D8F8040010F0020F40F0D680C8
:10DA3000B369434510D1F0682D18F560B46145F025
:10DA4000010565607269A24240F098814FF00001C3
:10DA50007161B160BDE8F8837269424509D1B1686E
:10DA60006D18B560746145F0010363606551BDE8F0
:10DA7000F88320F00707ED194FEAD7031F2B27D8AB
:10DA8000D8F80820D8F80C7006EBC30C0CF1280C61
:10DA9000624506D0914200F26681D068804540F030
:10DAA0006281974208D14FF0010101FA03F0326818
:10DAB00022EA0002326087E0674506D0B94200F2F0
:10DAC0005581BB68984540F05181D760BA607BE0D2
:10DAD000D8F81890D8F80C70B8450ED0D8F808309F
:10DAE000994207D8DA68904500F0438102E0DF6090
:10DAF000BB6021E0F2F7B0FB1EE008F11400D8F89B
:10DB000014703FB908F11000D8F8107017B913E07D
:10DB10001F68184607F114037A69002AF8D107F143
:10DB200010033A69002AF3D1814203D84FF0000173
:10DB3000016001E0F2F790FBB9F1000F44D0D8F892
:10DB40001C0000F14C0356F8232090450FD100F142
:10DB50004C0046F82070CFB9D8F81C104FF00102E5
:10DB600002FA01F2706820EA020070602CE031696C
:10DB7000894508D3D9F8100080450CBFC9F810704A
:10DB8000C9F8147001E0F2F767FBEFB133699F4207
:10DB900018D3C7F81890D8F8101039B132699142EB
:10DBA00002D339618F6101E0F2F756FBD8F8140017
:10DBB00050B13369984202D37861876104E0F2F78B
:10DBC0004BFB01E0F2F748FB45F001036360655150
:10DBD0007169A1420AD1B560BDE8F88320F0010364
:10DBE000C8F8043045F00102626065514FEAD50083
:10DBF0001F281BD806EBC00505F1280532684FF039
:10DC0000010101FA00F3134203D1134333602A46A2
:10DC100006E0AA683069824202D2F2F71DFB2A466A
:10DC2000AC60D460A260E560BDE8F8832B0A29D01F
:10DC3000B3F5803F29D2A3F580724FEA124101F07B
:10DC4000080003FA00F3A3F580524FEA124101F0F5
:10DC5000040103FA01F3A3F580424FEA124202F0F5
:10DC6000020203FA02F340188118C1EBD33303F127
:10DC7000150225FA02F000F0010103F10E0301EB99
:10DC8000430204E04FF0000201E04FF01F02E261A6
:10DC90004FF000036361236170684FF0010101FAE6
:10DCA00002F101420CD10843706002F14C0246F8C7
:10DCB000224006EB8202A261E460A460BDE8F88322
:10DCC00002F14C0356F823301F2A1ABF5208C2F142
:10DCD0001902002205FA02F200E00B46586820F013
:10DCE0000701A9421DD04FEAD2704FEA420200F16B
:10DCF000040153F821100029EFD100F1040203EBD5
:10DD000082023169914208D800F1040043F82040B2
:10DD1000A361E460A460BDE8F883F2F79DFABDE872
:10DD2000F8839A68306998420AD8824208D3D4604E
:10DD30009C60A260E3604FF00003A361BDE8F8833C
:10DD4000F2F78AFABDE8F883F2F786FABDE8F883BD
:10DD5000F2F782FA62E6F2F77FFA5FE6B868844289
:10DD60003FF4DCADDDE5F2F777FA2DE7F2F774FA70
:10DD70002AE7B96888453FF4BAAEBBE6BDE8F88348
:10DD80002DE9F84F80460C4617464B6823F00702F2
:10DD90008D1800698142C0F0728103F003010129EE
:10DDA00040F086816BE1D9B9FF2F11D907F1040149
:10DDB0008A4211D3D71B40F6D822C1F200029368E1
:10DDC0004FEA4300874294BF20460020BDE8F88F09
:10DDD0004FF00000BDE8F88F4FF00000BDE8F88F6D
:10DDE000BA4218D3D21B0F2A40F24F81E11903F037
:10DDF000010040F002031F43676042F003004860E7
:10DE00008B18586840F0010058604046FFF734FD19
:10DE10002046BDE8F88FD8F81810A94217D1D8F8D5
:10DE20000C105218974280F03381D01BE11903F097
:10DE3000010343F002021743676040F001034B60A7
:10DE4000C8F81810C8F80C002046BDE8F88FD8F8BC
:10DE50001410A94233D1D8F808105218974200F292
:10DE60001B81D11B0F2916D9E219501803F00103A9
:10DE700043F002031F43676041F0010353605150B8
:10DE8000436823F001034360C8F80810C8F8142061
:10DE90002046BDE8F88F03F0010343F00200104371
:10DEA0006060A218516841F0010353604FF0000018
:10DEB000C8F80800C8F814002046BDE8F88F16F02E
:10DEC000020F40F0ED8026F0070606EB02094F45F1
:10DED00000F2EA80C7EB090A4FEAD6061F2E27D8C0
:10DEE000AB68E96808EBC60C0CF1280C634506D05A
:10DEF000984200F2E580DA68954240F0E18099426C
:10DF00000AD14FF0010303FA06F6D8F8001021EA0F
:10DF10000601C8F8001085E0614506D0884200F28D
:10DF2000D2808868854240F0CE80D9608B6079E0ED
:10DF3000D5F818B0EE68B5420DD0AB68984207D856
:10DF4000DA68954200F0C28002E0DE60B3601FE054
:10DF5000F2F782F91CE005F114016E6936B905F19A
:10DF600010012E6916B913E01E68194606F1140354
:10DF70007269002AF8D106F110033269002AF3D140
:10DF8000884203D84FF00000086001E0F2F764F91E
:10DF9000BBF1000F46D0E96901F14C0358F823208A
:10DFA000954210D101F14C0148F82160DEB9E869D1
:10DFB0004FF0010202FA00F2D8F8041021EA02013F
:10DFC000C8F804102EE0D8F81000834508D3DBF819
:10DFD00010108D420CBFCBF81060CBF8146001E03C
:10DFE000F2F73AF9F6B1D8F810309E4218D3C6F8D5
:10DFF00018B0286940B1D8F81020904202D330619F
:10E00000866101E0F2F728F9696959B1D8F8103052
:10E01000994202D371618E6104E0F2F71DF901E0CB
:10E02000F2F71AF9BAF10F0F11D8616801F0010087
:10E0300040F0020343EA09026260A144D9F80410E7
:10E0400041F00100C9F804002046BDE8F88FE1194D
:10E05000626802F0010040F002031F4367604AF06B
:10E0600003024A6001EB0A00436843F00102426088
:10E0700040465246FFF700FC2046BDE8F88FF2F715
:10E08000EBF84FF00000BDE8F88F2046BDE8F88FB0
:10E090004FF00000BDE8F88F4FF00000BDE8F88FAA
:10E0A0004FF00000BDE8F88F4FF00000BDE8F88F9A
:10E0B000AC42E4D26E6816F0010F7FF474AEDEE776
:10E0C000F2F7CAF8AEE7F2F7C7F8ABE7B0688542F7
:10E0D0003FF43BAF3CE700BF2DE9F84FF42800F2D6
:10E0E00026820A2886BF00F10B0424F007041024BE
:10E0F0004FEAD40140F60013C1F200031D6825FA6F
:10E1000001F212F0030F35D082F0010404F0010691
:10E11000761803EBC60101F128018C68A3689942C7
:10E120000BD14FF0010101FA06F125EA010540F695
:10E130000013C1F200031D600EE040F60010C1F2B2
:10E1400000000269934205D3D868844202D1D960A5
:10E150008B6001E0F2F780F84FEAC60646F0030252
:10E160006260A619706840F00101716004F1080056
:10E17000BDE8F88F40F60010C1F2000083689C42B1
:10E1800040F24984002A00F09E804FF0020606FA11
:10E1900001F6C6F1000747EA060002FA01F2024062
:10E1A000C2F100031A4002F1FF324FEA123101F0CE
:10E1B000100622FA06F24FEA521707F008008119FA
:10E1C00022FA00F24FEA920303F004068F1922FAB2
:10E1D00006F24FEA520000F002017E1822FA01F224
:10E1E000C2F34003F71822FA03F2BF1840F60010FA
:10E1F000C1F2000000EBC70202F128029668B36882
:10E200009A420BD14FF0010202FA07F225EA020509
:10E2100040F60013C1F200031D600EE040F6001549
:10E22000C1F2000529698B4205D3D868864202D124
:10E23000DA60936001E0F2F70FF8C4EBC70544F031
:10E2400003017160341945F001006060655140F6CA
:10E250000012C1F2000293685BB340F60011C1F2F4
:10E2600000014F694FEAD30001EBC00808F128080C
:10E270000A684FF0010303FA00F0104207D110437F
:10E2800040F60011C1F20001086043460BE0D8F8E7
:10E29000083040F60011C1F200010A69934202D22F
:10E2A000F1F7DAFF4346C8F80870DF60BB60C7F8D3
:10E2B0000C8040F60010C1F200008560446106F158
:10E2C0000800BDE8F88F40F60011C1F200014B686C
:10E2D000002B00F0CB83C3F100061E4006F1FF3790
:10E2E0004FEA173202F0100027FA00F74FEA5711F1
:10E2F00001F008031E1827FA03F74FEA970202F00D
:10E300000401701827FA01F74FEA570303F00206D9
:10E31000811927FA06F7C7F3400227FA02F788188F
:10E32000C61906F14C0640F60013C1F2000353F87B
:10E330002620516821F007073F1B164608E0426877
:10E3400022F00703191BB9423CBF0F46064602469E
:10E3500010690028F3D150690028F0D140F600126E
:10E36000C1F200021069B04200F2DE8006EB04093F
:10E37000B14540F2D980D6F81880F568AE420DD08C
:10E38000B368984207D8DA68964201F05E8002E0EE
:10E39000DD60AB601FE0F1F75FFF1CE006F11401E8
:10E3A000756935B906F11001356915B913E01D68B5
:10E3B000194605F114036A69002AF8D105F1100322
:10E3C0002A69002AF3D1884203D84FF00000086080
:10E3D00001E0F1F741FFB8F1000F52D0F16901F10E
:10E3E0004C0340F60012C1F2000252F823008642AC
:10E3F00011D140F60011C1F2000141F82350EDB9EE
:10E400000846F3694FF0010101FA03F1426822EA7C
:10E410000102426035E040F60011C1F200010B69D3
:10E42000984508D3D8F8102096420CBFC8F8105071
:10E43000C8F8145001E0F1F70FFF15B340F60013D0
:10E44000C1F200031A69954219D3C5F818803069E2
:10E4500030B1824202D82861856101E0F1F7FCFE0B
:10E46000716971B140F60013C1F200031A6991425B
:10E4700002D369618D6104E0F1F7EEFE01E0F1F78E
:10E48000EBFE0F2F09D8391941F0030373607018A0
:10E49000426842F00101416041E044F003007060D5
:10E4A00047F00103C9F8043049F8077040F600113D
:10E4B000C1F20001886858B340F60012C1F20002B0
:10E4C00055694FEAD00302EBC30808F12808106829
:10E4D0004FF0010101FA03F2024207D1024340F674
:10E4E0000010C1F20000026043460BE0D8F808308B
:10E4F00040F60010C1F2000001698B4202D2F1F730
:10E50000ABFE4346C8F80850DD60AB60C5F80C8030
:10E5100040F60012C1F200029760C2F8149016F1A2
:10E52000080041F00D806FE2F1F796FE6CE210F109
:10E53000410F00F2678200F10B0424F0070440F65B
:10E540000013C1F20003D3F804C0BCF1000F00F0C7
:10E550005B82C4F10005230A00F07D87B3F5803F9C
:10E5600080F08387A3F580704FEA104101F0080026
:10E5700003FA00F3A3F580524FEA124101F00401BF
:10E5800003FA01F3A3F580424FEA124202F00202BD
:10E5900003FA02F340188118C1EBD33303F11502DB
:10E5A00024FA02F000F0010103F10E0301EB43082D
:10E5B00008F14C0240F60013C1F2000353F8222088
:10E5C000002A3DD0B8F11F0F02D106E04FF000083D
:10E5D0004FEA5807C7F1190606E04FF0000603E0BE
:10E5E0004FF01F084FF0000604FA06F64FF0000047
:10E5F0000746536823F00701091BA94202D2A1B1C3
:10E600000D46174653694FEAD67101F1040152F8DD
:10E61000212013B1934201D102E003460AB907E079
:10E6200003464FEA46061846E3E713460D461746EB
:10E63000002B41D102E04FF000073DE0002F49D10F
:10E640004FF0020202FA08F8C8F1000343EA080199
:10E6500011EA0C0C00F01387CCF1000000EA0C0268
:10E6600002F1FF304FEA103303F0100120FA01F0FD
:10E670004FEA501202F00803591820FA03F04FEA4B
:10E68000900202F00403C91820FA03F04FEA500286
:10E6900002F00203C91820FA03F0C0F3400220FA86
:10E6A00002F08B18181800F14C00B04951F82030D6
:10E6B000002BC0D1A8E113465A6822F00700011BC5
:10E6C000A9423CBF0D461F461A69002AF3D15A6978
:10E6D000002AF0D1002F00F0978140F60013C1F21C
:10E6E00000039868011BA94240F28E8140F6001297
:10E6F000C1F200021069B84200F2818107EB040800
:10E70000B84540F27C81D7F81890FE68B7420DD02A
:10E71000BB68984207D8DA68974200F0B48602E0F6
:10E72000DE60B3601FE0F1F797FD1CE007F1140114
:10E730007E6936B907F110013E6916B913E01E680B
:10E74000194606F114037269002AF8D106F1100384
:10E750003269002AF3D1884203D84FF000000860E4
:10E7600001E0F1F779FDB9F1000F52D0F96901F13B
:10E770004C0340F60012C1F2000252F82300874217
:10E7800011D140F60011C1F2000141F82360EEB949
:10E790000846FB694FF0010101FA03F1426822EAE1
:10E7A0000102426035E040F60011C1F200010B6940
:10E7B000994508D3D9F8102097420CBFC9F81060CA
:10E7C000C9F8146001E0F1F747FD16B340F60013F5
:10E7D000C1F200031A69964219D3C6F81890386935
:10E7E00030B1824202D83061866101E0F1F734FD38
:10E7F000796971B140F60013C1F200031A699142C0
:10E8000002D371618E6104E0F1F726FD01E0F1F7BA
:10E8100023FD0F2D09D82D1945F0030078607D19CF
:10E82000696841F001036B60E4E044F00300786044
:10E8300045F00103C8F8043048F805504FEAD50008
:10E840001F282AD840F60013C1F2000303EBC005CD
:10E8500005F128051A684FF0010101FA00F0104295
:10E8600007D1104340F60012C1F2000210602B469F
:10E870000AE0AB6840F60012C1F2000211698B4257
:10E8800002D2F1F7E9FC2B46C5F80880C3F80C80EA
:10E89000C8F80830C8F80C50ACE02B0A29D0B3F502
:10E8A000803F29D2A3F580714FEA114202F008009F
:10E8B00003FA00F3A3F580514FEA114202F004017C
:10E8C00003FA01F3A3F580424FEA124202F002027A
:10E8D00003FA02F340188118C1EBD33303F1150298
:10E8E00025FA02F000F0010103F10E0301EB4302EF
:10E8F00004E04FF0000201E04FF01F02C8F81C20B6
:10E900004FF00003C8F81430C8F8103040F600107B
:10E91000C1F2000043684FF0010101FA02F119420F
:10E9200012D140F60010C1F200001943416002F11B
:10E930004C0240F8228000EB8202C8F81820C8F888
:10E940000C80C8F8088055E002F14C0040F6001336
:10E95000C1F2000353F820301F2A1ABF5208C2F137
:10E960001902002205FA02F203E000BF00090010BC
:10E970000B46596821F00700854222D04FEAD27039
:10E980004FEA420200F1040153F821100029EFD1AF
:10E9900000F1040203EB820240F60011C1F2000113
:10E9A000096991420AD800F1040043F82080C8F8B0
:10E9B0001830C8F80C80C8F808801BE0F1F74CFC50
:10E9C00018E09A6840F60011C1F200010869984207
:10E9D0000ED882420CD3C2F80C80C3F80880C8F865
:10E9E0000820C8F80C304FF00003C8F8183001E0D8
:10E9F000F1F732FC17F1080040F0A28504E0F1F7CE
:10EA00002BFC01E04FF0FF3440F60013C1F200038D
:10EA10009B689C422AD81A1B40F60010C1F20000E5
:10EA200040690F2A0ED9031940F60011C1F2000106
:10EA30004B618A6042F0010159609A5044F003042E
:10EA400044600FE040F60012C1F200024FF00001F6
:10EA50009160516143F003024260C318596841F06C
:10EA600001025A6000F10800BDE8F88F40F600107E
:10EA7000C1F20000C268A24212D9131B40F6001274
:10EA8000C1F20002D36090690119916143F0010362
:10EA90004B6044F00304446000F10800BDE8F88FC7
:10EAA00040F6D825C1F200052E680EB9FEF728FE03
:10EAB00040F6D827C1F20007B96801F12F07C1F16C
:10EAC00000063D193540AC4280F0AF8440F600139B
:10EAD000C1F20003D3F8B80160B140F60012C1F2F0
:10EAE0000002D2F8B031E9188B4280F0A28488424B
:10EAF000C0F0A38440F60010C1F20000D0F8BC21A1
:10EB000012F0040F40F0DD8440F60013C1F2000360
:10EB1000996929B11846FEF7E5FD804600283FD1E6
:10EB20004FF00000F1F76AFB0746B0F1FF3F00F03D
:10EB3000BE8440F6D823C1F20003596801F1FF30CA
:10EB4000074200F0A684C7EB050C3A18C1F100019A
:10EB500011400CEB010940F60013C1F20003D3F899
:10EB6000B0314C4580F0A38409EB03004FF6FE72F0
:10EB7000C7F6FF72914500F29A84C649D1F8B821D0
:10EB80002AB1984240F29384904200F29084484621
:10EB9000F1F734FB874200F09F84074600F083BC06
:10EBA00040F60011C1F20001C868C0EB070909EB8B
:10EBB000040202EA06094FF6FE73C7F6FF73994591
:10EBC00000F275844846F1F719FB0746D8F80010A3
:10EBD000D8F804000A18974240F06584B7F1FF3F67
:10EBE00040F07A8400F063BC4FF6FE70C7F6FF7009
:10EBF000814500F2718404F130034B4540F26C848E
:10EC000040F6D826C1F20006B168C9F1000801F14A
:10EC10002F021019C9EB0006C1F100031E404FF688
:10EC2000FE71C7F6FF718E4200F256843046F1F74E
:10EC3000E5FAB0F1FF3F02D0B14400F04DBC4046D0
:10EC4000F1F7DCFA00F033BC2846F1F7D7FA0746B3
:10EC50004FF00000F1F7D2FAB7F1FF3F00F038842F
:10EC6000B0F1FF3F00F03484874280F03184C7EB7D
:10EC7000000904F12800814500F22E8400F028BC30
:10EC800040F60012C1F20002C2F8B41140F60013BF
:10EC9000C1F20003D3F81880B8F1000F0DD040F690
:10ECA0000011C1F20001D1F8C001D1F8C4218318CC
:10ECB0009F4241D1784800F020BC40F60010C1F2DC
:10ECC000000002690AB1974204D240F60011C1F275
:10ECD00000010F6140F60013C1F20003C3F8C071D8
:10ECE000C3F8C4914FF00000C3F8CC0140F6D8221D
:10ECF000C1F20002116859624FF0FF321A621946E0
:10ED000001EBC00303F12803DB609B6000F101000D
:10ED100001EBC00303F12803DB609B6000F10100FD
:10ED20002028EDD140F60010C1F200003946A9F1CB
:10ED30002802FEF70FFD5EE357488068D8B10668E9
:10ED400045687519AF42F8D1D7E30268904512D3F0
:10ED50004368D11888450ED209EB0302426040F6A1
:10ED60000011C1F20001CB680846896909EB030272
:10ED7000FEF7F0FC3FE340F60010C1F2000002692C
:10ED8000974280F0C08340F60013C1F200031F6178
:10ED9000B9E3414B9B68002B00F0EC81186881427D
:10EDA000F8D1BCE31E681F60596801EB0900586088
:10EDB00007F1080313F0070F1ABF5B4203F00708BF
:10EDC0004FF00008B84406F1080717F0070F1ABF04
:10EDD0007F4207F007050025751908EB0406C8EB0C
:10EDE0000502171B44F00304C8F8044040F6001164
:10EDF000C1F20001886985420BD140F60010C1F2D2
:10EE00000000C368FF18C760866147F0010777609C
:10EE1000AAE140F60013C1F200035A6995420CD1F1
:10EE200040F60013C1F200039A68BF189F605E614C
:10EE300047F001017160F75196E1696801F0030044
:10EE4000012840F0C58021F007094FEAD9031F2BA4
:10EE500032D8A968EA6840F60014C1F2000404EB55
:10EE6000C30404F12804A14208D00A480069814281
:10EE7000C0F05B83C868854240F0578391420DD152
:10EE8000044A4FF0010101FA03F0136823EA00037A
:10EE900013609BE000090010C00A0010A24208D0D5
:10EEA000B34B18698242C0F0438393689D4240F09F
:10EEB0003F83CA60916089E0D5F818A0EC68A5424C
:10EEC00012D0A86840F60012C1F2000213699842FD
:10EED00007D3C1688D4200F02E8302E0C460A060B9
:10EEE00021E0F1F7B9F91EE005F114016C6934B9BC
:10EEF00005F110012C6914B915E00468014604F10C
:10EF000014006269002AF8D104F110002369002B73
:10EF1000F3D1974A1069814203D34FF000030B608D
:10EF200001E0F1F799F9BAF1000F4FD0E86900F16B
:10EF30004C0340F60011C1F2000151F82320954224
:10EF40000ED18B4A42F82340ECB91046EB694FF0E2
:10EF5000010101FA03F1526822EA0102426035E040
:10EF600040F60010C1F2000003699A4508D3DAF8B0
:10EF700010108D420CBFCAF81040CAF8144001E0CE
:10EF8000F1F76AF914B340F60013C1F200031969EE
:10EF90008C4219D3C4F818A0286930B1814202D834
:10EFA0002061846101E0F1F757F96B6973B140F6B4
:10EFB0000012C1F2000211698B4202D363619C61AD
:10EFC00004E0F1F749F901E0F1F746F94D444F4407
:10EFD0006A6822F00101696047F001007060F75132
:10EFE0004FEAD7031F2B26D840F60010C1F20000CD
:10EFF00000EBC30404F1280402684FF0010101FA98
:10F0000003F3134207D1134340F60010C1F200008E
:10F01000036021460AE0A16840F60010C1F200003A
:10F020000269914202D2F1F717F92146A660CE603B
:10F03000B160F46098E03B0A29D0B3F5803F29D253
:10F04000A3F580724FEA124101F0080003FA00F3C1
:10F05000A3F580524FEA124101F0040103FA01F3D3
:10F06000A3F580424FEA124202F0020203FA02F3D1
:10F0700040188118C1EBD33303F1150227FA02F0CF
:10F0800000F0010103F10E0301EB430204E04FF035
:10F09000000201E04FF01F02F2614FF000037361C4
:10F0A000336140F60010C1F2000043684FF00101E7
:10F0B00001FA02F119420FD140F60010C1F200002E
:10F0C0001943416002F14C0240F8226000EB8202D9
:10F0D000B261F660B66047E002F14C0040F6001302
:10F0E000C1F2000353F820301F2A1ABF5208C2F1A0
:10F0F0001902002207FA02F200E00B46596821F0DB
:10F10000070087421FD04FEAD2704FEA420200F157
:10F11000040153F821100029EFD100F1040203EBA0
:10F12000820240F60011C1F200010969914207D83C
:10F1300000F1040043F82060B361F660B66013E0AC
:10F14000F1F78AF810E09A6809490869834209D3FF
:10F15000824207D3D6609E60B260F3604FF0000336
:10F16000B36101E0F1F778F808F10800BDE8F88F25
:10F170000009001040F60010C1F200004146FEF701
:10F18000B1FA05684268AD18A5F12F00A5F1270373
:10F1900013F0070F1ABF5E4206F007060026861915
:10F1A00008F110018E4238BF464606F1180A40F6B3
:10F1B000001BC1F2000B58463946A9F12802FEF7A0
:10F1C000C9FA4FF01B02726006F1080C0BF5E070F3
:10F1D0000FC88CE80F00CBF8C071CBF8C4914FF08A
:10F1E0000003CBF8CC31CBF8C8C14FF00702CAEB13
:10F1F0000501A1F10501C1F3800006F11C031946C8
:10F2000041F8042B8D4200F29D810AE003F10401D4
:10F210005A600B464A6001F1080003F1040385427D
:10F22000F4D8B04500F0E780C8EB060308EB030212
:10F23000516821F00100506043F00102C8F8042039
:10F2400048F803304FEAD3001F282AD840F60012AE
:10F25000C1F2000202EBC00505F1280513684FF06A
:10F26000010101FA00F0184207D1184340F60012DC
:10F27000C1F2000210602B460AE0AB6840F60012B3
:10F28000C1F2000211698B4202D2F0F7E5FF2B4672
:10F29000C5F80880C3F80C80C8F80830C8F80C50CE
:10F2A000A9E01A0A29D0B2F5803F29D2A2F58075CB
:10F2B0004FEA154101F0080502FA05F2A2F5805067
:10F2C0004FEA104101F0040002FA00F2A2F5804179
:10F2D0004FEA114101F0020102FA01F22818411827
:10F2E000C1EBD23202F1150023FA00F101F0010066
:10F2F00002F10E0200EB420104E04FF0000101E0D8
:10F300004FF01F01C8F81C104FF00002C8F814207D
:10F31000C8F8102040F60010C1F2000042684FF01B
:10F32000010000FA01F0104212D140F60013C1F2C0
:10F3300000031043586001F14C0143F8218003EBB6
:10F340008101C8F81810C8F80C80C8F8088052E08D
:10F3500001F14C0040F60012C1F2000252F82020E8
:10F360001F291ABF4908C1F11901002103FA01F14F
:10F3700000E00246506820F00700834222D04FEAA6
:10F38000D1754FEA410105F1040052F82000002830
:10F39000EFD105F1040302EB830040F60011C1F246
:10F3A00000010B6983420AD805F1040542F8258063
:10F3B000C8F81820C8F80C80C8F808801BE0F0F7DF
:10F3C0004BFF18E0936840F60011C1F20001086994
:10F3D00082420ED383420CD3C3F80C80C2F808805B
:10F3E000C8F80830C8F80C204FF00002C8F8182000
:10F3F00001E0F0F731FF40F60010C1F20000C168F3
:10F400008C421ED2091B40F60013C1F20003D960E2
:10F41000986902199A6141F00101516044F00304B6
:10F42000446000F10800BDE8F88F4FF00000BDE82F
:10F43000F88F4FF00000BDE8F88F4FF00000BDE8F6
:10F44000F88F4FF00000BDE8F88FA86886423EF4C0
